:020000040800F2
:10000000F8BF01201901020843FB040831FB040872
:1000100045FB040851FB04085DFB040800000000D8
:1000200000000000000000000000000069FB040860
:100030006BFB040800000000EDFD0408E101002056
:10004000010002086DFB040879FB040881FB040829
:10005000ED4D050801000208AD410508B341050852
:10006000B9410508BF410508C5410508451B0508FC
:10007000551B0508651B0508751B0508851B05082C
:10008000951B0508A51B05080100020800000000DB
:10009000000000000000000000000000CB41050847
:1000A00095FB04089BFB0408ADFB0408B3FB0408A4
:1000B000B9FB0408BFFB0408C5FB0408E5200508DC
:1000C000012105081D210508392105080100020844
:1000D00001000208010300200703002000000000C7
:1000E000EF41050873FB040801000208000000004E
:1000F000000000000000000000000000B51B050823
:100100000000000001000208CDFB04080100020805
:1001100000000000000000000000000000000000DF
:10012000C51B0508D51B0508E51B0508F51B0508BB
:10013000051C050800000000000000000000000091
:1001400000000000000000000000000001000208A4
:10015000151C0508251C0508351C05080D03002085
:10016000552105087121050800000000000000006D
:10017000000000000000000000000000000000007F
:100180000000000001000208000000000000000064
:1001900001000208010002080248002343643C30C9
:1001A00000F03AB970040020054B43F82010054BCD
:1001B00001221A60044B4FF080525A60704700BF12
:1001C000A00A0020A40A002000ED00E010F4FF7F48
:1001D00002BF024B0422C3F8002E704700E100E08A
:1001E0000D4B10B51C6801341C604FF0E02304F087
:1001F00001021B69094B53F822300BB12046984786
:10020000074B1B68A34205D1BDE8104005490020FB
:10021000FFF7CABF10BD00BF50090020A80A002088
:100220004C090020A5A8040838B5334B03EB800324
:10023000D3F88441002C37D06368196889B28A06E4
:10024000E18341D5608A00283AD0A28A92B2013275
:10025000B2FBF0F500FB1522E08A92B290422FD05B
:100260001968E1835968A3890B40A17AE9B1234950
:100270000968994219D1FFF78FFFA38BDD0631D4AE
:100280000125637AA28B5B0742BFE38B23F0100347
:10029000E383E38B1A4202D0206A00F0C1F8637A4C
:1002A00035B323F00403637238BDE17AA0690129F4
:1002B000A18A89B20CBF20F811304354A282DCE736
:1002C000DA6822F02002DA60C80642BFDA6822F05B
:1002D0001002DA600A0742BFDA6822F02002DA6010
:1002E0000025CEE76268D36843F01003D360C7E708
:1002F00043F00403D7E700BF700400206804002027
:100300000120FFF791BF0220FFF78EBF0620FFF705
:100310008BBF0000114B70B500220446DA6100F07B
:1003200071F80F4D0646EB68DA030CD4EB68DB0777
:1003300044BF0123EB60E86810F4F97007D000F0C7
:1003400073F8012003E0611CEDD00CB9032070BDEF
:1003500000F058F8801BA042E5D9F7E754090020C7
:10036000003C02402DE9F843DFF8948098F81830FB
:10037000012B05460F463FD001234CF2503088F840
:100380001830FFF7C7FF0446A0B94FF0FF333B60BA
:100390002B68012B14D1287C00F03AF84CF2503035
:1003A000FFF7B8FF154A136923F0040304461361ED
:1003B00000F03EF8002388F818302046BDE8F883A6
:1003C000AE68DFF83890D5E902231344B342EFD981
:1003D000297C304600F030F84CF25030FFF79AFF9D
:1003E000D9F8103023F0FA03C9F8103010B13E608C
:1003F0000446DDE70136E6E70224DEE7003C024082
:1004000054090020014B1868704700BF50090020B4
:100410005FF800F0BDF304085FF800F07DE2020829
:100420005FF800F0FDA204085FF800F06DF2040828
:100430005FF800F029F404085FF800F0E1F3040825
:020000040802F0
:10000000FEE700000F49D1F8883043F47003C1F8CF
:1000100088300D4B1A68002042F001021A60986087
:100020001A6822F0847222F480321A60074A5A60F9
:100030001A6822F480221A60D8604FF000638B6047
:10004000704700BF00ED00E000380240103000248F
:1000500030B5002495B010252A4621460AA80494FC
:1000600029F042FD284B01941A6C42F080521A6428
:100070001B6C03F080530193019B244B029419687D
:1000800041F4404119601B68059403F44043029316
:100090000122029B4FF48033CDE908234FF4800105
:1000A00002230F22CDE90E3112930423CDE90B4533
:1000B00003920825C02213934FF4A05C4FF48053A1
:1000C00008A8CDE91052CDE906C32DF0B5F810B15E
:1000D0000F482FF0F7F9119B109A3021DB00B3FB8A
:1000E000F2F3B3FBF1F201FB1232003A1299B3FBC7
:1000F000F1F118BF012203A82FF042FF08B1054813
:10010000E7E715B030BD00BF003802400070004086
:10011000886405089A6405080446DFF82CD00B496A
:100120000B4A0C4B03E051F8040B42F8040B9A42C3
:10013000F9D300200849094A01E041F8040B914233
:10014000FBD320462FF012BBF8BF01209087060892
:100150004004002070040020700400203C0F0020A8
:1001600040F8044B40F8045B40F8046B40F8047B13
:1001700040F8048B40F8049B40F804AB40F804BB03
:1001800040F804CB40F804DB68467047024B5A69DC
:10019000026058610020704770040020024B5A69C9
:1001A00012685A61704700BF70040020024B9A69C0
:1001B000C0E900219861704770040020044A9369E7
:1001C0001968916110B15A6818461047704700BF0E
:1001D0007004002038B5054D0446AB690BB1A3424D
:1001E00000D338BD0120FFF7E9FFF6E770040020D7
:1001F000C460056146618761C0F81C80C0F820902A
:10020000C0F824A0C0F828B0C0F82CD080ED0C8B2A
:1002100080ED0E9B80ED10ABC0F808E0FFF7B6BF95
:10022000124D6C6908B50CB92FF08CFA606020464D
:10023000FFF7D0FF23686B612046C46805694669F3
:100240008769D0F81C80D0F82090D0F824A0D0F88E
:1002500028B0D0F82CD090ED0C8B90ED0E9B90ED4B
:1002600010ABD0F808E00120704700BF70040020F8
:1002700010B50021044600F0F9FA18B914B120466F
:100280000DF0C6FD10BD002100F0F0BA10B501213F
:10029000044600F0EBFA18B914B120460DF0B8FD91
:1002A00010BDFFF7E5BF10B501220C4600F002FCBF
:1002B00018B914B120460DF0ABFD10BD00F0FABB2B
:1002C00000F0BABB2DE9F0432B4C864600254FF0D9
:1002D000030CD4F89C02002101310EEB01039A08B3
:1002E00003F00303825C5B0042FA03F303F00303B1
:1002F000022BF1D0D4F8A802090100EB0E108E08F1
:1003000089B300EB860603681A0729D1D4F8A8122E
:100310005A1AC2F3011E99424FEA92174FEA4E0E43
:100320004FEA12121CD8D4F8AC12994218D9D4F85A
:100330009C8218F8071041FA0EF303F003030CFA3D
:100340000EF9012B41EA09010AD104EB450E3F2DBC
:1003500008F807109ABF0135AEF8BC22C4F8B832CD
:100360000430B042CFD12DB1013D04EB4503B3F8C9
:10037000BCE2AEE7BDE8F0837004002030B51C4C51
:10038000D4E9A953C01AC109C0F3021E6B5C012253
:1003900002FA0EF223EA02036B54D4F8B022830966
:1003A0004FEA101CB2EB901FD4F89C0288BFC4F82F
:1003B000B032C15C4FEA9C0E0CF0030303255B00D6
:1003C00005FA03F321EA030100F80E100CF1010C09
:1003D000D4F89C024FEA9C0E0CF0030310F80E10A8
:1003E0005A0041FA02F202F00302022AE7D030BDBD
:1003F0007004002021F00F0138B50B1A134A144C79
:10040000013BDB00A2FB03235B0A9A00C4E9A703BC
:100410000546C4F8AC120732A1EB831101331D4429
:1004200003EBD202C4F8A8120021C4F8A45229F0A8
:100430005BFB002301214FF0FF32C4E9AC33C4E978
:10044000D0322381A4F83C1338BD00BFF32C23FA2B
:1004500070040020024A138902331381704700BFE1
:1004600070040020024A1389023B1381704700BFC9
:1004700070040020024B1889003818BF0120704713
:1004800070040020F8B51C4D2B89002243F00103B5
:10049000C5F8B8222B81C5F8402305F1080405F5FD
:1004A000F87654F8043F1A071AD1D5F8A822981AFA
:1004B000C0F3011193424FEA901C4FEA41014FEA09
:1004C00010100DD3D5F8AC22934209D2D5F89C7206
:1004D00017F80C2042FA01F303F00303012B02D0BA
:1004E000B442DED1F8BD03238B401A4307F80C2039
:1004F000FFF7E8FEF4E700BF7004002081B3F8B511
:10050000184E0F46051F002455F8043F1A071AD14C
:10051000D6F8A822981AC0F3011C9A424FEA90110B
:100520004FEA4C0C4FEA10100DD8D6F8AC229A4284
:1005300009D9D6F89CE21EF8012042FA0CF303F028
:100540000303012B03D00134A742DDD1F8BD0323FF
:1005500003FA0CF31A430EF80120FFF7B3FEF2E79B
:10056000704700BF700400202DE9F043614ED6F8BB
:10057000B832D6F89C1283B0C3B1D6F8A0320025A9
:100580009800C6F8B85288B10024A30804F003020A
:10059000CB5C5200134103F00303032B1FD0013443
:1005A0008442F2D3D6F8B832002BEAD1D6F8B4326E
:1005B0004FF000094FEAD3080127D6F8A43213F808
:1005C00009504FEAC9043DB304F00303E8074FEABA
:1005D00094024FEA430314D46D080134F4E7204633
:1005E000FFF770FED6F8A032D6F89C120134B4EBB7
:1005F000830F4FEA8300C8D3D6F8B832002BC0D19E
:10060000D4E78A5C42FA03F303F00303012B09D019
:100610006D0804F10104D7D1C84509F1010326D0C2
:100620009946CAE7D6F8A8C223016A465CF80330A7
:100630004FF445710CEB04105BB10CF085FD009B91
:100640003BB10DF029FEDDE900010DF0FDFD0DF0DF
:1006500039FED6F8A402E30804F00701C25C07FAE9
:1006600001F122EA0102C254D6F89C12D0E7002719
:10067000BE463A46032402250FE0012806D104FABB
:1006800003F32CEA03030B704FF0010ED6F8B432DB
:1006900001329A421FD8D6F89C12900802F0030348
:1006A00011F800C05B004CFA03F000F003000228D0
:1006B00001EB920119D00328DFD105FA03F32CEAEC
:1006C000030C81F800C0D6F8B432174601329A42C2
:1006D0004FF0000EDFD93389002223F00103C6E971
:1006E000AC27338103B0BDE8F083BEF1000FEAD040
:1006F000C5E700BF70040020044B1A89002142F0B6
:100700000102C3F8B8121A81FFF72EBF700400204F
:10071000554BD3E9AA122DE9F043521A0024D3E92C
:10072000A761C0E90144C0E90344C0E9054402608F
:100730004FEA810C22462146A146A6462746254679
:1007400016F809304FEA4E0E43FA0EF303F0030396
:10075000012B02F1010255D0022B24D033BB01370B
:100760009445876004F101046DD04FEA920902F0CC
:10077000030E16F809804FEA4E0148FA01F818F006
:1007800002013BD108F0030894452DD0B8F1010FC8
:1007900004D1C3689C4288BFC46000244FEA920918
:1007A00002F0030ECCE7013545600131944541D09C
:1007B0004FEA920902F0030E16F809304FEA4E088C
:1007C00043FA08F303F003089B0718D401292CD03F
:1007D000022903D1436901334361022183698B42BA
:1007E000D2D294458161D1D1C3689C4200D9C46002
:1007F0002D013F01C0E90157BDE8F083194694453A
:100800009ED1F5E701359445456025D04FEA920920
:1008100002F0030E16F809804FEA4E0148FA01F87B
:1008200018F0020FEAD108F00308036901330361ED
:100830000121D3E701299846F7D00229CAD083695C
:100840009942CED8D0E7C368A342D0D32D013F014F
:10085000C0E90157BDE8F083026901320261826993
:10086000002AC1D18361BFE7700400202DE9F8435D
:1008700000F10F0636093FD06E4C2389E3BBB4F874
:100880003C230D46E2BBD4F8B002D4F8A072B842C3
:1008900032D24FF0010ED4F89CC20138013F6044BF
:1008A00067440021CCF1010818E04A1C964255D952
:1008B00013F00C0F42D18A1C964240F2AA8013F02A
:1008C000300F41D10132964240F2A8803F2B2ED802
:1008D000511C8E4240F2A780B8420AD008EB0009B2
:1008E00010F8013F9A07E0D013F00C0F21D101223C
:1008F000E2E7BEF1000F0FD000231846BDE8F883F1
:10090000D4E9D012914226D2D4F8B002D4F8A07221
:10091000874288BF9E46BED832F0C1FFD4F8B002ED
:10092000D4F8A072B8424FF0010EB4D3E4E700212E
:10093000D2E713F0300F0CD10122C4E703F03002EC
:10094000B2FA82F25209C1E73F2B8CBF002101218C
:10095000C2E70022BAE732F0A2FF94E74FEA890922
:10096000A9EB0201012A01F1010704D109F10103F8
:100970009B08C4F8B032D4F8B4324B4538BF4B466C
:10098000B808C4F8B43207F0030E1CF800804FEA30
:100990004E0E0123023103FA0EF343EA08038945A0
:1009A0000CF8003012D34FF0020E8808D4F89CC225
:1009B00001F003031CF800805B000EFA03F3013121
:1009C00043EA080389450CF80030EED2D4F84033EE
:1009D000D4F8A8823344C4F8403308EB071312015B
:1009E0001846002129F080F8EA074FEA0716034667
:1009F00083D50022D4F8A40248F80620F908012281
:100A0000445C07F00707BA40224342541846BDE849
:100A1000F8834FEA890909F10109A1E74FEA890939
:100A200009F102099CE74FEA890909F103090A461D
:100A300096E700BF70040020034B1A89012A02D8F0
:100A400008B1FFF79BBC704770040020034610F00C
:100A50000F001CD1164AD2F8A812994216D810B429
:100A6000D2F8AC429C420ED95B1AD2F89C429A0949
:100A7000C3F30111A25C49000A4102F00302012AFA
:100A80004FEA131305D05DF8044B70477047002000
:100A9000704701301A18910802F00302615C52009D
:100AA00041FA02F202F00302022AF2D00001EAE760
:100AB000700400202DE9F84F0F460646002800F08C
:100AC000CA80734D2C89002900F09180002C40F0E1
:100AD0009280D5F8A802D5F8A0C2301A030903F114
:100AE000010E0F31BEEB8C0F4FEA11114FEA8C0A49
:100AF00080F0B780D5F89C92A4464FF001084FEAE9
:100B00009E040EF0030B19F804404FEA4B0B44FA15
:100B10000BF404F00304022C2BD02CB90CF1010CC3
:100B20000CEB08048C4226D341455CD065D3C44409
:100B30008C4525D2002A5ED0C209D5F8A412895C62
:100B400003F007031941384601F00101FFF78EFE5B
:100B5000044600284FD04FEA0812314628F080FFA3
:100B60002B89012B02D83046FFF708FC2046BDE850
:100B7000F88F08F101080EF1010EF245BFD1D3E75D
:100B80005C1843449C421FD9980803F0030219F8EB
:100B9000007052004FF0020C01330CFA02F23A439B
:100BA0009C4209F800200FD99808D5F89C7203F0F0
:100BB000030217F800E052000CFA02F2013342EA95
:100BC0000E029C423A54EFD1D5F8B432A1EB0802A0
:100BD0009C4238BF1C46120106EB08100021C5F8E4
:100BE000B44228F081FF34462046BDE8F88F012C3E
:100BF00001D8FFF7C3FB0024B8E75C18A00804F095
:100C0000030719F800E07F004FF0030CA8EB010187
:100C10000CFA07F72EEA0707012909F8007004F11A
:100C2000010410D003EB080EA708D5F89C3204F09D
:100C30000302D95D52000CFA02F2013421EA0202E9
:100C40007445DA55F0D1D5F8B0328342CBD9C5F826
:100C5000B0023446C8E701463846BDE8F84FFFF712
:100C600005BE0129BFD029B14FF00108002A7FF449
:100C700063AFC0E7D5F89C42800903F00303590035
:100C80000322235C8A4023EA02032354DBE700BFEC
:100C90007004002010B58AB0044603A8FFF738FDA1
:100CA000DDE90430039A00900749204600F09EFFDA
:100CB000DDE9083206980549CDE90020079A20466B
:100CC00000F094FF0AB010BD84AF0508A8AF050876
:100CD0002DE9F843DFF858914749D9F8A82207468B
:100CE00000F084FFD9F8A01289006DD0DFF84481AC
:100CF000002515F03F0633D005F003067600D9F83D
:100D00009C22AB08D35C334103F00303022B63D076
:100D1000032B5FD0012B4AD1D9F8A8222B01D2583E
:100D200042455BD0354B9A425AD0354B9A425BD004
:100D3000344B9A4256D0344B9A4253D0334B9A425A
:100D400054D0334B9A4251D0324B9A4252D0324B0C
:100D50009A424DD0314B9A4214BF68224D2227E06F
:100D6000A9421ED9D9F89C022C4602E001348C42DB
:100D700008D0A20804F00303825C5B0042FA03F38C
:100D80009B07F3D0621B7F2A0BD92549920938466D
:100D900000F02CFFD9F8A03224F03F05B5EB830F0B
:100DA00012D220492A01384600F020FFA7E72E2260
:100DB0001D49384600F01AFFD9F8A0320135B5EBCD
:100DC000830F4FEA830194D338461849BDE8F843AE
:100DD00000F053BB6D22EBE73D22E9E75422E7E741
:100DE0004C22E5E75322E3E74422E1E74122DFE733
:100DF0004222DDE74622DBE7F0AF050824EC0508D8
:100E00000CE40508FCF40508CCF4050834E10508F9
:100E1000C0E00508B4E8050850E9050890ED0508AC
:100E20000CB0050828B0050830B00508ECAF05087F
:100E30007004002044F60508064A0346506A1A6802
:100E40004168C1F31E018A4202D3521A1A607047E8
:100E50000068F5E770040020014441F20553884220
:100E600004D398B2012838BF0120704710F8012B35
:100E700003EB43135340F2E7034B044A5A62002248
:100E8000C3F8F421704700BF700400203425060821
:100E90002DE9F04781460F46002943D0FFF7DCFFDC
:100EA000214B5C6A82460CB9204637E094F9073042
:100EB000E668002B06F1FF364FF0000516DB013621
:100EC00004F11808B54215D32468ECE705EB0608D1
:100ED0004FEA580808F106033A4654F823104846EA
:100EE00028F066FE0028CCBF45464646731B012B02
:100EF000ECD8E4E7236933F815309A4510D16369DB
:100F00005B5D9F420CD158F825003A46494628F0CF
:100F100017FE28B96068C0F31E002844BDE8F087BA
:100F20000135CFE70120F9E7700400202DE9F843EF
:100F300080460F46FFF7ACFF002840F09280FF2F5D
:100F400003D9494949480CF063F9494DD5F8F431C2
:100F50007E1CABB1D5E97E1232448A422CD90246BE
:100F600031441846FFF7AAF9D5F8F4310446E0B940
:100F70000246D5F8FC111846FFF7A0F9C5F8F44170
:100F8000802E344638BF80242046FFF77CF9034684
:100F9000C5F8F401B8BB3046FFF775F90346C5F84C
:100FA000F40178BB30460CF033FFD5F8F821324419
:100FB000C5F8F821002BE3D0D5F8FC219C18324469
:100FC0004146C5F8FC2120463A464FF0000828F07B
:100FD00047FD04F8078039462046FFF73DFF81466C
:100FE000686AD0E90262B2422BD376000A2E38BF7B
:100FF0000A26C6EBC6001830FFF745F948B9C5F810
:10100000F401CFE734460022C5F8F841C5F8FC21C9
:10101000D2E700F1180202EB8602696A026102EB74
:10102000460242614A680160C968C0F80C80C2F398
:101030001E020A44416862F31E01C0E901164246DD
:1010400068620169436921F812909F54911D6B6A8F
:1010500043F82140D96858680131C0F31E00D960B7
:101060001044BDE8F88300BFAE640508A8E5050894
:101070007004002010B5044628F074FD0146204697
:10108000BDE81040FFF752BF07B5019001A8FFF778
:10109000D3FE019A036933F8120003B05DF804FB34
:1010A00007B5019001A8FFF7C7FE019B4269D05C1C
:1010B00003B05DF804FB07B5019001A8FFF7BCFE83
:1010C000019B063350F8230003B05DF804FB13B511
:1010D000019001A80C46FFF7AFFE019B4269D25C6C
:1010E0002260063350F8230002B010BD2DE9F8430A
:1010F0001D46002303600B6013602B60164BDFF866
:101100005C905C6A07468846164664B92B6832686C
:1011100013442B60BDE8F883336812F8010B0133E8
:10112000034433600DE04C45F0D03B6801333B6035
:10113000E268D8F800301344C8F800306269E36808
:10114000D1188A42E8D32046FFF780FC2B68246838
:1011500003442B60D9E700BF700400203425060843
:10116000F8B50B4B0B4F5C6A0CB1BC4200D1F8BD1B
:10117000E36804F1180505EB8306B54201D3246842
:10118000F2E755F8042B0449044800F02FFDF4E77A
:101190007004002034250608B664050814D4050838
:1011A00030B50023202511F8012F0AB9027030BD97
:1011B000120600F1010420D513B12023037020464C
:1011C0000B78124A03F07F036BB9013A12F8013F22
:1011D00013F0800F044600F101000BD003F07F03F1
:1011E00023700123DFE712F9014B002CFBDA013BEE
:1011F000DBB2E9E700F8013CE8E7012B04BF05702A
:1012000020460B7800F8013B0223CCE7BD640508BB
:1012100038B54368194403689942054610D9037BE1
:101220001BB1084800210BF0F3FF01F1100424F07A
:101230000704083480682146FFF735F82C60A86061
:1012400038BD00BFA8E5050870B504460E46114636
:101250001546FFF7DDFFD4E901302A461844314630
:1012600028F02EFC63682B44636070BD38B50129FB
:10127000044638BF01210025084621606560FEF75D
:10128000F7FF2573A06038BD38B505460C4601311F
:10129000FFF7ECFF6C6038BD0023C0E90132012389
:1012A000016003737047000038B514460546FFF728
:1012B000DDFF024B2560636038BD00BF49120208A4
:1012C000037B10B5044613B98068FEF7F9FF0023CD
:1012D000A36010BD38B505461020FEF7C9FF2946AA
:1012E0000446FFF7C3FF204638BD10B5044648B199
:1012F000037B13B98068FEF7E3FF2046BDE810408A
:10130000FEF7DEBF10BD000038B5037B04460D4676
:101310001BB1074800210BF07BFF0168806829445E
:10132000FEF7C1FF2368A0601D442560184438BD46
:10133000A8E5050838B504460D46FFF769FFD4E96E
:1013400001301D446560184438BDD0E900239A423D
:1013500010B5044602D10121FFF7D6FFD4E90132CE
:101360000021D154A06810BD10B50C460121FFF733
:10137000E1FF047010BD7F29F8B50C46CEB204D849
:101380000121FFF7D7FF0670F8BD06F03F06B1F563
:10139000006FC1F3871546F0800607D20221FFF7E0
:1013A000C9FF65F03F0505704670EDE705F03F05A4
:1013B000B1F5803FC1F3073745F0800508D203211E
:1013C000FFF7B8FF67F01F07077045708670DBE70F
:1013D0000421FFF7AFFFA40C07F03F0764F00F04F0
:1013E00067F07F07047047708570C670CCE738B52A
:1013F000054608460C4628F0B5FB2146024628461D
:10140000BDE83840FFF720BFF8B54768B942044649
:1014100028BF39460D4611461646FFF7F9FEA36868
:10142000A81959197A1B184428F04AFB6368A06868
:10143000334463602844F8BD43688B422CBF591A7B
:1014400000214160704738B50446154662688A42FB
:10145000084603D929448A4201D8606038BDA36890
:10146000521A1844194428F02BFB63685B1B636015
:10147000F4E70846114629F0BFBA70B5054608469C
:101480000E4628F06FFB044620B102466B682868C0
:1014900031469847204670BD2DE9F74F8A469DF8A2
:1014A000301091460D9A11F0DF0F0746A2EB0905A7
:1014B00052D0302954D1C3F34721002954D05F2999
:1014C0000CBF0526042692FBF6F106FB11210CBF8A
:1014D0002A482B4809B901350132711E92FBF6F4F6
:1014E00006FB14228A1A00EB020813F020023ED0F9
:1014F00005EBD573A5EB63045D10002D3BDDAB461A
:101500005E4532467B683868A8BF5A46414601921C
:101510009847019AABEB020BBBF1000FF0DCB9F17D
:10152000000F05D07B6838684A46514698474D44BD
:10153000002C0DDD2544A642B146A8BFA1467B681C
:1015400038684A464146A4EB09049847002CF2DC6F
:10155000284603B0BDE8F08FDFF828801026C4E7E6
:101560000DF130080126C0E7DFF81C80F6E713F024
:101570000104C2D02C460025D1E700BF28D40508BD
:101580002DD4050833D405081CD405082DE9F04FE7
:1015900093B09246CA07DDE91E761C9C9DF87490B4
:1015A000059380460D460BD48B0703D109687C4B0D
:1015B000994205D028460DF0C1FC450045F00105D3
:1015C00014F0210306D1B9F1300F03D1B742B8BFEF
:1015D00037461E46284610F0DAFE00280DF1280B8B
:1015E0001CDBA00716D52B238DF828300DF129031D
:1015F00022079DF814101FD5BAF1020F10D118461A
:101600004FF0300C00F802CB01F1010C83F801C05F
:10161000034611E0610701D52023E5E75B46E7E7D4
:10162000BAF1080F5BD130201870200645BF01F1D8
:101630000E0058700133023300200EAA1870012EDC
:10164000A3EB0B030B924FF010020693C4F3472356
:10165000C8BF1443CDE90C2014F01002CDE90213E9
:101660008DF82700059245D0CDE900A02B460DAAA4
:101670000CA90BA810F04EFD03782D2B824606D145
:101680008DF827300D9B013B00F1010A0D93012ECF
:101690007ADD0D9D059BB542B8BF35462BB19DF84F
:1016A000273003B10135069B1D4424F00103AF42EE
:1016B000079371DD14F00109A7EB05056DD1202317
:1016C0000195009337494B464A464046FFF7E4FEF2
:1016D0004D460446059B4FF03009C3B936E0BAF1D8
:1016E000100FA9D118464FF0300C00F802CB01F1D1
:1016F000170C8BE70AABCDE900A30DAA2B460CA96A
:101700000BA810F007FD8246C1E700252C469DF886
:10171000273053B100230122CDE900320DF127011A
:101720004046FFF7B9FE013F0444069B5BB100232E
:101730000122CDE900325946069A4046FFF7ACFE39
:10174000069B0444FF1A012ED8BF3E46CDE9009601
:10175000079B0D9A51464046FFF79EFE04444DB14B
:101760002023009300230F4901951A464046FFF7B6
:1017700093FE04440B980EAB984201D0FEF7A0FDF7
:10178000204613B0BDE8F08F059B0794002BBCD119
:101790001D461C463E46D9E7002500249AE700BFB7
:1017A0000CEB05084BA705082DE9F0430746900709
:1017B000984658BFC2F380038DB05ABF5B01DBB2BD
:1017C0002B23164600930A46159BDDF850902121E5
:1017D00003A80AF065FCF20504461FD52E2103A8D4
:1017E00028F006FAD0B9652103A828F001FAA8B9B3
:1017F0006E2103A828F0FCF980B9631C04F13002C3
:101800006A4430336B442E2102F8241C0234302207
:1018100003F8242CA3186B4403F8240C73060ED58C
:1018200004F13002631C0DEB0204252204F8242C81
:1018300003F130026A44002102F8241C1C4616F011
:1018400010051DD09DF80C302F2B4FF0000319D838
:10185000012203A9CDE900323846FFF71DFE09F148
:10186000FF390546013C0DF10D01CDE900893346F4
:1018700022463846FFF710FE28440DB0BDE8F0833D
:1018800003A9F2E703A91D46EFE700002DE9F04F99
:1018900081468BB014464FF000080B461D4613F8E6
:1018A000012B0AB1252AF9D1A94208D26E1AD9F81A
:1018B0000430D9F8000032469847B04429460B78E6
:1018C000002B00F08B8120234A1C03930027134632
:1018D00013F8016B3EB12D2E25D01ED8202E29D015
:1018E0002B2E24D00026154612F8013BA3F130011F
:1018F000092922D92E2B4CD16B782A2B23D00023F7
:10190000154612F8011BA1F1300009281ED80A2043
:1019100000FB031BABF13003F2E7302EE2D147F0BE
:101920001007039601E047F001071A46CFE747F09A
:101930000207FAE747F00407F7E70A2101FB06333D
:10194000A3F13006CFE754F8043B023523EAE37BEA
:101950002B786C2B08BF013595F800A0BAF1000F69
:1019600000F03C81BAF1780F09D8BAF1570F13D8BB
:10197000BAF1470F5AD8BAF1440F00F21D81D9F8D5
:101980000430D9F8000001222946984708F10108DF
:1019900085E04FF0FF3BDBE7AAF15803202BEED8A0
:1019A00001A252F823F000BF331A02087F1902087F
:1019B0007F1902087F1902087F1902087F1902089F
:1019C0007F1902087F1902087F1902087F1902088F
:1019D000851A0208AF1A0208331A0208B91B020856
:1019E000B91B0208B91B02087F1902087F190208F7
:1019F0007F1902087F1902087F1902087F1902085F
:101A00007F1902087F190208331A0208C51A020852
:101A10007F190208ED1A02087F190208331A02081A
:101A20007F1902087F190208331A0208BAF1500F11
:101A3000A5D154F8040B0AF0DF03502B014667D1FF
:101A4000BAF1640F6AD1002880F29D802D238DF8B1
:101A5000173041420A2251230DF1280A0A3B0DF1A9
:101A6000180BB1FBF2FC02FB1C1009288CBFC0183C
:101A700030300AF8010DDA458E4661465DD0724578
:101A8000EFD95AE054F8043B019653B1039B5549F2
:101A9000009304223B464846FFF7FEFC8044691C45
:101AA000FBE6039B009350493B460522F3E754F8BD
:101AB000043B8DF81830039B009301963B460122AE
:101AC00006A9E8E706A954F8040BFFF700FBBBF1F1
:101AD000FF3F014604D0069B9B4538BFCDF818B0A8
:101AE000039B0093069A01963B46D4E754F804AB57
:101AF000504628F037F8BBF1FF3F024602D0584568
:101B000028BF5A46039B009301963B465146C2E7C5
:101B1000BAF1640F97D0BAF1750F2ED02AF00F03E7
:101B200000220F3B8DF81720DBB21022002893D142
:101B300030238DF827300DF1270A17F0100B9DF890
:101B400017302DD0002B35D0039B0093012201923A
:101B50003B460DF117014846FFF79EFC013E8346C8
:101B6000039B00930AAA01963B46A2EB0A02514648
:101B70004846FFF791FC584490E700238DF8173052
:101B80000A226123D2E7BB0705D52B238DF8173036
:101B90000A225123CAE7C7F380035B01DBB2F5E7F2
:101BA000002BDDD006AA9245DAD90AF8013C0AF1E9
:101BB000FF3AD5E79B46D3E7073424F00704F4E85F
:101BC000020134F02DFACDE9006B00EE100A039B00
:101BD0003A4651464846FFF7E7FD5FE740460BB0FF
:101BE000BDE8F08FB88A0508BD8A05080EB403B5B4
:101BF00003AA52F8041B0192FFF748FE02B05DF8F9
:101C000004EB03B070470346007893F90020002AE4
:101C10000ADA00F07F004022104206D113F8012FAB
:101C200002F0C001802904D0704720EA0200520867
:101C3000F2E702F03F0242EA8010EFE7431C184649
:101C40000133027802F0C002802AF8D070470346C0
:101C50000020994200D8704711F8012D02F0C0020F
:101C6000802A18BF0130F4E703460144002099425E
:101C70001A4600D87047127802F0C002802A03F199
:101C8000010318BF0130F2E77F289DBF024B185CAB
:101C9000C0F340000020704743D405087F289DBF53
:101CA000024B185CC0F3C0000020704743D4050805
:101CB0007F289DBF024B185CC0F380000020704756
:101CC00043D405087F289DBF024B185CC0F38010E9
:101CD0000020704743D405087F2809D8064B1B5CB9
:101CE00013F00C0F06D1A0F15F0358425841704722
:101CF000002070470120704743D405087F289DBF0E
:101D0000024B185CC0F300100020704743D4050854
:101D10007F289DBF024B185CC0F340100020704725
:101D200043D4050808B50246FFF7E8FF02EB401070
:101D300008BD08B50246FFF7EBFF404220F01F0048
:101D4000104408BD3038092884BF20F0200007382F
:101D5000704710B502460144E5240020914203D8A3
:101D6000B0FA80F0400917E012F8013B30B103F0FF
:101D7000C003802B11D10138C0B2EFE7BF2B09D9C6
:101D8000F72B09D8DB0803F0060344FA03F303F04A
:101D90000300E3E71B06E1D510BD0020FCE7023994
:101DA00081420B4603D31A880239002AF8D0023345
:101DB000181A40107047B2EB131F70B504464FEA73
:101DC000131019D901EB4001101A03F00F0302465A
:101DD0002646012A0CBF0D880D68013A25FA03F545
:101DE00026F8025B01F10201F3D104EB400434F860
:101DF000023C03B9013870BD0020FCE7F0B5059C3A
:101E00000025121B2E46AC420FD101EB44031746AE
:101E100000EB4404411A9FB904EB420316B124F8C5
:101E200012600233181A4010F0BD31F8157033F803
:101E300015C067443E4420F81560360C0135E2E7D2
:101E40001D8835445D522E0C013F0233E3E7F0B4A8
:101E5000049F00260D463446D11BB7420BD105EB3B
:101E600047030A4600EB4707451B7AB907EB4101D8
:101E7000F0BCFFF794BF35F816C033F81620644461
:101E8000A41A20F8164024140136E6E71E883444CC
:101E90005C53013A24140233E7E72DE9F043079C31
:101EA000DDF828E0DDE908760239154684464FF66C
:101EB000FF78A4EB020955B900EB42011FB10123E1
:101EC00020F812300231BDE8F043FFF768BF31F867
:101ED000024F013D4444264405EB0904A5422ABFB4
:101EE00033F8024B4FF6FF744444744486EA040E00
:101EF00017FA8EF72CF8027B4FEA144E360C3F0C83
:101F0000D9E738B502290446806838BF02210D465A
:101F100018B12368B1EB930F07D96900FEF7C3F935
:101F20002368A06065F39F03236038BD38B504467D
:101F30000C20FEF79DF923682278054602F0010285
:101F4000C3F39D0023F0030313432B6063686B60AE
:101F50004000FEF78DF9A8602268A168C2F39D02D7
:101F6000520027F07DFD284638BD994210B511D3A7
:101F700013D800EB410002EB410209B9084610BD3D
:101F800030F8023D32F8024D1B1B002B02DB04D15E
:101F90000139F2E74FF0FF30F1E70120EFE710B52C
:101FA000044638B18068FEF78BF92046BDE8104042
:101FB000FEF786B910BD70B505460C460221FFF745
:101FC000A0FF002C2B78B4BF0122002262F3000393
:101FD000AA682B70B4BF61422146012388B2090C64
:101FE00014461E4622F8020B03F10103F6D16E607F
:101FF000208070BD0023C0E900338360704728B1A2
:1020000003789B0702D48068FEF75AB9704738B549
:1020100004460D464968FFF774FF2A782378A068C4
:1020200062F3000323706A686260A9685200BDE829
:10203000384027F015BD0A4629B90178426062F39D
:10204000000101707047FFF7B6BF08B5FFF7D2FF78
:10205000BDE80840FFF7EFBF920042F0020210B463
:1020600002600022C0E901215DF8044B1946FFF728
:10207000E2BFF8B59DF8187014461D4604210646C7
:10208000FFF73FFF22462B4627B1002D0CDA6242B4
:1020900065EB4503317867F3000131700021716011
:1020A00052EA030102D1F8BD0027F3E7D6E9011097
:1020B0004C1C746020F81120120C42EA03421B0CE5
:1020C000EEE72DE9F3418DED010A019D0378EA0F5A
:1020D00062F300030370C5F30F4313F4FF4380461C
:1020E0000BD198F8003023F0010388F8003000236A
:1020F000C8F8043002B0BDE8F081B3F5FF4FF0D06E
:10210000C5F3C754A4F17F06002EEADB05D10121F7
:1021100002B0BDE8F041FFF74EBF162EC5F316051D
:10212000A4F16F07D8BFC6F1170645F400054FEAC2
:102130002717D5BFF540963C00260936D4BF344654
:1021400024113946C8BF06F00F06FFF7DAFEC8F8BB
:1021500004702CB1D8F808006200002127F0C4FCFC
:102160004EB1D8F8083005FA06F223F81420C6F16B
:102170001006F5400134A742BCD0D8F8083023F847
:1021800014502D0CF6E72DE9F84304468F18C2F3DE
:102190005B020D46511C9846089EFFF7B2FE23785D
:1021A00068F300032370AC4600221FFA86FEBC458C
:1021B0006046626002D3401BBDE8F8830178A1F15C
:1021C0003003092B0CF1010C05D9A1F14103192BA6
:1021D00012D8A1F13703B342EDD2A06890468146F0
:1021E000B8F1000F0FD100EB420113B120F812300B
:1021F0000231091A4A10DAE7A1F16103192BDAD882
:10220000A1F15703E7E7B9F800100EFB013329F8F5
:10221000023B08F1FF381B0CE2E7F8B5044615460F
:102220001E46C1B1531E1E444FF0FF37E9000F3167
:1022300009092046FFF765FE2378002123F00103FA
:10224000237061600B4645B9A06800EB4101FFF7C0
:10225000A6FD6060F8BD0127E8E700220F2B08DC2F
:10226000307898400243013D92B203F108033E44A6
:10227000F4D1A068013100EB41006160103B20F80F
:10228000022CE0E738B505780B7805F0010203F081
:1022900001030446981A08D1D1E90132D4E90110AA
:1022A000FFF763FEEB0748BF404238BD884210B5D8
:1022B000044601D0FFF7ABFE237823F0010323701F
:1022C00010BD884210B5044601D0FFF7A0FE636838
:1022D0003BB12378C3F3000282F0010262F30003F2
:1022E000237010BD88421FB5044601D0FFF78FFE52
:1022F000626862B901212046FFF703FEA26801234C
:1023000013806360237843F00103237010E0237887
:10231000D9070FD523F00103237001230093A1688F
:10232000ADF80E3008460DF10E03FFF790FD60602A
:1023300004B010BD511C2046FFF7E3FD01230093BC
:10234000D4E90121ADF80E3008460DF10E03FFF778
:1023500055FD6060D6E74B682DE9F04705460E460F
:10236000144603B12AB931462846BDE8F047FFF7C5
:102370004EBE02F10F014FEA111803EB1111FFF7E6
:10238000C0FDD6E9012308EB0207A96807F1004068
:1023900014F00F0400F1FF3008BF10244FEA400989
:1023A00001EB400003EB4203114686464FF0000C60
:1023B000C4F1100409BB6FF001035A4383182CFACF
:1023C00004FCC8F1010820F802C003EB48034FEAFF
:1023D00048021846524227F087FB09F102090346DA
:1023E0004B4417B133F8022D9AB16F6032782B78D5
:1023F00062F300032B70BDE8F08733F802AD4AEAC0
:102400000C0C2CFA04FA2EF802A94FEA0C4C0139F4
:10241000D0E7013FE5E72DE9FF410D464968064653
:10242000144601B132B92946304604B0BDE8F04146
:10243000FFF7EDBDFFF765FDB768D5F808806A685E
:10244000234641463846FFF7B6FC7060297833785A
:1024500061F300033370DB0702460AD50023696885
:10246000ADF80E302009994201D0834204D1814257
:102470000AD804B0BDE8F08138F813509DB10123AB
:102480008142ADF80E3012D904F00F04012338F860
:10249000101003FA04F4013C214206D1BDF80E30BD
:1024A000002BE6D003E00133DDE7ADF80E30012369
:1024B00012B93B807360DCE7009339460DF10E03DF
:1024C0003846FFF79BFC7060D3E72DE9F3410D46DA
:1024D0005768D1F804803B46144606469268A868BF
:1024E0004146FFF742FD01301EBF23462C461D46E4
:1024F00023782A7883EA020318BF4746DB0719D4FA
:10250000791C3046FFF7FDFC6B680093D4E901218C
:10251000AB68B068FFF772FC7060237832780028EF
:102520000CBF002303F0010363F30002327002B01A
:10253000BDE8F08139463046FFF7E3FC6B68009355
:10254000D4E90121AB68B068FFF781FCE4E72DE92D
:10255000F3410F464E68D2F8048014464346314694
:1025600092680546B868FFF700FD01301EBF23469C
:102570003C461F4623783A7883EA020316BFB046EA
:1025800001260026DB0719D508F101012846FFF7CF
:10259000B8FC7B680093D4E90121BB68A868FFF709
:1025A0002DFC686018B1207800F0010070402B7895
:1025B00060F300032B7002B0BDE8F081414628466D
:1025C000FFF79FFC7B680093D4E90121BB68A868F2
:1025D000FFF73DFCE5E74B682DE9F04F0C465168ED
:1025E0008B42154621BF2546194613461C462B78BB
:1025F000DB0785B0064622D4237813F001071ED1ED
:10260000FFF77FFCD4E9011CB068AD683B469942F6
:102610000CD100EB4101FFF7C2FB00237060327860
:1026200063F30002327005B0BDE8F08F35F8132077
:102630003CF81340224020F813200133E7E7013132
:102640003046FFF75EFC2F782378D5F804C0B068D9
:10265000A26887EA0301C94301F0010E41F30001BA
:1026600089B207F0010947F300070291B9B201915D
:10267000A968A1F10208616803F0010A43F30003AD
:102680009BB2A1EB0C0100936746834603918FB97F
:1026900000EB4C01BEF1000F03D0012320F81C30E9
:1026A0000231FFF77CFB706022782B78C2F30002C6
:1026B0001340B4E738F8021F019B5940039B013FC8
:1026C0008944D9198F4225BF32F8021B009B00991B
:1026D00059408A44029B09EA0A0159401EFA81F1D5
:1026E0002BF8021B4FEA1A4A4FEA19494FEA114EDA
:1026F000CDE72DE9F84F4B680D4651688B421446E3
:1027000021BF2C46194613461D462378DB07064693
:1027100031D42B7813F001072DD1FFF7F2FBD5E967
:10272000012EA0686468D6F808C0A41A3B469A42F5
:1027300013D10CEB4203214600EB4202ACEB00004C
:10274000A1B903EB4403A3EB0C035810337870607A
:1027500061F300033370BDE8F88F30F813103EF8D2
:10276000135029432CF813100133E0E71588155254
:1027700001390232E4E701313046FFF7C2FB277826
:102780002B786168B068A468D5E901E203F001091B
:1027900047F3000543F3000307F00108ADB29BB215
:1027A000A4F1020C0F4683464FF0010AAEEB010E76
:1027B0002FB900EB4101FFF7F2FA0121C6E73CF81F
:1027C000024F013F6C40A0440EEB0704A7422ABF12
:1027D00032F8024B1C465C40A14448EA0904E44339
:1027E0001AFA84F42BF8024B4FEA19494FEA1848B9
:1027F0004FEA144ADCE74B68F0B50D4651688B424E
:1028000024BF19461346144624BF2C461D4627787C
:102810002B785F4017F0010785B0064636D1FFF7E9
:1028200070FBD4E901212478B06814F00104D5E9E3
:10283000015324D1521BA54212D101EB450314468A
:1028400000EB4505411AACB905EB4201FFF7A7FAC9
:1028500000273378706067F30003337005B0F0BD74
:1028600031F8147033F814C087EA0C0720F814709C
:102870000134E0E71F885F52013C0233E3E7CDE912
:102880000277CDE90057FFF708FBE1E70131FFF7D9
:1028900038FB2B78DB4303F0010303932378DB43FE
:1028A00003F001030127029301976B680093D4E9B9
:1028B0000121AB68B068FFF7F0FACAE72DE9F04FE5
:1028C0004B6885B004460E4615460BB1536843B9B4
:1028D000237823F0010323700023636005B0BDE873
:1028E000F08F81422DD1FFF721FBA5420646074616
:1028F0002ED06B68716820461944FFF702FB2268EE
:10290000A068C2F39D025200002127F0EDF8B368E1
:10291000D4F808E0D6F804900193AB680293002243
:102920006B6803930EEB4908F4461146039B9342F0
:1029300033D0DDF804B0CDF80090ACF102000023F4
:102940001AE0824206D1FFF7F1FA05460746D0E7C2
:102950000546CEE70027CCE730F802AF53441946CE
:10296000029B3BF802AB33F8123003FB0A130099C9
:10297000038001391B0C009100990029ECD14146DC
:10298000881C13B1A8F800300146A1EB0E014910D4
:102990000CF1020C01328046C8E761602A78337876
:1029A00053402278384663F30002227005B0BDE838
:1029B000F04FFFF7F4BA4B6870B50546144613B1F3
:1029C0001378DA0706D52B7823F001032B70002348
:1029D0006B6070BD636823B9BDE870400121FFF7EB
:1029E000EABA0846FFF7A2FA06462046FFF79EFA23
:1029F000012104462846FFF7DEFA636883B1A36825
:102A00001B88DB0704D5324629462846FFF756FFC8
:102A1000D4E9012101230846FFF7CDF9606038B9F8
:102A20003046FFF7BCFA2046BDE87040FFF7B7BA62
:102A3000324631463046FFF741FFDEE72DE9F04FE1
:102A40000C4651688FB09346013105460393FFF75A
:102A500058FADBF80420A86801325200002127F060
:102A600043F82B78002623F001032B706E60DBF80F
:102A7000041020460131FFF744FA59462046FFF77B
:102A8000C6FA039BD4F80890D4F80480D3E9013740
:102A90000293AB6804933A46029B41464846FFF7CF
:102AA00064FA002833D1049A6060012313806B60BC
:102AB00023786268002A0CBF002103F0010161F352
:102AC0000003039923709BF8003009784B40DB0723
:102AD00040F1FD806B682978003B18BF012363F348
:102AE00000012970002A00F0F2800BA84FF0FF319E
:102AF000FFF7ABFA0BAA29462846FFF7E6FC039A34
:102B0000214620460FB0BDE8F04FFFF7DEBC013094
:102B100001D16E60CCE7029B03F10042013A4FEA1B
:102B2000420A37F8121033460E0403F101004ED565
:102B30009BB209EB48014FF0000C08F10100C3F112
:102B4000100629F818C0019160600231CE46059642
:102B50008E4540D337F812209A400592029A012AF6
:102B600009D907EB0A02C3F1100132F8022CCA405E
:102B7000059911430591029A801A6860049A00F140
:102B80000040013802EB400207920AF1020209926A
:102B9000BA1E0892D4F804A0029A524529D30AF129
:102BA000004A0AF1FF3A09EB4A0A0022C3F1100079
:102BB000D14573D96FF000416B682BB104985A1856
:102BC00030F81220002A73D06FF0004175E0490000
:102BD00089B20346A8E7BEF8008008FA03F64CEA7B
:102BE000060C059E2EF802CB28FA06F81FFA88FC80
:102BF000AEE7019A0198118832F8022C42EA0142AC
:102C00000599B2FBF1F20999411A06910899069FBC
:102C100000200E4686460199B9420DD8098808441D
:102C2000A8BB079921F80229019A0791023A01925B
:102C30000AF1FF326260ADE736F8021FB7F8008094
:102C4000994041EA1E4E1FFA8EF1514318FA80F85E
:102C50001FFA81FC090CA8EB0C0CC1EB204127F8F2
:102C600002CB01EB2C40D6E738F8021F994041EA2D
:102C70001E4EBCF80010394411FA8EF12CF8021BDC
:102C80000F0C01996145EFD83844013AC8E7002795
:102C9000DDF82080DDF818C0BE46F2E7BAF8001073
:102CA00041FA03F6324381402AF802298AB27FE7CB
:102CB000013B6B6080E7013B63606368002B3FF47E
:102CC000F7AE5A1839F81220002AF4D0F0E60FB007
:102CD000BDE8F08FF0B51F464B6885B004460D4641
:102CE00016464BB11378DA0706D47B68012B0BD15B
:102CF000BB681B88012B07D1237823F001032370C5
:102D00000023636005B0F0BD01212046FFF753F9B1
:102D10007368002BF6D02846FFF708F905463046C1
:102D2000FFF704F90023CDE90133064603937368E6
:102D3000B3B1B3681B88DB070AD52A462146204673
:102D4000FFF7BCFD3B462246214601A8FFF776FE71
:102D5000D6E9012101230846FFF72DF8706058B924
:102D600001A8FFF74CF92846FFF719F9304605B0DE
:102D7000BDE8F040FFF713B92A4629462846FFF779
:102D80009DFD3B462A46294601A8FFF757FECEE7A0
:102D900010B5D0E90121034601EB42020020914227
:102DA00004D31B78DB0748BF404210BD32F8024D08
:102DB00044EA0040F3E730B5D0E90124002304EBF6
:102DC0004202944206D30278D20748BF5B420B60AE
:102DD000012030BDB3F5004F04D232F8025D45EA60
:102DE0000343EEE70020F4E72DE9F74FDDF830C0AC
:102DF000019206460F4609B30CEB0300D6E90189A0
:102E0000012400211A46A2468E46B8F1000F17D1C0
:102E10000199002945D0002A43D1002B41D0002F31
:102E20003BD09CF800302CB13478DB4384EAD314D7
:102E300004F00104204603B0BDE8F08F6046DDE7F2
:102E400039F8025B0EF1100E45EA0141BEF1070FA1
:102E500002DC08F1FF38D8E796F800B08DB21BF01D
:102E6000010F1FBFED435AFA85FA1FFA8AF5CAF31C
:102E7000072A42B91CB1EDB2B5FA85F46409AEF186
:102E8000080E090AE2E7EDB227B100F8015C01384B
:102E9000013AF4E700F8015BFAE7634413F8013CF8
:102EA000C1E7337813F0010F14BFFF210021002F79
:102EB00018BF604626F018FEBCE70000D0E90132DA
:102EC0009FED0C0A9FED0C7A02EB43039A4205D367
:102ED0000378DB0748BFB1EE400A704733F8021DA4
:102EE00007EE901AF8EEE77AE0EE077AB0EE670A9E
:102EF000ECE700BF00000000000080472DE9F74F1D
:102F00000A2944689DF830A00D9E154614BF04227E
:102F10000322804689460092A4B98DB1013D324614
:102F200015F8011F134641B930221A70002203F828
:102F3000012F981B03B0BDE8F08F02F8011BEFE7EB
:102F40003346F1E7640020460193FDF791F9D8F884
:102F500008102246074626F083FD019B3046B34603
:102F600007EB040C3A3BACF102040021A742A64651
:102F70001DD9303139295C4688BFC91804F8011BB6
:102F800039468C458E461DD83846FDF799F965BB04
:102F900098F80030DB0744BF2D2304F8013B33468B
:102FA000621E9A4233D800232370A01BC2E7BEF8EA
:102FB00000E04EEA014EBEFBF9F124F8021909FBCC
:102FC00011E1D3E7BEF800200231002AD9D0BAF1CE
:102FD000000F08D0009A211A914204D10BF102048B
:102FE0008BF801A02046A346BDE7284626F0BAFD8F
:102FF00029185A460B46AB4204D88D4288BF0020A0
:103000000444C5E713F8017D02F8017FF3E719785E
:10301000107803F8010B02F80119C2E7D0E9023277
:1030200093423DBF5A1C826018784FF0FF307047C2
:103030000368013B033310B5044602D84068FDF72E
:103040003FF92046BDE81040FDF73AB9F8B505460E
:1030500010200C461F461646FDF70AF9054B846002
:10306000C0E900743444C4606B60034B2860AB60FB
:10307000F8BD00BF1D3002083130020802690A2A7B
:10308000F8B504461BD18369013383610123E361F1
:10309000237D2361637D237500260A27256EB5B144
:1030A0006B1CA26D2366555D626D934201D366650C
:1030B0002666237D0D2B14D0BDB16575F8BDC3699F
:1030C000092A04BF073323F007030133DFE7D4E9FC
:1030D00001039847431CECD0012838BF0120054666
:1030E000E7E70A2D2775D9D0E6E7237D002BE4D04A
:1030F0000A2B18BF0A25E0E701692729024601D0FB
:10310000222912D1012024E0137D272BFAD0222B73
:10311000F8D0722914D1662B16D1507D2728F1D012
:10312000A0F12203584258417047A1F162001328D0
:1031300004D8084B034113F00100E5D0002070478C
:10314000662904D1722B00E0622B02D1E5E76229E7
:10315000F8D07047EEFFF6FF38B504460D462069FB
:10316000D0B10A2806D10DB1636AB3B12046FFF78A
:1031700085FFF4E7FEF788FD0028F7D12369232BAC
:1031800008D12046FFF77AFF2369002BE7D00A2BEE
:10319000F7D1E4E75C2B02D00025284638BD237D1B
:1031A0000A2BF9D12046FFF769FFDFE72DE9F04F41
:1031B0000023044685B001214364FFF7CDFF276A51
:1031C000A3696363002FE369A36307DA072384F825
:1031D0003C300137276205B0BDE8F08F04D00623EC
:1031E00084F83C30013FF5E7002835D039462046C9
:1031F000FFF7B2FF052384F83C30D4E90B3003F12C
:103200000042013AE56930F81220013D9542E2D0D2
:1032100009D8013B30F81320954218D3DBD00223A4
:1032200084F83C30D7E7A16A8B4207D308314900C4
:10323000FDF739F8A36A20630833A362E36A5A1CD6
:10324000E26220F81350236A01332362C3E7226A43
:10325000E362013A2262DCE7256915B984F83C5043
:10326000B9E72046FFF748FF0646002800F00C8229
:1032700084F83C702369722B6CD008D8622B0CD078
:10328000662B71D0B9460025A8460B230EE0753B8E
:10329000D3F1000949EB0309F5E7237D722B4FF0C9
:1032A000000569D0A8464FF001090C2394F83C2092
:1032B000002A6AD184F83C30B9F1000F08D02046CA
:1032C000FFF7DCFEB9F1020F02D12046FFF7D6FE70
:1032D0002369222B0CBF2223272320460193FFF7CB
:1032E000CDFE2369019A934240F08680237D93426C
:1032F00040F082802046FFF7C1FE2046FFF7BEFE69
:103300004FF0030935B1A36E23B9A64904F1640057
:10331000FEF76DF804F140034FF0000B02932169B2
:10332000002900F0A881B9F1010F02D10A2900F0AB
:10333000A281CB4563D3594604F14000FEF77CF8E7
:1033400001212046FFF708FF2046FFF7D5FE0028A1
:1033500090D11CE0237D622B0DD0662B10D0002570
:10336000B0464FF0010990E7237D722B354608D017
:103370004FF00008F5E70025B0464FF0020994E74A
:103380003546B0464FF002097FE79A4294D0A36ECB
:10339000002B3FF420AF292104F16400FDF7E4FF86
:1033A000236E04F15006002B40F06B810321304660
:1033B000FDF7C0FF23690370237D4370637D837035
:1033C000D4E91A57216E2A463046FEF71DF82A46E0
:1033D000394626F045FB0023A366236EA26D581CD8
:1033E0002066D15C2161991C2166105C2075033335
:1033F0002366535C6375EEE64FF0010982E7019B9B
:103400008B4209D1029819460BF1010BFDF7B3FF6E
:103410002046FFF733FE82E7002D60D15C2940F0A3
:10342000278120460391FFF729FED4F810A00399C5
:10343000B8F1000F6CD00298FDF79DFFD346D2E0A3
:1034400004F1640B28215846FDF78EFFD4F868A0DC
:103450000022216979B172BB3A290CD07D290AD0AA
:10346000212928D1207D7238012829D8607D3A2869
:1034700001D07D2824D1D4E91A21881810F8010C34
:103480003D2809D1A2EB0A02514404F14000FDF7A6
:10349000DBFEA26E013AA266924508BF042358469D
:1034A00008BF84F83C302921FDF75EFF2C215846E7
:1034B000FDF75AFF24E021F020005B280AD10132F9
:1034C000C9B258460392FDF74FFF2046FFF7D6FDDD
:1034D000039ABEE75D2808BF02F1FF32F0E77B29BF
:1034E0009CD120460391FFF7C9FD23697B2BA7D10F
:1034F00004F140000399FDF737FF2046FFF7BEFDBA
:103500007B2104F14000FDF72FFF4FF0000B06E791
:10351000BAF1780F09D8BAF15B0F0AD8BAF1220FC5
:1035200053D029D8BAF10A0F23D05C2104F140000E
:1035300082E7AAF15C021C2A73D8DFE802F0467227
:103540007272728A2A7272723A72727272727272C3
:10355000307272720F722D3D37725C004FF00D0B9E
:1035600094F83C300B2B77D1594604F14000FDF71D
:1035700002FF4FF0000B4BE7BAF1550F1CD0D4D827
:10358000BAF1270F21D0BAF14E0F4AD106480AF0FE
:1035900021FE4FF0080BE3E74FF0090BE0E74FF097
:1035A0000A0BDDE7088B0508118B05084FF00B0BA4
:1035B000D6E74FF00C0BD3E794F83C200C2A06D149
:1035C0005C2104F14000FDF7D6FED346C8E7BAF10E
:1035D000750F14BF4FF0080A4FF0040A4FF0000BAC
:1035E000BAF1010A0AD2BBF5881FB9D34FF0010323
:1035F00084F83C30BDE74FF0020AEFE72046FFF7C2
:103600003DFD226903921046FEF75CFB002800F0A6
:103610005081039A1046FEF795FB4FEA0B1B83443B
:10362000DEE7AAF1300BBBF1070F3FF67EAF4FF09C
:10363000030A06E02046FFF721FD2269303A02EB3B
:10364000CB0B227D303A072ACDD8BAF1010AF1D14D
:10365000C9E74FF0070B83E7BBF1FF0FC6D80C2B70
:10366000C4D15FFA8BF104F14000FDF77DFE80E7E5
:103670000298C9B2F9E7CB453CBF032384F83C303C
:1036800059E6033B23669BE62846FEF707FB2169C4
:10369000D8B95F2919D07F2917D80846FEF708FB4B
:1036A000002855D123692E2B4DD0844D00262F782C
:1036B0001FB12369BB4240F0A4802046FFF7DEFC27
:1036C000002F40F0A6800123AAE5082384F83C30AF
:1036D00004F14005C9B22846FDF746FE2046FFF733
:1036E000CDFC2069D8B92846FDF72FFE744F064659
:1036F000002557F8041B304626F042FA00281CD15A
:103700000E35EDB2112D84F83C507FF464AD6D4B55
:10371000D3F80032002B14BF0E23102380E5FEF7F0
:10372000BDFA40B920695F2805D07F2803D8FEF78D
:10373000BFFA0028D7D0217CCDE7FFF64CAD01358C
:10374000242DD6D147E5207DFEF7B2FA0028ACD073
:1037500021692E292AD10A2384F83C30002504F15E
:1037600040063046FDF707FE2046FFF787FC0A2794
:10377000206900283FF42FAD55BB20F02003452BD6
:1037800026D16521304684F83C70FDF7F4FD2046D3
:10379000FFF774FC21692B2901D02D29E8D130468F
:1037A000FDF7E9FD2046FFF769FCE1E70923302931
:1037B00084F83C30D2D1237D43F02003623BDBB25E
:1037C000162BCBD8404DDD4015F00105C7D1C5E71C
:1037D000FEF764FA28B121692E290DD184F83C70D6
:1037E000DDE72069FEF764FA0028F4D123692E2B67
:1037F000F1D05F2BD6D0EEE421F020034A2BCED1BE
:10380000ECE7652F01D0632F00D10135013601357A
:103810004DE7212F08D123693D2B7FF454AF20467B
:10382000FFF72CFC3923FBE42E2F0FD123692E2B1D
:1038300002D1237D2E2B01D05C23F1E42046FFF73B
:103840001DFC2046FFF71AFC0D23E9E4033533463F
:1038500015F8027C632F18D0652F16D01B4AD35C55
:1038600084F83C30543BDBB2052B3FF6B4AC01226C
:1038700002FA03F313F02A0F18D113F0150F3FF4D7
:10388000AAAC636A13446362A5E415F8012C2169AC
:10389000914206F1010607D12046FFF7EFFB3346C0
:1038A000652FDBD00235D3E7632FFAE7636A013B6C
:1038B000E9E7012384F83C30834651E6C38A0508D2
:1038C000C4D40508700400200120400054D5050828
:1038D0007FB5064601AD742085E80E00FCF7C8FCF4
:1038E0000446034695E8070043F8046B83E80700A5
:1038F00001236FF001020025C4E906320A22C4E95F
:103900000A23C4E908551420FCF7B2FC20212063E7
:1039100004F14000FDF7AAFC294604F15000FDF730
:10392000A5FC294604F164002566FDF79FFC236B86
:1039300020461D802561A582FFF7A0FB2046FFF7EA
:103940009DFB2046FFF79AFB2046FFF72FFCA36B59
:10395000012B06D094F83C30052B1CBF062384F8BD
:103960003C30204604B070BD30B585B001AC054692
:103970002046FFF76BFB94E80E002846FFF7A8FFF0
:1039800005B030BD30B585B001AD044601462846CE
:1039900020F0ACFC95E80E002046FFF799FF05B03B
:1039A00030BD10B50446B0B1C3684068984704F113
:1039B0004000FDF785FC04F15000FDF781FC04F1A7
:1039C0006400FDF77DFC206BFCF77AFC2046BDE827
:1039D0001040FCF775BC10BDD0E90432013B036117
:1039E00052F823007047036942695B1A013B52F8A1
:1039F00023007047F8B5446A06460D46B4B1D4E9D1
:103A000000030B44834222D908310022014420469E
:103A1000FCF754FC0246B8B9616820460831FCF74F
:103A20004DFC63682360336A63603462802D2F46E7
:103A300038BF802707F10800FCF71AFC0023076055
:103A400043600446706202E023682B442360606890
:103A50000544656008342044F8BD38B50D460C2196
:103A60001446FFF7C7FF4FF49D72C0E901240560BB
:103A700038BD38B5D0E903329A4204460D4608D322
:103A8000103399004069FCF70EFCE3686061103365
:103A9000E360D4E90432591C216142F8235038BD57
:103AA000F8B504461D46D0E9000383420F4616468A
:103AB00008D31030C100A068FCF7F5FB2368A060B4
:103AC00010332360D4E90103421C626053F83010C4
:103AD00067F3170143F8301003EBC002D67055604E
:103AE000F8BD10B48469CAB20023616B5DF8044B61
:103AF000FFF7D6BFF0B593B0044668460E461746AA
:103B00001D46FCF775FB10B1002013B0F0BD3A461E
:103B1000314620460AF098F90446FCF73FFBA3071C
:103B200003D12268024B9A42EED02C600120ECE7D0
:103B300020E2050810F00102034604D040F0010322
:103B40000B6001207047A8B110F0030013D11A795F
:103B50003A2A11D19B680B6013F00100F1D19A074A
:103B60000AD11868054B9842EBD0054BC31A58424E
:103B70005841704770471046704700BF0CEB05086E
:103B8000B4E8050810F001021CD110F003030CD0BA
:103B900000F00F03062B15D00A2B11D100090D38A8
:103BA00003288CBF00200120704770B102793A2AA7
:103BB00008D02D2A08D18068B0FA80F040097047FB
:103BC000104670470120704718467047C20702D55B
:103BD00040F001007047830710D0030900F00F0088
:103BE000062803D1D80040F002007047A3F10E0070
:103BF000022809D8064B53F82000704730B10379EA
:103C00003A2B03D1806870470248704702487047DA
:103C100080D50508D4F1050808F6050838B505462D
:103C20000C46FFF7AFFF38B12846FFF7CFFF0BF088
:103C3000C9FA031B5842584138BD2DE9F0410F46DF
:103C400005461446114689B9204612F06FFE01461A
:103C500000F10808A4B90A4628463946FFF7FDFED8
:103C600001462846FFF705FF012007E001392846F5
:103C7000FFF7B9FEFFF786FF0028E4D1BDE8F08129
:103C80002846FFF7A9FE0646FFF7A0FF013C48F8CB
:103C90002400002EDED0B307DCD1686A00F10803EF
:103CA0009E42D7D3426813449E42D3D273681B0A04
:103CB0000233A2EB83024260CCE70000F7B58669CD
:103CC00096F83C20A2F1080305460F46042B52D873
:103CD000DFE803F003232B384C00D6E91110FDF781
:103CE00025F9902F04460ED1C100002241F00201B7
:103CF00005F128000AF014FE28B14268D3071CD54C
:103D000042F0010002E0200140F002000146284696
:103D100003B0BDE8F040FFF7ACBE0022D6E91110B9
:103D2000334608F003FC0246E8E70096D6E9111096
:103D30000023012208F032FD0246716B2846FFF78E
:103D40008CFEE3E7D6E911100A2906D8FDF7EEF854
:103D500030B1000140F00600D8E7FDF799F8F7E729
:103D6000D6E91121064810F0C9FEE5E7D6E91110A1
:103D700010F0A4FFE0E7120142F00A00C6E700BF1E
:103D8000FCF4050810B5FFF7D5FE50B10B6813F031
:103D9000010007D19A0704D11868034BC31A58428F
:103DA000584110BD0120FCE70CEB05080021FFF78E
:103DB00035BF0121FFF732BF2DE9F04F2D2A85B025
:103DC0000446884616461D460BD10021FFF70BFE20
:103DD000C0B1820702D10379922B13D005B0BDE8A0
:103DE000F08F922A2ED10021FFF7FDFD014648B148
:103DF000830707D14768FBB2952B18D12046FFF700
:103E0000EBFD013DA6F12303DFB2092F00F2EB80A9
:103E1000092B00F2CF80DFE813F0ED00ED00ED009C
:103E20001E011E011E014501ED00CD008F01962BE4
:103E3000E8D127F0FF07204647F09207FFF7CCFDB7
:103E40004F60CBE7962A13D1D0E9012303EBC203DD
:103E5000013513F8153C2D2B40F0AD802A46FFF7B5
:103E6000ECFE002800F0A7806368023B6360B5E7C2
:103E7000A2F11E03012B5FD9202A00F08380052ABE
:103E8000C0D10021FFF7AFFD0746002800F0938066
:103E900010F0030A05D1436803F0FE03562B00F02F
:103EA0008A8001212046FFF79EFD00F00F03022BC0
:103EB00040F08180BAF1000F7DD13B792C2B7AD173
:103EC000BB6803F00F02022A75D11B09482B72D17F
:103ED000FB68002B6FD09A076DD11A79302A6AD10E
:103EE000D3F808B04FEA10195846FFF74BFE0028E8
:103EF00040F0FD80B749B8480DF08AF8A1693A68EA
:103F00000968054653460DF065F92846FCF788F91F
:103F10001E2E0AD1FFF74DFF18BB3846FFF746FFAC
:103F200000B9D3460BF1FF3A0BE0FFF73FFFC0B9F2
:103F30003846FFF73EFFF3E705F1FF3A8DB1AB4698
:103F4000A94609F1FF3949462046FFF74CFD236990
:103F50006269A3EB0B03074642F82300B9F1000F97
:103F6000D6D10021514508D16D1A012D3FF436AF4D
:103F7000362E00F04281332E3DE12046FFF72CFD26
:103F80000131EFE70021FFF72EFD0746FFF70EFF97
:103F900068B93846FFF70DFF68B1EA212046FFF700
:103FA0001BFD204605B0BDE8F04FFFF762BD4FF4A2
:103FB0008571F3E72B26A91C89002046FFF71AFD1F
:103FC00046EA05230746C0F80080436000F1080177
:103FD000002D40F01B81962E03D139462046FFF775
:103FE00048FD3946DDE7922E00F0FE80062E00F0F7
:103FF0000481BDE7691E2046FFF7F5FC01A9FFF724
:1040000099FD0028B7D0022F9ABFA6F10D095FFADB
:1040100089F94FF02209AF1E002F09DA002D40F078
:10402000CD80019AD30740F1CE8042F00101B8E77C
:1040300039462046FFF7D7FC02A9FFF77BFD002891
:1040400099D0DDE9011201AB4846FFF753FD002886
:1040500091D0013FE0E7691E2046FFF7C4FC01A9AB
:10406000FFF768FD002886D0AF1E002FD6DD791E31
:104070002046FFF7B8FC02A9FFF75CFD00283FF4DB
:104080007AAF39462046FFF7AEFC00092438DDE957
:10409000011201ABC0B2FFF72DFD00283FF46BAF5A
:1040A000023FE2E700212046FFF79DFC01A9FFF750
:1040B00041FD00283FF45FAF01212046FFF793FC4C
:1040C000C0F30710332801990BD1CF0707D4880715
:1040D0007FF451AF0A68414B9A427FF44CAF022003
:1040E00001E03F38C0B209F0EDF8019096E758467C
:1040F000FFF76CFD4FEAC9030A46074643F0020189
:1041000004F128000AF00CFC47604846FCF7D3FF96
:1041100003785F2B204608D1FFF75EFC0025204680
:10412000FFF75AFCA84608266CE6FFF755FC5946EF
:104130002046FFF79EFC3EE701212046FFF753FC97
:1041400000F00F03022B07467FF415AF0021204635
:10415000FFF749FC00283FF40EAF10F003027FF494
:104160000AAF0379322B7FF406AF3909C900D0F8C2
:1041700008901B4841F002010AF0D2FB00283FF4EE
:10418000FAAE406802AA4FEA191108F0DDFF029B5F
:10419000002B3FF4F0AED9070AD49A077FF4EBAEB8
:1041A0001A680E498A4203D00E498A427FF4E3AE70
:1041B000039A002A7FF4DFAE01932FE72046FFF732
:1041C0000BFC013D2AE729462046FFF746FC014645
:1041D000E7E600BFAA8B050860E505080CEB0508BB
:1041E0008CD50508B4E80508D4E9012303EBC20324
:1041F00013F8053C2D2B7FF4DEAE2A4641462046BF
:10420000FFF71BFD00287FF4E9ADD4E62046FFF759
:10421000E3FB013D41F82500DAE600BF03460068F4
:1042200030B550B184070AD14468E5B28D4206D159
:1042300000F10803200A136030BD0346FBE70120AC
:10424000F9E700002DE9F04FA94B97B0CDE9073110
:1042500002900D4605A8A74901920024FBF7A6FF8E
:1042600040234FF40070CDE90934FCF701F8202316
:104270000B908020CDE90C34FBF7FAFF2146CDE905
:104280000E0513A8CDE911440AF014FB019B002B85
:1042900048D0022B0CBF3F2222460023696B964F69
:1042A00009A8FFF7FDFB00230A9C002C00F06481A5
:1042B000013C0B9991480A9401EBC40251F8341067
:1042C000D6785268C1F3170A8D4911F806B08D49A6
:1042D000895D632E88BF41F4807100EB41080BF0CB
:1042E000300110290BF00F091ED020294BD0002BD4
:1042F00000F01B81B9F1020F40F00A81012A40D081
:1043000000211BF0010F02F1FF3306D0B8F80200C4
:104310003840B0F5805F08BF5308012B40F0E580BE
:10432000E1B1E2E03D22B8E702B1BBB108EB4208DF
:1043300025E0C34638F8023B03EA0701B1F5805F88
:104340000ED195F83C10C3F30B03994216D109A87E
:104350003146FFF7B3FC2846FEF728FF0023A3E70A
:10436000531C4B4504D23246514609A8FFF798FB2F
:10437000BBF8001009A8FFF7B4FBEFE70132914545
:10438000D7D8012390E773B102F10043013B38F81D
:1043900013303B40B3F5405F21D1002109A80392BF
:1043A000FFF767FB039A08EB420491452BD8019B6A
:1043B00083B1052E0ED1002109A8FFF714FB48B9DF
:1043C000012109A8FFF70FFB830744D000F00F007D
:1043D000022845D1002408EB4903A1465AE0012AEE
:1043E000CFD995F83C30062B40F0F4804649474839
:1043F0000CF00EFE6A6B2968044600230CF0EAFEFE
:104400002046FBF70DFF039434F8021B01EA070076
:10441000B0F5805F16D195F83C00C9B288420ED144
:10442000082805D1314609A80392FFF747FC039AF3
:1044300003922846FEF7BAFE039A0132B5E7002A36
:104440009FD0CEE7531C5146324609A8FFF728FB00
:10445000039B19888EE70028BCD003793A2BB9D189
:1044600009A8FFF7B9FA09A8FFF7B6FA002308224E
:10447000514609A8FFF7A0FC70E733F8022D02EAC5
:104480000701B1F5805F10D1D2B2082A02D1013400
:1044900009F101094345F0D1B9F1010F1CD11BF01D
:1044A000400F19D00026314610E0214609A8039399
:1044B000FFF799FA039B08B109F101090134E9E713
:1044C000FFF78AFA0136002818BF0146A64209A85C
:1044D000F6D1FFF7CEFA41E71BF0800F04D00021A0
:1044E00009A8FFF7C6FA013423463246C0E700BFE9
:1044F000A33902084BD0020800F0FFFF78D6050868
:1045000000DA0508C8D50508B68B05083CE505089E
:10451000012A3FF436AF12F001013FF4F2AEB9F1D7
:10452000030F7FF45EAF0121EBE609EA020303F01B
:10453000010338F8134004EA0701B1F5805F13D195
:1045400095F83C10C4F30B04A14202F1010409D117
:104550001BB9314609A8FFF7B1FB2846FEF726FE36
:104560002246E2E72246C5E6531C5146324609A8D8
:10457000FFF796FA2146FDE613A80AF0AFF9129864
:1045800050B1416822460831FBF798FE129B5A68E9
:104590001A60119A5A60119395F83C30002B7FF401
:1045A00020AF0D9B002B3FF41CAF0E9B0B981B689C
:1045B0001093FBF785FE0E98FBF782FE0120FBF7B8
:1045C000FDFDDDE91001029B83E80300184617B0EA
:1045D000BDE8F08F022B01D1034908E7042B0CBF83
:1045E00002490349034803E7BF8B0508E68B05082A
:1045F000F98B050860E5050838B50446406808B938
:10460000606038BD4568FBF75BFE2846F7E70000B1
:10461000F8B5054630200E461746FBF742FE072D3B
:1046200004460570C66001D0012D0FD1B368C3F3F5
:104630000F13A38208F08AF9042320612783E384FF
:104640002020FBF715FEE0622046F8BD014B5B5DC4
:10465000EFE700BFB0DA050810B50446C06AFBF703
:104660002FFE2046BDE81040FBF72ABE30B5058D71
:1046700004460022954201D8002030BDE36A03EBD6
:10468000C20043688B42F8D00132F3E770B50446AC
:104690000D461646FFF7EAFFC0B9E38C228D9A4219
:1046A00008D30633D900E06AFBF7FDFDE38CE06236
:1046B0000633E384238DE26A591C02EBC300218593
:1046C00002F83360002343704380456070BD0346A9
:1046D00018465B68002BFBD1FFF7C8BFF8B54468EC
:1046E0000E462CB9F8BD042BFCD105230370F9E765
:1046F000254628466D68002DF4D077683946FFF7C7
:10470000B5FF0028F5D00378043B022BEAD8062534
:104710003570002239462046FFF7B8FF0378002B9A
:10472000E1D105706468F4E7036A1B8B012B1EBF9F
:10473000C3685B18C3607047836A10B504469B6FFB
:10474000406A9847238B226A0133918C9BB299422D
:10475000238338BF938410BD038B10B5013B0383C3
:10476000836A0446D3F88430406A98472046012182
:10477000BDE81040FFF7D8BF2DE9F04F85B00446E3
:104780000D46039298461BB1CB8A43F00803CB82B7
:10479000039BEB83236ADA8A42F03002DA821B78C9
:1047A000002B46D1A36A039AD3F8B460606A4346EB
:1047B0002946B44605B0BDE8F04F6047DB6A03EB1D
:1047C000C60B13F83630053B012B1DD84FF00009FE
:1047D00017E0EB6A03EBC90213F83930062B0ED150
:1047E000DBF804105368994209D1A36ABBF8022090
:1047F0001B69606A1F460023B8470AF1010A09F1E4
:1048000001092B8D4B45E4DC0136236A1A8DB24237
:10481000D4DCBAF1000FC5D0A36ACDF80080D3F87C
:10482000B860606A039B52462946B04705B0BDE8B0
:10483000F08F0026B246E8E7836A10B50446D3F845
:104840008830406A00219847A36A606A1B6B0F2179
:104850009847A36A606AD3F8CC3001219847204674
:104860000321BDE81040FFF75FBF38B5836A0446F7
:104870005B6C406A00229847A36A606AD3F8C05014
:1048800000231A461946A8472046BDE83840FFF7DE
:10489000D3BF836A89681B6D406A002209091847E3
:1048A000836A8968DB6B406A184710B5044608467E
:1048B00011461A46FFF7ACFE236A4360002383606B
:1048C000E3690BB9E06110BD1A469B68002BFBD170
:1048D0009060F8E72DE9F04F87B0054600AF0C4631
:1048E00011B90121116013E011F0030619D10B7900
:1048F000682B19D1CB681B0913608C68002CF0D091
:10490000012604F00F03022B0DD12109002EE9D05E
:10491000AB6A686ADB6A002298471C37BD46BDE86F
:10492000F08F0026EDE716B9A3681B091360A046B7
:1049300058F8043F4FEA132A08EB8A030AF1FF3BB9
:10494000BB60C14659F8040F0009FCF7A9FBBB681E
:1049500099458344F6D10BF1070323F00703ADEB30
:10496000030DC7F80CD0E946002358F8040F3B604C
:1049700007F114010009FCF7AAFB7A697A60014685
:10498000484625F06DF83B687A6801339A454A44F9
:1049900005D091464FF02E0209F8012BE5E7594664
:1049A000F868FCF7C3FAAB6A0146DB6A686A002262
:1049B0009847002EB1D00834BB689C42ADD054F863
:1049C000041FAB6A686A1B6D002209099847F3E768
:1049D00031B1826801F00303134304BF0B688360A5
:1049E00070472DE9F04107461E4659B111F0030505
:1049F00010D14B68D8B290420CD14FEA13280C1D4D
:104A0000454501DBBDE8F08154F8041F3846B04746
:104A10000135F5E738463346BDE8F0411847000058
:104A2000F8B504460E4611461A46002385780769F4
:104A3000837003610E4BFFF7D4FF6368BBB9618AD3
:104A400051B1228A42B9A36A606AD3F8A03098476C
:104A5000A36A606A1B6C9847238A628A31462046A3
:104A6000FFF78AFE003D18BF0125A5702761F8BD3C
:104A7000CD52020870B54378012B05460C4606D18D
:104A8000036A0A461B8B0221FFF70FFF2061A26811
:104A9000216928464C23BDE87040FFF7C1BF70B5BF
:104AA00013464278012A05460C4604D10A460721DE
:104AB000FFF7FBFEA061A669E2682846462331465F
:104AC000FFF7AEFFB08A70BD024B89689D22FFF7E9
:104AD00088BF00BFD9570208024B89686B22FFF7D5
:104AE00080BF00BF7173020838B543680D460446A5
:104AF00011464BB905480CF08BFA294660602046F8
:104B0000BDE83840FFF764BF38BD00BF60E5050869
:104B1000014AFFF7E9BF00BFFD8B05080B79092BA0
:104B200070B50CBF858AC58A4FF6FF739D42044657
:104B300002D1064AFFF7D8FF218B628BA36A606A15
:104B40005B6F8A1A2946BDE8704018470A8C050831
:104B500038B5054679B101F00F03022B0DD10C09D0
:104B6000204609F023FD002806DA064906482246B9
:104B70000CF0E4FA6860002038BD044AFFF7B4FF87
:104B8000F9E700BF238C0508F4E40508288C050824
:104B900070B51446054612780E4683B132B1032A29
:104BA00004D0104ABDE87040FFF79EBF0326267070
:104BB0006168286AFFF78BFD00B1067070BD62B9AD
:104BC00001232370006A2146FFF788FD2378012B1B
:104BD000F4D1054A31462846E4E7062AEED0034AD6
:104BE000E0E700BF2F8C05083C8C0508498C0508C0
:104BF0002DE9F3414378012B04460D461AD10B7978
:104C0000102B0CBF4FF001084FF0000808D0036ACA
:104C10001B782BB9114A02B0BDE8F041FFF764BF21
:104C200001AA6D2105F10800FFF7F8FA00260746F2
:104C3000B74202D102B0BDE8F081019B206A53F86F
:104C4000261000220909FFF721FD434602462946A6
:104C50002046FFF79DFF0136EAE700BF508C0508AC
:104C60004278012A0B4602D1006A02F013BE816A23
:104C7000026A406A203102F01CBE4278012A0B46CB
:104C800002D1006AFFF702BD816A026A406A1031F0
:104C900002F00FBE70B505460C4600292ED0CA079B
:104CA00006D5836A5B6B4910686ABDE87040184797
:104CB0008B0717D004F00F04022C4FEA11110AD011
:104CC000062C0CD0052919D0836A406A1B6BBDE8FD
:104CD0007040C9B21847BDE87040FFF7CEBF836A85
:104CE0009B6BE1E7836A0968DB68406A9847227931
:104CF000034B214653F822302846D6E770BD00BF4B
:104D0000B8DA05082DE9F74F05460C4616461F464A
:104D10002046FFF74BF840B16EB9AB6A9B6E39463F
:104D2000686A03B0BDE8F04F18472046FFF741F826
:104D300020B1002EF1D103B0BDE8F08F002C48D097
:104D4000A30746D163684FEA132BDBB21E2B18D1A1
:104D5000DEB1043404EB8B0B5C45ECD054F8041F3B
:104D60003B4632462846FFF7CDFFF5E75AF8041FC9
:104D7000019243462846FFF7C5FF09F10109019A50
:104D800011E01F2B1FD1002EE3D0D5F80C8008F1C5
:104D90000103EB600BF1FF3304F1040A4FF000094B
:104DA000009386F00102009B4B45DFDC0BF1010113
:104DB0003B4654F8211032462846FFF7A3FFAB6A62
:104DC00041469B6AACE7202B03D1A46886F001061C
:104DD0009EE721462846FFF75DFFAB6A686ADB6EF7
:104DE0003A46314603B0BDE8F04F184738B5026A7D
:104DF0001278072A04460B4606D0022A04D0BDE8E2
:104E00003840144AFFF770BE9D6885B9A36A606A8E
:104E10001B6B0F219847A36A606AD3F8CC3000213E
:104E2000984720460121BDE83840FFF77DBCAB071D
:104E30000BD12B79AF2B08D12046A968FFF72AFFA9
:104E40002046BDE83840FFF7F7BC29462046FFF76B
:104E500021FFE0E7628C050870B54378CE68012B2E
:104E60000446154606D1036A0A461B8B2946FFF7FE
:104E70001CFD7061002371691A462046FFF77CFC17
:104E8000F1682046FFF706FF062D05D1A36A606A88
:104E9000D3F8883000219847A36A606AD3F8BC50E1
:104EA0000023AC461A46BDE870400121604738B582
:104EB0000C460546C968FFF7EDFEA1682846BDE827
:104EC0003840FFF7E7BE0B79342B70B504460D462A
:104ED00010D18968FFF7DEFEED68AD6885B9A36A79
:104EE000606A1B6B0F219847A36A0422D3F8A03095
:104EF00002211AE0836A406A1B6B0F219847ECE796
:104F0000AB071FD12B799A2B13D1A36A606A1B6B55
:104F10000F219847A9680029E6D02046FFF7BAFE7E
:104F2000A36AD3F8A03004220321606ABDE8704070
:104F300018479B2B06D1A9682046FFF7ABFEEB680C
:104F40009968E8E729462046FFF7A4FECCE710B5AC
:104F500004468968FFF79EFEA36A606ADB6CBDE8C1
:104F600010400021184700002DE9F7438D680446E2
:104F700016465DB9002A75D0836AD3F8A0300222A4
:104F80002946606A03B0BDE8F043184715F00307EF
:104F900040F08A802B79372B13D132B1836A406A73
:104FA000D3F8A03002220121984720462946FFF776
:104FB00071FEA36A606AD3F8A43003B0BDE8F04381
:104FC00018479F2B70D1EB681A79A12A5AD1A221D8
:104FD00001AA03F10800FFF721F9A968804621B36F
:104FE0008B0722D10B79372B1FD136B1A36A411C15
:104FF000D3F8A030606A02229847A9682046FFF7DC
:1050000049FEA36A606AD3F8A43098474FF00109BB
:10501000474510D1B9F1000F24D1A36A606AD3F8D3
:10502000A0300322791C98471CE02046FFF732FE8F
:105030004FF00009ECE7019B53F82710A9B18E0748
:1050400013D10E79A6F13700464246412046FFF7BC
:1050500021FEB9F1000F11D04EB9184A2946204659
:10506000FFF742FD03B0BDE8F0830026EEE7A36A38
:10507000606AD3F8A43098470137C9E7002EFBD007
:105080000F4AEBE7AB685BB19A0709D11B79372B65
:1050900006D10422294603B0BDE8F043FFF7DCBE89
:1050A000052229462046F6E729462046FFF7F2FD6D
:1050B000A36A0322D3F8A030012162E76D8C0508B2
:1050C0007E8C05080122FFF74FBF70B50D46C968F9
:1050D0000446FFF7DFFDA968A36A606AD3F8983039
:1050E000C1F30711332918BF3F39BDE8704014BF21
:1050F000C9B202211847F8B54F680C4689680546C1
:10510000FFF7C8FD3F0A0C3400260236B74204F10F
:10511000080400DCF8BD54F8041C2846FFF7BAFD6B
:1051200054F8081CAB6A686AD3F89C300909243922
:10513000C9B29847E9E72DE9F0410C464E6854F8AA
:10514000081F0546FFF7A6FDA6F10D085FFA88F8CF
:10515000360A0127B74201DBBDE8F08154F8041F8D
:105160002846FFF797FDAB6A686AD3F89C30414642
:1051700098470137EEE72DE9F0414E6804460D46A9
:10518000360A8968FFF786FD032E83BFD4F80C80AA
:1051900008F10103E3604FF0000801277B1C9E42E9
:1051A00022DC032E55D9E568606A6B1CE360A36AB4
:1051B00029469B6E9847A36A606A9B6A4146984756
:1051C000A36A606A9B6801219847A36A606A1B6EA4
:1051D0009847A36A606ADB6D9847A36A606A9B6A16
:1051E0002946BDE8F0411847296920460237FFF7F4
:1051F00051FDB74207DAA36A606A5B6D9847A36AFC
:10520000606A5B6E9847EB68A26A606AD2F89C207D
:1052100003F00F010A2911D1C3F30713252B1ABF7D
:10522000343BD9B206219047B74205DAA36A606AD7
:105230001B6F4246002198470835AFE71979852949
:1052400001D13221EFE79B680BB90721EBE733214E
:10525000E9E7BDE8F08110B504468968FFF71AFD5B
:10526000A36A606AD3F89830BDE81040032118475C
:105270002DE9F0470D46D0F80C8055F8046F5FFA21
:1052800086F9A9F11E03D3F1000949EB030908F1DE
:1052900001030446C360360A0027B74206DBA36A4F
:1052A000606A9B6A4146BDE8F047184755F8041FFD
:1052B00020460137FFF7EEFCB742F0DAA36A606AD6
:1052C0001B6F424649469847E7E7000001F00F038D
:1052D000022B70B5044612D00B79492B09D0483BFC
:1052E000082B18D8DFE803F008170717171717055A
:1052F00007000123A37070BD8E680D6975B9A3788E
:10530000002BF8D1638A002BF5D020461D4ABDE85A
:105310007040FFF7E9BBD1E90265EFE7A3783BB343
:10532000238A01339BB2012B23820ED1618AD4E9F7
:105330000903D1B1D3F8A03000229847A36A606A6C
:10534000D3F8A03002220021984729462046FFF7D3
:10535000A1FCA36A606A9B6B31099847A36A606AE3
:10536000D3F8A430BDE8704018471B6C9847E5E7B8
:10537000638A0133638229462046BDE87040FFF707
:1053800089BC00BF898C05082DE9F041C568D1F8BA
:105390000C800E46AB1C04460022D8F80810C360EF
:1053A0002B46FFF7AFFCB1682046FFF773FCA36AFA
:1053B000606A9B6E6F1C39469847A36A606A9B6A55
:1053C00029469847A36A606A9B684FF0FF31984767
:1053D000D8F80C102046FFF75DFCA36A606A9B6A50
:1053E0003946BDE8F04118472DE9F047C668D0F8C6
:1053F00014A0B0F81A908682B31CC36006F10108AD
:10540000038BA0F816800446438388680D46FEF798
:10541000CDFCF8B9E768A8687B1CE360FEF7C9FC1F
:1054200020B9A36A606A9B6E41469847A36A606A86
:105430009B6A39469847E9682046FFF72BFCA36A28
:10544000606A9B6A41469847A9683B46012220460C
:10545000FFF758FC2969C4F814A02046A4F81A9054
:10546000FFF718FCA36A606A9B6A3146BDE8F04703
:1054700018472DE9F347C668731CC3600446886863
:105480000D46FEF793FC0246E8B9E768A9687B1C65
:10549000E36020463B46FFF735FC2046E968FFF70E
:1054A000F9FBA868FEF785FCD8B92B690BB96B69C5
:1054B00023B1A36A606A9B6E31469847A36A606A0B
:1054C0009B6A3946984701AA712105F11000FEF741
:1054D000A5FE002781464F450BD169692046FFF79D
:1054E000D9FBA36A606A9B6A3146984702B0BDE85F
:1054F000F087019B53F82780D8F80800FEF756FC88
:10550000024600BBD4F80CA0D8F808100AF1010339
:10551000E36020465346FFF7F5FBD8F80C10204611
:10552000FFF7B8FBD8F80800FEF743FCD4E90923DD
:105530000028D6D19B6E314610469847A36A606A10
:105540009B6A514698470137C5E70000184B2DE983
:10555000F041D3F8007204460D463FBBC668896827
:10556000731CC36001223346FFF7CCFBA36A606A59
:105570005B691F2101229847E96851B12046FFF776
:1055800089FBA36A606AD3F8BC503A463B460121C6
:10559000A847A36A606AD3F8C83001219847A36A74
:1055A000606A9B6A3146BDE8F0411847BDE8F0816A
:1055B0007004002070B58D6804463DB9836AD3F845
:1055C000C8302946606ABDE870401847AB070ED165
:1055D0002B795E2B0BD1A968FFF75CFBE9682046AD
:1055E000FFF758FBA36A0221D3F8C830EAE729463F
:1055F0002046FFF74FFBA36A0121D3F8C830E1E74B
:1056000010B504468968FFF745FBA36A606ADB6D45
:10561000BDE81040184700002DE9F041026A1278F9
:10562000072A044604D0BDE8F0411A4AFFF75CBAE5
:105630008D685DB9836A406A1B6B0F219847A36A26
:10564000606AD3F8C430BDE8F041184715F0030292
:105650001DD12B791B2B1AD1C668EF68731CC36050
:10566000B9683346FFF74EFBA9682046FFF712FBE7
:10567000A36A606AD3F8C4309847A36A606A9B6AD9
:1056800031469847F9682046FFF704FBD7E72946DB
:10569000F9E700BFA78C05082DE9F0410C46054647
:1056A00054F8046F360A04EB8607BC4208D1AB6A93
:1056B000686AD3F8A03031460022BDE8F0411847AF
:1056C00054F8041F2846FFF7E5FAEEE7896810B49E
:1056D000034641B9826A406AD2F8A0400A4623468E
:1056E0005DF8044B18474A68120A022A0BD1CA68AF
:1056F0004AB1940707D11279AC2A04D15DF8044B62
:105700000622FFF7A9BB5DF8044B1846FFF7C4BF9C
:105710002DE9F0410E46054656F8043F0F464FEA84
:1057200013280024444501DBBDE8F08156F8041F2E
:105730002846FFF7AFFA6B683BB10234284657F8AA
:105740002410BDE8F041FFF743B90134EAE710B592
:105750000446FFF7DDFFA36A606AD3F89C30BDE81A
:1057600010402221184770B58D68044645B9836AF8
:10577000D3F8A03001222946606ABDE8704018477E
:10578000A9071ED16B68DAB2922A1AD11B0A022B22
:105790000CD1EB6853B19A0708D11B79AC2B05D11A
:1057A00029460322BDE87040FFF756BB2946204634
:1057B000FFF7AEFF6968A36A0122D3F8A030090A97
:1057C000DAE729462046FFF765FAA36A0122D3F8F3
:1057D000A0301146D0E7000001F00F03022B2DE9A5
:1057E000F04705460C4604D1BDE8F0470909FFF72C
:1057F00037BA002955D011F0030652D10B792C2B62
:1058000038D18968FFF746FAE668002E49D016F0CD
:10581000030846D17768FAB28E2A334609D13F0A87
:1058200006F1040907F1FF3AC24510DC013756F8CA
:1058300027301A79312A12D199682846FFF72AFAB7
:10584000AB6A686ADB6CBDE8F0470221184759F87B
:10585000041F2846FFF71EFA08F10108E4E7322A80
:105860001FD19968AB6A686A1B6DBDE8F0470222D8
:10587000090918472D2B14D18C6894B163681B0A51
:10588000022B06D0271D6368B6EB132F10D3BDE89B
:10589000F087E368002BF5D09A07F3D11B79AC2B86
:1058A000F0D121462846064ABDE8F047FFF71CB96B
:1058B00057F8041F2846FFF78FFF0136E3E700BFC4
:1058C000B38C05082DE9F8430446006AC68A1746DA
:1058D000B2070D4606D5374A29462046BDE8F843AB
:1058E000FFF702B901F00F02022A18D1A3780909C3
:1058F0008BB1838B013383834FF000094FF0010894
:10590000002955D00022FEF7C1FE03780646002B81
:1059100038D0294AE0E7438B01334383ECE70A7927
:10592000BA4289460BD18968A37809091BB1838BD8
:1059300001338383E2E7438B01334383DEE79A42FB
:1059400018D1A378002BC6D10122A270896879B33F
:1059500001F00F02022A18BF894646F0040618BF5C
:10596000D9F80810C68206BF0909994609094FF0FF
:105970000308C5E7896846F002060909C6824FF0A8
:105980000508BDE70423037080F80180236A1B8BA0
:10599000032B0DD1482F0BD1B9F1000F08D0D9F846
:1059A0000C102046FFF7D4F8737843EA00137370A5
:1059B000BDE8F883F98B0508BD8C0508492348220A
:1059C000FFF780BF4F234E22FFF77CBF2DE9F04F3A
:1059D0000E468DB0016200214270C1603378072B02
:1059E0000446154605D08B4A0DB0BDE8F04FFFF7D1
:1059F0007BB8012A05D0036B021D1B68C06A2946CB
:105A000098476378D6F80C80032B10D10BAA462157
:105A100008F10C00FEF702FC236B0B9A9B68014611
:105A2000E06A984763687083002B40F0BC80D8F828
:105A30001010C1B101F00F03022B10D10B09752B0F
:105A40003FD006D83E2B3ED05E2B0CD0724A20466B
:105A5000CAE740F2EA429342F8D1032304E06F4AD6
:105A60002046FFF741F80223049309AAD8F814301E
:105A70000893192108A8FEF7D1FB4FF00009069002
:105A8000069B994521D16378012B16D9236B049984
:105A90005B68E06A98476378042B0ED1206A049B08
:105AA000E26A0393438B02930023CDE9003305217F
:105AB000D2E90232006906F059FF6368002B72D107
:105AC00014E00023D0E70123CEE7099B53F8291007
:105AD0000B79082B4FEA890B02D109F10109CFE7B5
:105AE000052B06D04E4A2046FEF7FEFF0DB0BDE85E
:105AF000F08F8B68002BF5D09A07F3D1CA68002A83
:105B0000F0D11A792C2AEDD19E6806F00F02022AF4
:105B1000E8D1D3F80CA0BAF1000FE3D01AF0030FCC
:105B2000E0D19AF80430302BDCD10AAAA4210AF182
:105B30000800FEF773FB360940F2F9339E42074630
:105B40001BD1012805D10A9A136803F00F03022B19
:105B500004D0344A099B53F80B10C4E7E168012DC7
:105B600001F10103E3601AD01268236BE06ADB687D
:105B70001209984798B92C4AECE740F232339E421A
:105B800015D1012803D10A9B1968CB0701D4274AF4
:105B9000E0E7012D03D0E06A491002F0BFFB636823
:105BA000002B9AD0D046D8F80030A3609EE7B6F517
:105BB0005E7F23D1012804D90A9B1A6812F00106DE
:105BC00001D11B4AC6E7012DE9D0531007930A9A69
:105BD0000BA952F82600FEF7D5F808B9154AB9E71F
:105BE000E36A0B9805930CF0DCFC0136024607993A
:105BF000059802F09AFBB742E9D1D0E7012DCED04B
:105C0000236B0246D3F810B0E06A0A9B3146D847AE
:105C1000C5E700BFC78C0508DD8C0508E18C0508C9
:105C2000E98C0508F78C0508038D0508078D050824
:105C3000138D0508258D05084278012A0B4602D1EF
:105C4000006A01F027BE816A026A406A183101F0D9
:105C500030BE00002DE9F14F8F0704460D46164671
:105C600013D001F00F03022B18D102F0FD06012E14
:105C70004FEA111104D001B0BDE8F04FFFF7DCBFCF
:105C800001B0BDE8F04FFEF7F8BF4968CBB22D2B4D
:105C90007FD00BD8062B0ED02C2B13D0514A29467F
:105CA000204601B0BDE8F04FFEF71EBF2E2B00F0DE
:105CB00084809D2BF2D1002EF0D105F10802090A53
:105CC00020467FE0022A02D0A968FEF7E3FFEF68D2
:105CD000002FE3D017F00309E0D17B68DAB28E2AF7
:105CE000B8460DD1022E4FEA132805D007F1040A59
:105CF00008F1FF3BD94515DB08F1010857F828806A
:105D000098F80430312B27D1022E13D1A36A606A90
:105D10005B6E9847A36ADB6C0121606A01B0BDE845
:105D2000F04F18475AF8041F2046FEF7B3FF09F159
:105D30000109DFE72046D8F80810FEF7ABFF012E77
:105D4000D4E9090305D19B6D9847A36A0021DB6C58
:105D5000E3E7DB6C0121E1E7322B9FD1012ED4E98F
:105D600009030CD15B6D9847A36AD8F808101B6D26
:105D70000022606A090901B0BDE8F04F1847022E01
:105D800001D11B6E9847A36AD8F808101B6D012239
:105D9000EFE7AA68002A81D0002E7FF47FAF516818
:105DA000090A022907D1D3682BB1980703D11B79BF
:105DB000AC2B3FF473AF083282E7002A7FF46EAF5A
:105DC000A96821B901B0BDE8F04F00F073B88E07A3
:105DD00003D10B79922B0A46E1D005F1080201218B
:105DE0006EE700BF308D05082DE9F047C7681E46F5
:105DF000BB1CC360836A04460D469B6A406A3946F1
:105E000090469847A36A606AD3F88C3007F101097D
:105E100049469847A96800222046FFF71BFF2D69D5
:105E200065BB41462046FEF735FF236A19780629EF
:105E3000D4E909031CD1D3F8CC3029469847204631
:105E40000121FEF771FCA36A606ADB6D9847A36AC3
:105E5000606A9B6E39469847A36A606A9B6A4946A6
:105E60009847A36A606AD3F89030BDE8F0471847B6
:105E7000B200D3F8A83005329847E8E72B79AD2B6C
:105E800007D1A9683B4600222046FEF73BFFED689C
:105E9000C6E7E9682046FEF7FDFEA36A606AD3F80C
:105EA000883001219847731C424629462046FFF757
:105EB0009BFFCCE72DE9F84304460D46904601F1DF
:105EC000FF3900264FF0FF37B9F1FF3F0CD17B1CA3
:105ED00005D1A36A606AD3F8AC30294698470026FA
:105EE000AE421DD1BDE8F88358F8261071B18A077B
:105EF0000CD10B79222B09D101370BD1A36A606A2F
:105F0000D3F8B0304A46314698473746013609F152
:105F1000FF39D9E72046084ABDE8F843FEF7E4BD5B
:105F200058F82610B74208BF896800222046FFF7BC
:105F300091FE0136D4E700BF3B8D05082DE9F047FF
:105F40000446904699460F4621B9BDE8F0471946E8
:105F5000FEF7A0BEC668731CC360156835B315F0A4
:105F6000030A23D12B797B2B20D1A968FEF792FE5F
:105F7000524631462046FEF7DFFBE968524620468E
:105F8000FFF768FE4B4608F10402791E2046FFF732
:105F9000D5FFA36A606ADB6F31469847204603212C
:105FA000FEF7C2FBBDE8F047FEF7D6BB2946204608
:105FB000FEF770FE204600223146FEF7BDFBA36AC5
:105FC000606ADB6D9847DDE737B50C46054601AAE8
:105FD0007A2104F10800FEF721F9E368019A0146ED
:105FE0002846FFF7ABFF03B030BD2DE9F04F8B68BB
:105FF00003F00F03022B89B004460D4640F00081E8
:10600000CB68002B00F0FC80980740F0F9801A79EB
:106010002C2A40F0F5809A6802F00F01022940F026
:10602000EF8012097C2A40F0EB80DB681A79302A75
:1060300040F0E6809B68069307AAA42106A8FEF715
:10604000EDF8431E022B00F2DB80079B01281A6843
:1060500000F0C980022800F0C4809E68F10740F17A
:10606000CF80710800F0CC80D3F8049032B1930750
:1060700004D11179A639022940F2C280B9F1000F8A
:1060800008D019F0030F05D199F80410A639022998
:1060900040F2B680AB6801932B696F690293E568A3
:1060A0006369218B0493638B039305F1010BAB1C94
:1060B000618319F0010805F104010593A582A4F894
:1060C00016B005F1030AE16005D149462046059264
:1060D000FEF7E0FD059A11462046FEF7DBFDA26AB9
:1060E000606A926E51469047A26A606A926AA91CE1
:1060F0009047A26A606A526D90470022019920463B
:10610000FFF7A8FD02992046FEF7C4FDA26A606A67
:10611000926A5946904731462046FEF7BBFDA26A77
:10612000606AD2F89C200E219047A26A606A926A47
:1061300051469047D4E90902B8F1000F57D1936D49
:106140009847A36A606A1B6E9847A36A606AD3F88F
:106150009C30002EACBF002101219847A36A606AE1
:10616000DB6EAA1C01219847049B6361039B638338
:10617000002F43D0A36A606ADB6D9847B8F1000F27
:1061800003D1A36A606ADB6D984739462046FEF763
:1061900081FDE668606A731CE360A36A31469B6E0A
:1061A0009847A36A606A9B6888F0010101319847AB
:1061B000A36A606A9B6A29469847A36A606ADB6D96
:1061C0009847B8F1000F03D1A36A606ADB6D984766
:1061D00027B1A36A606A9B6A3146984709B0BDE857
:1061E000F08F032640E791460326024646E7526DAC
:1061F000904749462046FEF74DFDA6E73E46D7E7C5
:10620000E668238BB4F81A9063836FEA46436FEA1B
:106210005343D4F814A0A382771CF31CE968E3600D
:106220002046E782FEF736FDA36A606AD3F888301D
:1062300001219847A36A606A9B6A39469847A36A16
:10624000606AD3F88C3006F1020841469847002274
:10625000A9682046FFF7FEFC29692046FEF71AFDD3
:10626000A36A606A9B6E39469847A36A606A9B6A14
:1062700041469847A36A606AD3F8903098476969A5
:10628000C4F814A02046A4F81A90FEF703FDA36AF0
:10629000606A9B6A314609B0BDE8F04F18472DE9A6
:1062A000F74F0446174698460E4629B9194603B0DB
:1062B000BDE8F04FFEF7EEBCC5682B1DC360136848
:1062C00005F1010A05F1020B05F10309002B00F0AD
:1062D000D28013F0030240F0CE8019797B2940F080
:1062E000CA80996801920093FEF7D4FCA16A606AA3
:1062F000496D884740F20D312046FEF7B6FADDE9D8
:1063000000322046D968FFF7A5FC02222946204624
:10631000FEF712FAA36A606A9B68032198473A1D48
:106320004346711E2046FFF7BAFFA36A606A9B6866
:106330006FF002019847A36A606AD3F880602A462A
:1063400051465B46B047A36A606A5B6D9847A36A93
:10635000606A5B6E9847A36A606A1B6E9847A36A7F
:10636000606A5B6C002240F20E319847A36A606A53
:106370005B6E9847A36A606A5B6E9847A36A606A1F
:106380005B6D9847A36A606A1B6D00220A219847DB
:10639000A36A606A1B6E9847A36A606A1B6B0F2131
:1063A0009847A36A606AD3F8C05000231A460321B5
:1063B000A8472046FEF740FAA36A606ADB6E4A46A9
:1063C00000219847A36A606ADB6D9847A36A606AF8
:1063D0001B6B0F219847A36A606A9B6E49469847DA
:1063E000A36A606A9B6802219847A36A606A9B6AF5
:1063F00059469847A36A606A5B6E9847A36A606AC9
:106400005B6E9847A36A606A9B6A51469847A36A85
:10641000606A5B6C002240F20E319847A36A606AA2
:106420001B6B0F219847A36A606A5B6D9847A36A4C
:10643000606A5B6D9847A36A606AD3F8C050002316
:106440001A460321A8472046FEF7F6F9A36A606AB8
:10645000DB6D9847A36A606A9B684FF0FF319847ED
:10646000A36A606A9B6A49469847204603B0BDE824
:10647000F04FFEF771B919462046FEF70BFCA36AF0
:10648000606A5B6D9847204640F20D31FEF7EDF9EA
:10649000A36A606ADB6D984737E72DE9F041CD6864
:1064A00004460E4665BB0378C3B1036A1D78ADB9D7
:1064B00040F21B31FEF7E1FBB1682046FEF7EAFB34
:1064C000A36A606AD3F8BC602A462B460121B04714
:1064D000A36A606ADB6DBDE8F0411847B1688B07BD
:1064E00007D001F00F03022B08D12046FEF7D2FBA4
:1064F000EEE70029F9D00B793A2BF6D1BDE8F0810F
:10650000AF0740F0AF806B68DAB25B2A11D1ED685B
:10651000002D4AD1006A0378072BEFD1896801F07A
:106520000F03022BEAD10422BDE8F041D140FEF76F
:10653000ADB8562A13D101228968FFF78BFBE968B1
:106540002046FEF7A7FBA968A36A606AD3F89C30CF
:1065500009093E39C9B298470222B1687DE0572A3D
:1065600025D11B0A5F1E013355F82310FEF792FB5D
:10657000002F03DDA36A606A5B6D9847B168002253
:106580002046FFF767FB04350026BE42B6DA013627
:10659000BE4203DAA36A606A5B6D984755F8041F30
:1065A00000222046FFF756FBEFE7A9075AD16B6898
:1065B000DAB2062A56D1B768002F53D0BA0751D1A4
:1065C0007A68D1B206294DD11B0AB3EB122F4FEADC
:1065D000122847D1A8F10203012B43D8BB6823B18D
:1065E000980702D11B79222B3CD0FB6823B1990775
:1065F00002D11B79222B35D0B8F1020F06D03B69AE
:1066000023B19A0702D11B79222B2BD0A9682046EF
:10661000FEF740FBE9682046FEF73CFBB8F1030FAC
:1066200007D120462969FEF735FBA36A606A5B6ED5
:106630009847A36A606A1B6E9847B9680022204693
:10664000FFF708FBF96800222046FFF703FBB8F1CB
:10665000030F7FF453AF396900222046BDE8F041B3
:10666000FFF7F8BA29462046FEF714FB002274E72C
:106670000023032A2DE9F04104460D4616464270D8
:106680000162C36080F8342002D1C08E50BBA06389
:10669000A36A606A1B684FF000083146A4F8368090
:1066A0002A46984706212046FEF73EF86778EE68AE
:1066B000012F04BFA5F82280A5F82480B6B1B20747
:1066C00014D133793F2B11D1B168FEF7E3FAA36AF5
:1066D000606AD3F8C4309847A36A606A5B68BDE813
:1066E000F04118478000F9F7DCFDD0E72B78072B45
:1066F00000F29380DFE803F0049125414141410E0F
:1067000031462046FEF7C6FAA36A606A1B6B0F216A
:106710009847DCE7012F12D10023A370F168574B93
:1067200046222046FEF75DF92B8B032B07D13169FA
:106730002046FEF70DFAEB8A43EA8013EB8271697B
:10674000DFE7A36A3168DB68606A98476378012BEA
:1067500007D10023A370B168494B4C222046FEF7B5
:1067600040F9F1682046FEF795FAEB8ADB07AED5D3
:10677000A36A606ADB6D9847C6E7012FD6F80C80E4
:1067800005D1206A04223946FDF780FF6F83A36A92
:106790003168DB68606A98472B78032B24D1A36AA1
:1067A000D3F8A0300122606A002198472B78062B8D
:1067B00028D1A36A606A1B6C984701212046FEF726
:1067C0005CFAA36A606A1B6C9847A36A606A1B6CD8
:1067D00098470023B26841462046FFF705FB2B7817
:1067E000062B7FF474AF8FE7042B04D1A36A022237
:1067F000D3F8A030D7E7052BD8D1A36A0322D3F86A
:10680000A030D0E720460121FEF737FAA36A606A7C
:10681000D3F8883001219847DBE7012F04D1042207
:106820000A212846FDF732FF17212046FEF725FAF8
:1068300016212046FFF700FAB168A36A606A9B6BD5
:10684000090998471A212046FFF7F6F931692046D1
:10685000FEF720FA0A212846FDF708FF0246D4E990
:1068600009031178042902D11B6B0F2150E71D6920
:10687000528800230A21A84729E700BFBD59020812
:10688000C5590208036A10B51A8B0446FEF707F9CA
:1068900001462046BDE81040FFF7CEB92DE9F04F84
:1068A0008D682B79032B85B004460AD12946FFF762
:1068B000E9FFAA69D38A43F00103D38205B0BDE89A
:1068C000F08F026AD28AD20706D4624A294605B0FE
:1068D000BDE8F04FFEF708B9162B40F0AD80C66852
:1068E000E968331DC360FEF7D5F9A36A606A5B6C83
:1068F000002240F20F319847A36A606AD3F8C07053
:1069000000231A461946B847E76863690093638B0A
:106910000193BB1CE360238B6383A36A606A9B6A59
:10692000A78207F1010806F1010B4146A4F8168081
:106930009847012259462046FDF7FEFEA36A606A89
:106940005B6D9847204640F21131FDF78EFFA96834
:1069500020460022FFF77EF9A36A606AD3F89430DC
:1069600006F10209002249469847A36A606A9B6AB9
:1069700059469847A36A606AD3F8D0309847A36A0B
:10698000606A5B6D9847A36A606A5B69012240F2A6
:10699000C7219847A36A606AD3F89C3008219847BA
:1069A000A36A606ADB6E06F1030A5246002198472B
:1069B000A36A606ADB6D9847A36A606AD3F8943073
:1069C000012231469847A36A606A9B6A51469847FC
:1069D000A36A606A9B68012198472046FDF7BCFEC8
:1069E000A36A606AD3F8D4309847A36A606A9B6A46
:1069F0004946984729692046FEF74CF9A36A606A20
:106A00009B6E41469847009B6361019B6383A36A29
:106A1000606A9B6A3146984769692046FEF73AF9F1
:106A2000A36A606A9B6A39469847A36A606ADB6D0D
:106A300005B0BDE8F04F184703AA7A2105F1080018
:106A4000FDF7ECFBEB68039A01462046FFF727FCB5
:106A500034E700BF428D05082DE9F04F85B0C568C9
:106A60001E460E9B03936B1C0293AB1C0446C36033
:106A70000F46934629460122FDF75EFE3946204621
:106A8000FEF708F9A36A606AD3F894300022691C03
:106A90009847A36A606A9B6A29469847A36A606A16
:106AA000D3F8D0309847D4F80C9009F10103E36093
:106AB00000275F4518DB2046FDF74EFEA36A606A9B
:106AC000D3F8D4309847A36A02999B6A606A9847C2
:106AD00003992046FEF7DEF8A36A606A9B6A49467E
:106AE00005B0BDE8F04F18473346D4F80CA01A683B
:106AF00001920AF10102E260019AD2F8088004369C
:106B00000137B8F1000F4FD1BB4542D1A36A606A8B
:106B1000DB6D98470025A846019B2046D968FEF703
:106B2000B9F825B3A36A606A1B6B0F219847A36A63
:106B3000606A9B6A41469847A36A606A9B68012124
:106B40009847A36A606A1B6B0F2198472946204625
:106B5000FFF772F829462046FEF782F8A36A606ABA
:106B60009B684FF0FF3198472046FDF7F5FDA36A7B
:106B7000606AD3F89430012249469847A36A606A54
:106B80009B6A51469847A36A606A9B6801219847AF
:106B90008FE720461E4A1968FDF7A6FF204605B07C
:106BA000BDE8F04FFDF7D8BD18F003052DD198F8DA
:106BB0000420762A434603D1DD68D8F808802D09E1
:106BC000A36A606A5B6D984741462046FEF762F80B
:106BD000A36A606AD3F89C3008219847A36A606A68
:106BE000DB6E524600219847002D8FD02946204663
:106BF000FFF722F8D4F80C8008F10103E3600222C9
:106C000041462046FDF798FD86E70025D8E700BFFE
:106C1000598D05082DE9F347C76898467B1C164631
:106C20000D46C36002223946DDE90AA90446FDF794
:106C300083FD002E2DD1A36A606A9B6803219847CB
:106C400029462046FEF726F8A36A606A9B686FF023
:106C500002019847A36A606A1B6B0F219847A36AD9
:106C6000606A9B6A39469847A36A606A9B680121FB
:106C7000984749462046FEF70DF8A36A606A9B686C
:106C80004FF0FF319847204602B0BDE8F047FDF7CE
:106C900063BDCDF800A04346324629462046FFF7A3
:106CA000DBFED7E7F0B5CE683379782B85B00546A3
:106CB0000C4609D1B36801930023009389681A46F2
:106CC000FFF7A8FF05B0F0BD742B03AA4FF07701C2
:106CD00013D106F10800FDF7A1FA3769A168039BFB
:106CE0000246F06827B900902846FFF7B5FEE9E7AD
:106CF000BC68CDE900042846E2E704F10C00FDF78A
:106D00008DFA00230093A168039B0246ECE7000084
:106D100001F00F03022B70B504460D46164602D053
:106D20001E4AFDF7E1FE31462046FDF7B3FFA36A98
:106D3000606A5B6D98476378012B4FEA151610D196
:106D4000226A1378033B032B0BD85068314600F0BE
:106D5000A1FD0346206A1A78032A08D13146FDF7BF
:106D600095FC31462046BDE87040FEF765BF002225
:106D70003146FDF78BFC236A5B685B68002B02469B
:106D80000CBF0123002304D00178012904BF002196
:106D9000017029462046FDF7FBFEE2E7308D05082D
:106DA0002DE9F04F87B0CDE90221044605AAA421C0
:106DB00003A81D46FDF732FA00260190B14637467A
:106DC000B0464FF0010B019B9E4211D127B1A36A3F
:106DD000606A5B6B49469847029AD4E90903002A26
:106DE00076D0D3F8C0403B4642462946A04713E040
:106DF000059B53F826A0BAF1000F5BD01AF0030FE1
:106E000058D19AF80420A62A1AD1B80707D5324AD1
:106E100051462046FDF768FE07B0BDE8F08F1D2EF5
:106E200001D92E4AF4E70BFA06F2DAF808102046E8
:106E300049EA0209FDF72EFF013501270136C2E7B5
:106E4000A72A0DD1A26A606A126C9047DAF808107E
:106E500047F002072046FDF71DFF08F10108EDE7A6
:106E6000A82A27D1DAF80C2072B191070CD1117938
:106E7000AA2907D19268DAF808102046FFF748FFE0
:106E80000135DBE7AC290FD0DAF8081001F00F026A
:106E9000022A01D0124ABBE7A26A606A926B090912
:106EA0009047DAF80C10D5E7062251462046FDF748
:106EB000D3FFE5E7BB0701D50A4AA9E7B8F1000F00
:106EC00001D0094AA4E751462046FDF7E3FED7E783
:106ED000D3F8BC4087E700BF718D0508788D0508A1
:106EE000848D0508918D0508988D050870B50D46AF
:106EF000417801290446134603D12A46FDF7D5FC03
:106F00006861A36A606A9B6C98476E6900231A46A1
:106F100031462046FDF730FCA36AB18A9B6B606A5C
:106F20009847E96829B18B0703D10B79A32B08BFD8
:106F30000021204602230022FFF732FFB08A70BDF5
:106F4000002389681A46FFF72BBF00002DE9F8439C
:106F50000C4689680546FDF79DFEE668002E56D072
:106F60007768296AFBB209788E2BA36819BF04F1F0
:106F70000C0601273F0A0836072903F00F024AD101
:106F8000022A46D11A099A2A47D133681A79302A37
:106F90003FD19B68002B3CD10A212846FDF76DFEAE
:106FA0002A6AD36A128D32B93168404A2846BDE850
:106FB000F843FDF799BD5978C9070FD55968284698
:106FC000FDF75BFE022FD5E909030AD8D3F8BC40D0
:106FD00000231A460221A047012416E0013A083393
:106FE000E1E7726811793229F0D1B468217930294A
:106FF000ECD191685B6C012209099847A1680023D4
:1070000001222846FFF7CCFE0324A74225D8BDE87D
:10701000F8830024F9E7022AFBD11B09B3F5057FA9
:10702000F7D133681A79302AF3D19B68002BF0D05E
:1070300013F00304EDD11B792F2BE6D1AB6A686AFC
:10704000D3F8BC80224623462146C04733682246F7
:1070500099682846FDF788FFBEE704F10108B845A6
:1070600056F824104FEA84031AD20A79322A17D12B
:107070003344D3F8049099F80430302B10D1896848
:10708000AB6A686A5B6C002209099847D9F8081056
:10709000002301222846FFF783FE08F10104B4E72C
:1070A0002846FDF7F7FDA046F7E700BF9F8D0508CE
:1070B00010B5026A1278072A04460B4606D0022A47
:1070C00004D0BDE81040064AFDF70EBD2046194623
:1070D000FFF73CFF2046BDE81040FDF7ADBB00BF09
:1070E000B28D0508D1E90212FFF712BE036A10B58E
:1070F0001A8B0446FFF7FAFE01462046BDE8104011
:10710000FEF79ABD2DE9F04F044685B0884602AAE5
:10711000422108F10800FDF781F8236A00271E8B41
:107120008346BA465F450AD1D8F80C100B79032B79
:1071300051D132462046FDF7B2FC054659E0029B8C
:1071400053F82730019303AA6C2103F10800FDF7DF
:1071500065F8039B19680A09732A05460DD0204675
:10716000FDF798FD4FF00109A94528D3019BD96887
:1071700069B12046FDF78EFD09E0022809D02A4AB0
:107180002046FDF7B1FC35460AF1010A2E460137CB
:10719000C8E759680B09412B0DD040F239429342A0
:1071A000F2D040F2FC42934207D040F23D3293428B
:1071B000E5D10425E8E70125E6E70325E4E7039B9D
:1071C000606A53F82910A36A00221B6D09099847C9
:1071D00009F10109C8E7442B17D18F6832463946B7
:1071E0002046FDF75CFCBA69D38A43F001030546EB
:1071F000D3820027ABEB0A0ABA450BD829462046B2
:10720000FEF71AFD05B0BDE8F08F32462046FFF7C5
:107210006DFE92E7A36A606AD3F8BC6000231A4649
:107220000121B0470137E7E7BD8D05082DE9F3419E
:107230008D6805F00F030A2B04460E4607D0002D7B
:1072400031D015F003012ED12B79652B1ED100957D
:10725000002501AA65216846FCF7E0FF019B00219B
:1072600003EB800040F2CA52834215D1F26840F22B
:107270001A439A4237D1236A1F78B7B13B4A314645
:10728000204602B0BDE8F041FDF72EBC622BEDD1E7
:10729000AB680093ED68DCE753F8047B97420CBFC2
:1072A00001310331E0E70021E0E7A36A606A5B6B2C
:1072B0009847A36A606A9B6B05219847A36A606A36
:1072C000D3F8A0303A460121984701AA2946204622
:1072D000FDF700FBA36A606ADB6A0222394602B04E
:1072E000BDE8F0411847A36A606A5B6B984706F1F6
:1072F0000C006A466A21FCF791FF00270646B74258
:10730000D4E9090313D1D3F8A030002231469847BD
:10731000294601AA2046FDF7DDFA0025B542D4E949
:1073200009030DD1DB6D984702B0BDE8F081009AEA
:107330009B6B52F827209168090998470137DEE7CF
:10734000009ADB6A52F82580D8F808703F09394660
:1073500001229847D8F80C1029B939462046FEF783
:107360006BFC0135DAE70909F8E700BFD58D0508A0
:10737000836A37B504460D465B6B406A0021984727
:10738000A36A606A1B6B0F2198472946204601AA11
:10739000FDF7A0FA0199204603B0BDE83040FEF7A2
:1073A0004BBC00002DE9F04F9BB0CDE9020110204D
:1073B0009D4D1446F8F75CFF2B694360582200216D
:1073C000064604A822F090FB4FF0FF33012113A8DA
:1073D00009938DF8104007F06DFA039BD900012244
:1073E00041F0020113A807F09BFA0123436000213A
:1073F00016A80BF01BFC029A95F8043212680021C3
:1074000004A8FDF752FA054611A800F029FF874BA2
:107410000B9F01900D900E934FF0000B0FB1059C48
:107420001CB30B9C14B1059B002B3ED00198DFF8D8
:10743000FC91DFF8FCA1594600F019FF0B9C0027D6
:10744000DDF81480002C00F03981B8F1000F00F055
:10745000F1800C9C04A8E168FDF7BAFAA38A069AA9
:107460000399404609F0B6FE2CE13B8B042B4FF00C
:107470000102394604A807D1FEF7A8FA079BBF68A6
:107480009B4538BF9B46C9E7FFF7F2F83B8D9C420E
:10749000F4D2FB6A03EBC40113F83430012B02D1A0
:1074A0003846FDF71BF90134F0E7E28A520716D59A
:1074B000218D013913D3E76A07EBC1024FEAC10EF0
:1074C000507810F0020F25D04BB1D3E9008C92E830
:1074D000030083E8030047F80E80C2F804C04FF0B1
:1074E000000323840027B4F828C0674518DB002375
:1074F0009C454ED1D4F804E0BEF1000F08D0002026
:10750000BEF828A00346504553DB002B40F08A808C
:10751000A46887E7002BCCD1012808BF1346C8E731
:107520002378D4F82C80012B4FEAC70A08EBC7094F
:1075300005D1D9F804300A2B12D10137D3E718F856
:1075400037300DD9012B0BD14FF0030308F837303A
:10755000238B032B16D0E38A43F01003E38203E06E
:1075600018F80A30032BF3D018F80A30042B03D094
:1075700099F80130DB07E0D5238C5A1C2284A9F846
:107580000230DAE7D9F8040007F010F80128EBDC44
:10759000E1E7E26A02EBC30112F83320052A06D1C3
:1075A0004A78D7075FBF228C4A8001322284013398
:1075B0009EE7DEF82C2002EBC00912F83020053AD5
:1075C000012A14D8002710E0E26A02EBC70812F87B
:1075D0003720062A08D1D9F80410D8F8042091429F
:1075E00004BFA8F8023001330137BC45ECD10130AB
:1075F00089E7E06A00EBC20110F83200062802D1E8
:107600004878C00702D5488818444880013294451C
:10761000EFD1628B12FA83F26283228C12FA83F327
:10762000238475E70022F2E770040020A4DB05083C
:10763000A8DC0508238B042B17D10F9B1BB95846D8
:1076400004F042FC0F9000230D9303224A4B109349
:10765000214604A8FEF7BAF9059B23B90422214666
:1076600004A8FEF7B3F9A468EAE6023B012B21D88F
:1076700037B95B4607AA05A911A803F07DFD0746A7
:10768000CDE90D7A0222214604A8FEF7F1FF059B01
:10769000002BE8D10322214604A8FEF7E9FF059B51
:1076A000002BE0D10422214604A8FEF7E1FF0028C8
:1076B000F8D0D8E7019BCDE90D39E3E7B8F1000F29
:1076C0007FF4C7AEDDF81490D5F81080B9F1000F43
:1076D00016D0019800F0D3FD002F41D10F9808B1CA
:1076E00004F007FC0298FCF787FF2846AD68FCF71A
:1076F000B3FF002DF9D10598002835D0F8F790FD9B
:10770000139C1898C4F3DC046400033400EB940069
:107710008000F8F7ADFD24F003040444F460DDE9D3
:107720001441B06001F1040CA1450BD1189A00235B
:107730009342CED0199951F82300F16841F8230003
:107740000133F5E751F839303BB1042B1FBF5CF82A
:1077500039205210DB0820F8123009F10109E3E763
:10776000384603F02BFDB9E72A46314640461BB0A8
:10777000BDE8F04F05F00CB984DD0508F0B52DED3E
:10778000028B884283B007460C4604D1012003B027
:10779000BDEC028BF0BD244B984201D10020F6E7EE
:1077A0009942FBD007F0ECFA0546204607F0E8FACC
:1077B0008542F3D11D4B9D4213D17A6863689A428A
:1077C000ECD13E1D043400257B68AB42DED954F871
:1077D000041F56F8040FFFF7D1FF0028DED0013553
:1077E000F2E72146384607F08DFD0028D6D0104B31
:1077F0009D42CBD1384609F049FEB5EE400AF1EE84
:1078000010FAB0EE408AC1D1204609F03FFE8DED5E
:10781000010A18EE100A019B00F0004003F000433B
:10782000C31A58425841B2E7C0DE050844F60508BD
:10783000B4E80508C90010B50122044641F0020170
:10784000083007F06DF843683BB9A368C3F3DC0365
:10785000013B5B0043F001034360C3F34F0010BDE5
:1078600070B505460E460024EB69A34208D83146A0
:1078700005F114000BF097F8EC69013C204670BD4F
:107880002B6A314653F82400FFF778FF0028F5D122
:107890000134E9E710B501220446FCF7F7FE03784E
:1078A000012B05D12378012B8CBF04230223037005
:1078B00010BD70B505460E46104619461C46FCF72D
:1078C000D5FE03785A1E012A06D873680022214685
:1078D0002846BDE870401847032B02D17368012287
:1078E000F5E736684288042B21462846B44608BF8F
:1078F0000023BDE8704018BF012360474379012B86
:1079000007D083681944036981605A8C9142C8BFCB
:1079100059847047002383714379012B1EBF036A8A
:10792000C26A43F8212070476FF00301FFF7E6BFFA
:107930000421FFF7E3BF6FF00201FFF7DFBF426AE8
:1079400003464079032888BF586B114494BF1846FA
:10795000801859627047827903460AB11846704709
:10796000C26A40790328114401D8D962F6E7986ABF
:10797000D9620244586B1044704710B50C4601217F
:10798000FFF7E9FF047010BD10B51446FFF7B6FF0E
:107990000121FFF7E0FF047010BD53220121FFF722
:1079A000F3BF54220121FFF7EFBF57220121FFF758
:1079B000EBBF58220221FFF7E7BF59224FF0FF31FA
:1079C000FFF7E2BF5A220021FFF7DEBF5B22002152
:1079D000FFF7DABF5D224FF0FF31FFF7D5BF19B1D6
:1079E00003215F22FFF7D0BF5E22FBE7A1F1300247
:1079F000D2B20021FFF7C8BF62226FF00101FFF78A
:107A0000C3BF10B5632204464FF0FF31FFF7BCFF40
:107A10000123A37110BD10B501F164020446D2B276
:107A20004942FFF7B1FF0123A37110BD10B501F169
:107A300067020446D2B24942FFF7A6FF2269D38A01
:107A400043F00103D38210BD38B504461D46FFF74D
:107A50009BFF2A4620460249BDE8384013F0A6BDE8
:107A60005779020870B504460D46C0681946164697
:107A7000FFF7E0FE3246034629462046BDE8704047
:107A8000FFF7E2BF0B4610220121FFF7EBBF1132D7
:107A90000B46D2B20121FFF7E5BF20B40B4602F13D
:107AA00014055100C1F10101EAB25DF8045BFFF772
:107AB000D9BF16320B46D2B24FF0FF31FFF7D2BF1B
:107AC00019320B46D2B20021FFF7CCBF70B4C468A4
:107AD0002678042E1D4608BF6668638808BF46F8EE
:107AE00023505D1C658070BCFFF7AEBF03F1280119
:107AF0001346CAB20021FFF7A7BF022A02F12A02E9
:107B00000B46D2B214BFC1F101010121FFF79CBFA6
:107B100003290AD004290AD101210B460A4443EA69
:107B20008203C9432F22FFF78FBF0021F5E7002111
:107B30000223F3E70B4630220139FFF785BF10B46B
:107B4000144641EA0223214431225DF8044BFFF739
:107B50007BBFF8B516461F46FFF7D0FE8479054671
:107B600004BB4379022B25D9C46A036AC4F1FF24FC
:107B700053F8273004F57F04FE34442E1C4412D8F9
:107B800014F1400F14DB3F2CD4BF00270127E41B66
:107B9000B91C2846FFF7DFFE06706FB9442E98BF68
:107BA00040344470F8BD7F2C94BF00270127EEE7D6
:107BB0000127ECE70127EBE76B79442E98BF04F52A
:107BC0008044042B05D1B4F5004F24BF012385F870
:107BD000383064F07F03E41143708470E2E710B53D
:107BE0000B46044642220021FFF7B3FF0123A37195
:107BF00010BDF8B505460C4621F400471646CAB933
:107C00000B040ED55921FFF7B8FE59212846FFF77E
:107C1000B4FE59212846FFF7B0FE59212846FFF748
:107C2000ACFE3B46422200212846FFF792FF01238B
:107C3000AB71F8BD3B4640220021FFF78AFF210AC5
:107C400021F07F013143C9B22846FFF796FEEEE7E7
:107C50000B46B2FA82F120B4490902F14705EAB2B3
:107C600049005DF8045BFFF774BF0B464B2201210E
:107C7000FFF76FBF10B50B4604464A220021FFF7FD
:107C800068FF0123A37110BD264BD3F80032022BED
:107C90002DE9F047044689460ED88669B1420BD9D2
:107CA000C56A43698E1BED1A40F2FF7756EA050359
:107CB00004D1E36AC4E90539BDE8F087062E01D98D
:107CC0000F2D1AD91F2DAA4628BF4FF01F0A1F2DAE
:107CD00010D8032EB04628BF4FF0030801212046DC
:107CE000FFF72DFE4AEA48130370A5EB0A05A6EB41
:107CF0000806DBE74FF00008F0E7BE42B0464FF061
:107D0000020128BFB8462046FFF719FE4FEA1813B4
:107D100003F070032B4363F07F03037080F801804E
:107D2000AA46E2E77004002010B5044631B9552296
:107D30004FF0FF31BDE81040FFF726BE022904D105
:107D4000FFF72BFE2046FFF741FE56226FF002019F
:107D50002046EFE7134621B143224FF0FF31FFF7F2
:107D6000F8BE4422F9E7134621B145224FF0FF3116
:107D7000FFF7EFBE4622F9E7322938B5044611D0A5
:107D8000332912D000252939CAB220464FF0FF31DD
:107D9000FFF7FAFD65B12046D322BDE83840002147
:107DA000FFF7F2BD01250621EDE701250721EAE7EE
:107DB00038BD012A10B40B46044608D0022A0ED161
:107DC0005DF8044B69224FF0FF31FFF7DDBD11462E
:107DD0001B322046D2B25DF8044BFFF743BE4FF092
:107DE000FF31F5E770B50D46044611462AB92B461A
:107DF0001322BDE87040FFF735BE022A04D1FFF719
:107E0000CCFD2046FFF7DEFD2B4618226FF0010166
:107E10002046EEE710B4044643B90F2A06D8503A7C
:107E20005DF8044BD2B20121FFF7AEBD03F124018E
:107E3000204613465DF8044BCAB20121FFF704BE89
:107E400010B404464BB90F2A07D8403A5DF8044BEA
:107E5000D2B24FF0FF31FFF797BD03F12601204664
:107E600013465DF8044BCAB24FF0FF31FFF7ECBD8B
:107E700070B4DDE90365D2B203EB460443EA06239E
:107E800015B101320134D2B2091B70BCFFF7DCBD61
:107E900007B5CDE900230B4634220021FFF7E8FFA8
:107EA00003B05DF804FB07B5CDE900230B4636228D
:107EB0004FF0FF31FFF7DCFF03B05DF804FB10B5B6
:107EC0000446C068FFF7CCFC23220346012120466C
:107ED000BDE81040FFF7B8BD01F110033F2B73B5AB
:107EE00006460C4608D8A1F18002D2B2012102B0A8
:107EF000BDE87040FFF748BD012122220DF10505C4
:107F0000FFF742FD294604F07F00E3B2E4112A4660
:107F100005F8010D601C0128F5D8013403F0400379
:107F200014D11BB97F2305F8013C951E491B30462F
:107F3000FFF711FD01AC6A1E014612F8013FA24293
:107F400008D11044401B037002B070BD002BEDD06F
:107F50000023E8E763F07F0301F8013BEDE770B52C
:107F60001446D6B2049A134305460B6907BF202274
:107F7000C4F10101E1432122FFF7A8FD3146284663
:107F8000BDE87040FFF7F9BC1A4308BF32220B6905
:107F900016BF332201214FF0FF31FFF797BD0000DC
:107FA0000D2910B504460BD10949C068FFF758FCEC
:107FB0002322034601212046BDE81040FFF744BDBF
:107FC0004231CAB2BDE810400121FFF7DDBC00BF5D
:107FD000D4F1050838B504460D460F21FFF7E0FF40
:107FE00020462946FFF796FC02215C22FFF7CCFCD5
:107FF00020466FF00301BDE83840FFF77FBCF8B5BD
:1080000004460F460F211D461646FFF7C9FF2046BE
:10801000FFF7D8FC39462046FFF7E1FD3146204600
:10802000FFF778FCFFF7C1FC012220462121FFF772
:108030002EFD20460821FFF79FFE2A4620460021FC
:10804000BDE8F840FFF786BE4379012B70B50446C2
:1080500014D0C26B436A00259B1AC3630564206970
:10806000038DAB420CD86379032B1BD1606AE36AA2
:10807000A06223631844F8F714F96063012070BD0F
:10808000C36A03EBC50213F83530052B08D1012173
:1080900020469678FFF753FC0670236C0133236467
:1080A0000135DCE7042BE9D1D4E90A13626A8A427C
:1080B00002D1216B994203D0A26223630020DEE744
:1080C00094F838301BB10649064805F0A1F8E2687B
:1080D000C38A5268616B006904F03FFCCEE700BFC1
:1080E000E78D0508A8E505082DE9F74F164600239A
:1080F000C0E90423378C83608371C362436280F8D4
:108100003830738CB6F82490B6F81A80B6F816A0FA
:10811000B6F81EB0417101221F449742B8BF1746FE
:108120004FEA8905013F826105F0040508F003026A
:108130001543FA0002F07802B38B04460AF00F0AE6
:1081400015433F094FEA59094FEA980847EA0902DF
:1081500042EA0A0242EA08021A4352EA0B0234D106
:1081600001212046FFF7EBFB05706379022B18D93C
:10817000D4E90F787D0008F0010305F07E054FEA91
:108180005808BF091D4358EA07094FF0010120466E
:1081900018BF45F08005FFF7D2FB0570B9F1000F5D
:1081A000E8D1636AB18AE363E068FFF743FB2B49D8
:1081B0000246204613F0FAF90025738BB28B134464
:1081C000AB4248DD318D002241E001212046019380
:1081D000FFF7B5FB65F07F053A0105704FEA8A1598
:1081E000019B02F0300205F0400515430BF001023F
:1081F0001543DA0002F0080215434FEA880202F044
:10820000040215434FEA490202F002021543BF0877
:108210004FEA59094FEA5A0A4FEA58085B084FEAF1
:108220005B0B93E7F36A03EBC2035878C0070DD5E5
:108230005888A8420AD15968E068FFF7FBFA074955
:108240000246204613F0B2F90135B6E701329142F9
:10825000E8DC0521F0E703B0BDE8F08F3F790208C4
:1082600010B504464420F8F71CF8C46010BD10B5E2
:108270000446C1618800F7F7FBFF206210BD10B50E
:108280000446006AF8F71CF82046BDE81040F8F7ED
:1082900017B810B5044601618800F7F7E9FF60617F
:1082A00010BD10B5044611B1C068F8F709F860694F
:1082B000BDE81040F8F704B8012938B504460D466A
:1082C0000BDC0269406992004FF0FF3121F00CFC99
:1082D000002325706370636038BD4068F7F7C8FFFE
:1082E0006368E060A360F3E70246407810B548B9E0
:1082F00013785468022B08BFD368214408BF1819AB
:10830000516010BD0020FCE7002343700378012B6F
:108310009EBF4369426843F82120704742684B1E64
:10832000134449420B404360704738B50C4615462C
:10833000FFF7DAFF10B10444A04200D138BD00F8C5
:10834000015B2D0AF8E710B50C460221FFF7CCFFC0
:1083500010B10470240A447010BD38B50D460421D4
:108360001446FFF7C1FF28B1057084702D0A240A56
:108370004570C47038BD012970B5054606DC00297A
:1083800009DA023921F00104FE2606E08B1E012BDA
:10839000F7D80024F8E70024F22646F435412846B1
:1083A000FFF7D1FF44B17F2C09D844F4304141F0AC
:1083B00080012846FFF7C7FFC5E9066470BDA3002A
:1083C000A201DBB202F4E0421A4342F450624FF2DF
:1083D000AD212846FFF7C1FFEEE7C16910B504469D
:1083E00029B17F290BD841F43041FFF7ACFFA169D7
:1083F000204641F43D41BDE81040FFF7A4BF8B008B
:108400008A01DBB202F4E0421A4342F450624FF2B6
:108410000D21FFF7A2FFEAE7114341EAC301FFF78D
:1084200092BF072A85BF083AD200D20042F040022C
:10843000072985BF08391143114341F0800141F4F8
:108440008C41FFF780BF30B4DCB244EA02225C10FA
:108450001D0104F48064C3F3033305F4E0452343B2
:108460002A43194330BCFFF778BF38B5436953F846
:1084700021404368E41A043C0546C4F34A0141F430
:108480006041FFF760FF2B78022B0AD1B4F5006F33
:1084900007D36FF30A0414F5006F14BF0020012006
:1084A00038BD0120FCE7F8B5446954F82240426821
:1084B000A41A043C074665101E46BBB9EDB245EA56
:1084C000012141F45041FFF73EFF3B78022B0BD1D5
:1084D000FF2C09D924F0FF0414F5807F14BF002479
:1084E000012426463046F8BD0124FAE76211C5F39F
:1084F0000A0502F400522A43A512231205F48065EE
:10850000C4F3053403F4006325431A4345EA81119B
:1085100042F4004241F47041FFF71FFFE2E738B533
:10852000436953F821404368E41A043C0546C4F308
:108530004F02C4F30A3142F4784241F47041FFF72C
:108540000CFF2B78022B0AD1B4F5800F07D36FF301
:10855000150414F5800F14BF0020012038BD012040
:10856000FCE7F8B5476804460D46164613460A462A
:108570004FF24021FFF767FF2046330C2A464FF2A7
:10858000C021FFF760FF3846F8BD072910B4044644
:1085900009D8FF2A07D842EA01215DF8044B41F4CB
:1085A0000051FFF7D0BEB2F5803F08D213462046F7
:1085B0000A465DF8044B4FF24021FFF744BF2046C6
:1085C0005DF8044BFFF7CDBF2DE9F84341EA020700
:1085D000072FDDF8209006460C4615464AD803FAC8
:1085E00009F7FF2F0CD8914201D0FFF71AFF47EA95
:1085F000042141F440513046BDE8F843FFF7A3BEE3
:10860000FF2B4FEAC10814D8914218D043EA012346
:1086100043F40051FFF797FE44EA891141EA08014B
:108620003046FFF790FE48EA8511214341F4C051DE
:10863000E1E7914203D03A46FFF7A7FFF3E784F062
:108640000709012505FA09F545F434413046FFF7DD
:108650007AFE3A4649463046FFF797FF44EA8911C9
:1086600041EA080141F4C0513046FFF76CFE45F481
:108670003C41C0E7BDE8F88308B50378012B04D975
:10868000FF2902D9054805F0A5FDC9B241EA02213A
:10869000BDE8084041F41041FFF755BEF28D0508D2
:1086A00008B50378012B04D9FF2A02D9054805F043
:1086B00091FDD2B242EA0121BDE8084041F41841DF
:1086C000FFF741BEF28D0508D2B242EA012141F422
:1086D0002841FFF738BE38B5436953F82230426865
:1086E0009B1A43F001030C4605460A460A3B4FF22B
:1086F0004021FFF7A8FE2346284622464FF4324188
:10870000FFF78AFE210101F0800104F007042143F4
:1087100041F48841284641F07801BDE83840FFF730
:1087200012BE000073B51F2B069E05460C4611D8DD
:10873000114307290ED81A49895D44EAC20241F063
:10874000010142EAC12141EA831102B0BDE8704053
:10875000FFF7F9BD03FA06F1B1F5805F0DD242EAE9
:10876000461641EA043246F4784141F09001284629
:1087700002B0BDE87040FFF7F0BD1F3B2146284620
:108780000096FFF721FF064B9B5DE10043F00103DC
:1087900041EAC321214341F4F8612846D5E700BFEF
:1087A0007CDC05082DE9F7431F2B0A9F06460C4683
:1087B0001546984610D841EA0203072B0CD8204BE7
:1087C000D95D44EAC12141EAC20141EA881103B0FE
:1087D000BDE8F043FFF7B7BD08FA07F2B2F5805FD6
:1087E0000DD245EA471141F4784142EA043241F0A2
:1087F0008001304603B0BDE8F043FFF7AEBD4FF057
:10880000010909FA05F949F434413046FFF79BFDA7
:10881000A8F11F032A46294630460097FFF7D4FEE9
:10882000074BDB5D44EAC50141EAC32141F4F8612D
:108830003046FFF788FD49F43C413046C7E700BFAA
:108840007CDC0508436953F821104368CB1A043BCC
:10885000013110B4C3F34A0204460ED0D91C0CDA1D
:1088600023F4FF6121F0070111F5006F05D15DF8D8
:10887000044B42F46041FFF766BDC3F30A33204660
:1088800042F438425DF8044B43F47041FFF765BD94
:10889000436953F822204368D31A043B013230B4B1
:1088A00005464FEA63040ED0DA1C0CDA23F0FF020F
:1088B00012F5807F07D1E4B244EA012141F450412E
:1088C00030BCFFF740BD5A11C4F30A0402F4005251
:1088D00022439C12181204F48064C3F3053300F49D
:1088E00000602343024343EA8111284642F40042D8
:1088F00030BC41F47041FFF730BD37B51446022259
:108900000B460092214607220546FFF70BFFE100C8
:1089100041F48F41284603B0BDE83040FFF713BD56
:1089200007289ABF024B33F8100040F20720704727
:1089300080DC0508C36C19440369C164012B04DDA4
:10894000436D5A8C9142C8BF5984704770474FF0AD
:10895000FF31FFF7EFBFFFF7FABF6FF00301FFF73B
:10896000E9BF704738B5C36C1944036A994205469C
:1089700008D9083121F00304406AE100F7F793FCBD
:10898000C5E9084038BD70B504460E4601211546BC
:10899000FFF7E8FFE16C626A02EBC10302F83160A5
:1089A000012159705D602046BDE87040FFF7C2BFED
:1089B00070B504460E4601211546FFF7D3FFE16C62
:1089C000626A02EBC10302F8316002225A705D60F4
:1089D00020460121BDE87040FFF7ACBF00221146E0
:1089E000FFF7E6BF0A460221FFF7E2BF70B50D1E92
:1089F000044605DDFFF7B6FF00231E46AB4205DB4C
:108A000029462046BDE87040FFF794BFE26C616ADA
:108A10001A4401EBC200012D46700CBF94F82800E7
:108A2000002001F832000133E8E7F8B5D0E90B5334
:108A30000133AB4204460E46174606D90435406B57
:108A4000A900F7F730FCE5626063D4E90C30C6F3A7
:108A50000E015A1C226300EB830541EAC73220F85D
:108A600023204FF6FF73A06D6B8032460021FFF785
:108A700032FEA06D0022BDE8F8400321FFF7FCBDE7
:108A80000246007D28B1D36C526A5B1A013B12F892
:108A90003300704737B5456DED8AED070B46144638
:108AA00008D502220092806D06222146FFF77AFE49
:108AB00003B030BD806D03B0BDE83040FFF7DCBDD2
:108AC00070B5002405462646EB6CA34200DC70BD61
:108AD0006B6A03EBC4035A78012A07D15E70B5F8BC
:108AE0004A105A6821442846FFF7D4FF0134EBE7C7
:108AF000F8B504461E4617460D46FFF7E1FFA06D88
:108B00003A463146FFF741FDA06D29460322BDE8F4
:108B1000F840FFF7F2BE38B504460D46FFF7D0FF28
:108B2000A06D29460322BDE83840FFF7E6BE10B528
:108B300008210446FFF7EFFF002220461146BDE85A
:108B40001040FFF720BFF8B5044617461E460D46F5
:108B5000FFF7B6FFA06D3A460021FFF716FDA06DA6
:108B600032460121FFF711FDA06D29460322BDE821
:108B7000F840FFF7C2BEF8B5C76C04460E46BF1AF0
:108B80000025E36CAB4200DCF8BDBD4211D0636A46
:108B900003EBC5035A78012A0BD15A68B24208D1B7
:108BA00000225A70B4F84A10324629442046FFF792
:108BB00071FF0135E5E738B5002205460C46114640
:108BC000FFF7D9FFE200A86D42F002020021FFF793
:108BD000DCFC002228461146BDE83840FFF7D3BE32
:108BE00013B5446DE48AE407134607D502220092C8
:108BF000806D0622FFF796FD02B010BD806D02B0B9
:108C0000BDE81040FFF74CBDF8B5C3699E5C602E0F
:108C10000446154606D1476813480A46134908F02A
:108C20008DFA3860022D0DD8636D9A8C52B9DB8AAB
:108C3000DB0707D40E4B5A5D31462046BDE8F840AD
:108C4000FFF7A1BE002211462046FFF794FFB4F8BB
:108C50004A20636C1A44521B013A00212046FFF758
:108C6000BFFF0022E8E700BFF4E40508088E05080E
:108C700080DD050873B503681A785D88042A04BF8F
:108C80005A6842F825106A1C044602265A800021C0
:108C9000B0F84820FFF7A4FF00960022A06D3346ED
:108CA0001146FFF73FFD00960022A06D2B461146AE
:108CB000FFF738FD02B070BD73B5002204460D46C3
:108CC0001146FFF758FF626D2068D38A43F02003F6
:108CD000D3822946FEF7C4FD0226B4F84820054693
:108CE00000212046FFF77CFF00960022A06D114670
:108CF0000123FFF717FD00960022A06D1146032304
:108D0000FFF710FD00960022A06D11462B46FFF7DD
:108D100009FD00221146204602B0BDE87040FFF771
:108D200032BE00000D2902D10749FFF7C5BF0F2948
:108D300003D100225421FFF73BBEB1F10E0218BF50
:108D400001220121F7E700BFD4F10508F8B5C76C8F
:108D5000446A07F10053023B04EBC3040546D4E91F
:108D6000020184E80300667856B9B5F84A203A440F
:108D7000013A31462846FFF733FF012363706660EE
:108D800028464FF0FF31BDE8F840FFF7D3BDF8B5F6
:108D900004461E4617460D46FFF792FEA06D3A4662
:108DA0003146FFF7F2FBA06D29460322BDE8F840EB
:108DB000FFF7A3BD10B402F1290400230A46E1B273
:108DC0005DF8044BFFF7E3BF70B504460E46154649
:108DD00062B1037D53B1084605F0E8FB021E05DDD4
:108DE00020467021BDE87040FFF7E2BD06353246EF
:108DF000E9B220460023FFF7CAFF002220461146B1
:108E0000BDE87040FFF7BFBD07B5134602220092D0
:108E10000722FFF787FC03B05DF804FB38B50D4669
:108E200014463BB9037D2BB1806D5268FFF7ADFB53
:108E3000207838BD237833B96268806D2946FFF702
:108E4000A4FB0020F5E7012B06D162680132806D9A
:108E50002946FFF7D9FFF4E79A1E012A04D8626871
:108E6000520042F00102E8E7542B01D10022EEE764
:108E7000014805F0AFF900BF1D8E0508F8B505469D
:108E8000FFF71EFE00242746EB6CA34200DCF8BD72
:108E90006E6A06EBC4025378022B0ED15770012183
:108EA00000232846FFF7BAFF06F83400B5F84A1049
:108EB000012221442846FFF7EDFD0134E4E738B5EF
:108EC00004460D46FFF7DAFFA06D2946FFF7BAFC0E
:108ED000A36D01225A7038BDF8B504460E461746F8
:108EE0000A4619461D46FFF746FEE36C616A9B1B66
:108EF00001EBC30211F833303B705378012B0DD0D6
:108F0000022B14D0CBB9B4F84A20E36C1A44921B5C
:108F100029462046BDE8F840FFF762BE5268AA42E3
:108F20000BD0A06D2946BDE8F840FFF77ABA0023C0
:108F300029462046FFF772FF3870F8BD10B513467A
:108F400004460A460121FFF7C7FF20464FF0FF31D4
:108F5000BDE81040FFF7EEBC70B5049E04461D4608
:108F6000FFF7ECFF324629462046BDE87040FFF788
:108F7000E5BFF0B585B001250DF10F030DF10E0130
:108F8000009500220446FFF7E7FF9DF80F709DF85B
:108F90000E602A4639462046FFF7F5FC314620464A
:108FA0000022FFF7F0FC2A4639462046FFF7EBFC8B
:108FB00000223146204605B0BDE8F040FFF7E3BC93
:108FC0002DE9F041DDE9068604461D46089FFFF7BE
:108FD000B5FF424629462046FFF7B0FF3A463146E4
:108FE0002046BDE8F041FFF7A9BF2DE9F04186B06A
:108FF00002260DF11703012501930DF115010DF165
:1090000016030296009500220446FFF7D9FF9DF84B
:1090100017809DF815109DF8167020460022FFF766
:10902000B2FC324641462046FFF7ADFC2A4639469F
:10903000204606B0BDE8F041FFF7A5BC30B587B0CB
:109040000DF117030025019302230446009301222A
:109050000DF116030DF115010295FFF7B1FF204642
:109060001921FFF758FD2A462946204607B0BDE8DA
:109070003040FFF788BC73B504460E46154672B9FA
:1090800001220DF10701FFF759FF0C35002332468D
:10909000E9B2204602B0BDE87040FFF778BE00217B
:1090A000FFF7EEFC20B901220DF107012046EAE7A7
:1090B0000A4620460DF10701FFF740FF9DF8072003
:1090C000204601230421FFF713FDA06D002201219A
:1090D000FFF7A7F9D9E7000037B500220DF1070126
:1090E0000446FFF72BFF9DF807302BB107490848CE
:1090F000656808F023F8286022212046FFF70BFD61
:10910000A36D01225A7003B030BD00BF228E050846
:10911000F4E40508022A7FB504460E46154614D825
:10912000436D9A8C8AB9DB8ADB070ED4184B0DF19C
:109130000F015A5DFFF702FFE3699DF80F10585DBC
:10914000602813D1595504B070BD0DF10F012046B0
:109150000022FFF7F3FE626CB4F84A3013445B1B45
:109160000022591E2046FFF795FCE5E78842EAD029
:10917000FFF7D6FB02460846FFF7D2FB05496468B5
:10918000009013460448324607F0D8FF2060DAE723
:1091900080DD05082C8E0508F4E4050870B504464A
:1091A0000D4616464BB90F21FFF7BCFD3246294646
:1091B0002046BDE87040FFF7ADBF70BD03297FB505
:1091C0000446164613D101220DF10F01FFF7B6FE3A
:1091D00018253146204600230DF10F02FFF77CFED3
:1091E0002946204604B0BDE87040FFF794BC05292D
:1091F00006D101220DF10F01FFF7A0FE1725E8E7C8
:109200000223009301220DF10F030DF10E01FFF770
:10921000A3FE1925DDE7F0B5044685B00E461546D8
:10922000CAB90223077D02750DF10E0100930122D8
:109230000DF10F03FFF790FE27752B4632462321D1
:109240002046FFF7A4FD00221146204605B0BDE8E8
:10925000F040FFF798BB012A09D100230DF10F025E
:109260002946FFF739FE2B4632462421E8E70DF167
:109270000F010022FFF762FE2521204605B0BDE860
:10928000F040FFF748BC10B50446D0E90C3003F1BC
:109290008043013B00EB8303DA7822F08002DA702E
:1092A000043B98420BD893F90320002AF8DA1A8875
:1092B000A06DC2F30E020021FFF70DFA05E059B9C7
:1092C000A06D4FF40051FFF73EF8A06D0022BDE8FD
:1092D00010400321FFF7D0B910BD10B5044601219D
:1092E000FFF7D1FFA06D01220021FFF7D9F900227D
:1092F00020461146BDE81040FFF745BB73B5046B2F
:1093000005460E46DCB1436B04F18044013C03EB9F
:10931000840292F90120002A20DA33F82430C3F3C2
:109320000E038B421AD100230DF107020121FFF732
:10933000D3FDA86D00220121FFF79EF901242846E4
:10934000FFF79CFDA86D3146FEF7DEFF44B100211A
:10935000284602B0BDE87040FFF795BF0024EEE755
:1093600002B070BD38B50D46044611467AB1806D25
:109370004FF40051FEF7E7FFA06D00220121FFF737
:109380007BF929462046BDE83840FFF798BDFFF736
:109390007AFFF6E72DE9F04104460D4672B3D0E9B5
:1093A0000C3C03F18043013B0CEB83030021184686
:1093B00016460F4690F901E0BEF1000F09DA90F968
:1093C00003E0BEF1000F04DA002F08BF0746E1B941
:1093D0000146013EA0F10400ECD1A06D21BB6FF06D
:1093E000030672439E18B44518D94FF40051FEF796
:1093F000AAFFA06D00220321FFF73EF925F40041EA
:109400002046BDE8F041FFF75ABDB0F80080B1F842
:1094100002E068F30E0EA1F802E0D9E79A5AC2F30F
:109420000E02FFF758F9E4E74B8847F6FE7262F345
:109430000E034B8025F400423146FFF74CF9A06D36
:1094400032461321FFF718F9A06D32463146FFF777
:109450009CF8A06D32460121FFF70EF93D88C5F357
:109460000E05CBE77FB504460E4615468AB90DF1C9
:109470000F01FFF763FD3246204601230921FFF764
:1094800086FC2A462946204604B0BDE87040FFF716
:109490007ABA012A35D11146FFF7F2FA024688B9A5
:1094A000022300930DF10E010DF10F032046FFF78B
:1094B00053FD012332460E21204604B0BDE8704022
:1094C000FFF765BC0DF10F02204600230221FFF7D4
:1094D00003FD2B469DF80F2020460421FFF708FBD3
:1094E000A06D00220221FEF79CFF0DF10E01204627
:1094F0000022FFF723FD4FF0FF312046FFF71AFA55
:10950000D7E70DF10F010022FFF718FDA06D4FF412
:109510000851FEF718FFCCE738B5FFF718FA0446F4
:109520000122806D0021FFF7BBF822212046FFF7C2
:10953000F2FAD4E90C35013B05EB830523636B8814
:1095400047F6FF72C3F30E03934228D01322A06D97
:109550000021FFF7A5F8A06D4FF42051FEF7F3FEB0
:10956000A368A06D1A680021FFF792F9698847F691
:10957000FE73C1F30E029A420BD1A06D4FF48E41DF
:10958000FEF7E1FEA36820461968BDE83840FFF702
:10959000B5BEC1F30E012046FFF791FCF2E738BDDE
:1095A0002DE9F3410E460021174604461D46FFF7FC
:1095B00067FA024648BB0DF107012046FFF7BEFCE3
:1095C0001DB901212046FFF7B5F910212046FFF70C
:1095D000A2FA1DB99DF8073084F828302046FFF71D
:1095E0004DFCA06D4FF420515EB3FEF7ACFE3A4641
:1095F0000121A06DFFF74CF945BB4FF0FF3120462C
:1096000002B0BDE8F041FFF795B90A4620460DF1DA
:109610000701FFF793FC1DB901212046FFF78AF9E6
:109620009DF80700431E022BD3D9FFF779F90949AA
:10963000D4F804800246084807F080FDC8F800000E
:10964000C7E7FEF780FE3A463146D2E702B0BDE8F2
:10965000F08100BF3C8E0508F4E405080023FFF705
:109660009FBF0123FFF79CBF426D83682DE9F34143
:10967000D58A928C1E68C66005F011031343044618
:1096800000F0F98015F0010506F1020721D1B0F8CC
:10969000482029464FF00208FFF7A2FACDF80080D3
:1096A000A06D01232A462946FFF73CF8CDF800803B
:1096B0002A46A06D01232946FFF734F805212046EC
:1096C000FFF729FAB4F848102A4601312046FFF77F
:1096D000E1F9D4E915309A8C002A67D1D98A11F0C2
:1096E000010508D14FF42051FEF72DFEA06D3A463A
:1096F0002946FFF7CDF800221146A06DFEF7E4FFE2
:1097000020212046FFF707FA4FF42051A06DFEF705
:109710001AFE3A460021A06DFFF7BAF8636DD98AA8
:1097200011F0010100F08E80A06D012200210225C0
:10973000FEF7B6FF0095A06D052306220021FFF776
:1097400031F8A06D2A460021FEF71FFFA06DFEF73D
:1097500044FE39462046FFF7D1FD636DDB8ADB0707
:1097600040F18980B4F84820204601320021FFF7FB
:1097700037FAA06D4FF48E41FEF7E5FDA06D43680A
:10978000236414220021FEF78BFFA06D4FF40451D7
:10979000FEF7D9FDA06D01221421FEF76DFF2221F5
:1097A000204602B0BDE8F041FFF7B5B94FF40051D3
:1097B000FEF7C9FDA06D00221321FEF75DFFA06D2D
:1097C00000220121FEF758FF751C3A46A06D0421C6
:1097D000FEF781FF29462046FFF790FD0022114643
:1097E000A06DFEF771FF20212046FFF794F90336A4
:1097F000A06D4FF42051FEF7A6FD3246A06D012169
:10980000FFF746F8A06D4FF40051FEF79CFD0022D3
:10981000A06D0321FEF730FFA06D44F22071FEF72A
:1098200092FD31462046FFF769FD0322A06D042119
:10983000FEF736FF4FF43051A06DFEF784FD2A4647
:10984000012168E7B4F8482020460132FFF7C8F943
:1098500005212046FFF75FF9D4E91530D98A11F0C8
:1098600001017FF461AF0122FEF71AFF2221204699
:10987000FFF751F96DE702B0BDE8F08170B505461C
:10988000D0E91560F68AF6070C460BD544EAC40405
:109890009200FEF77AFEA86D44F4CC51BDE870400A
:1098A000FEF751BDBDE87040FEF70EBF2DE9F84F41
:1098B00004460F469146FFF703F90025A8464D459B
:1098C00010D10026B3464E452BD171422046FFF7FA
:1098D00031F8B4F84A20E36C39461A44BDE8F84F31
:1098E000FFF7CCBFE66CD4F824A0013E761B0AEB50
:1098F000C6025378022B12D182F801800123394627
:109900002046FFF78BFA0AF83600B4F84A10E36CE9
:10991000194401393A46491B2046FFF7BBF8013587
:10992000CDE7E36CD4F824A003F1FF38A8EB0608D8
:109930001AF83820BAB1B4F84A501D44013DAD1BA5
:109940002A4600212046FFF74BF91AF83820012358
:1099500004212046FFF7CCF8002229462046FFF7D5
:1099600099F80AF838B00136ADE70000037D37B545
:1099700004460D4613B15F4804F02CFC426DD38AB7
:1099800043F00103D382FFF779FA012D0BD1A368CD
:10999000196820460231FFF792FAA3681968204639
:1099A0000131FFF7ABFC012200212046FFF77EFFCB
:1099B000002202212046FFF76DF8A06D0122002150
:1099C000FEF7E3FDA06D00221221FEF755FEA3680D
:1099D000A06D1A680021FEF77EFEB4F84810002240
:1099E00001312046FFF756F8E168A06DFEF72AFF27
:1099F000A368A06D1968FEF787FC236BBBB1626B8F
:109A000003F18043013B02EB83039A420FD893F9A1
:109A10000310002926DA1A88A06DC2F30E02002175
:109A2000FEF759FEA06D00220321FEF725FE01215D
:109A30002046FEF7DBFFBDB9A06D14222946FEF7D4
:109A40002FFEA06D4FF40451FEF77DFCA06D0122A6
:109A50001421FEF711FE2221204603B0BDE830405C
:109A6000FFF759B8043BD0E7A368196820460231D4
:109A7000FFF744FCA06D14220221FEF711FEA06D39
:109A800000220121FEF781FDA06D01221421FEF7C5
:109A9000F3FD0DF1070120460122FFF74FFA0023E5
:109AA0000DF1070220460121FFF716FA2046022297
:109AB0000021FEF768FF012220460221FFF7F6FE93
:109AC00020463021FFF727F8A06D4FF42051FEF714
:109AD0003AFCA368A06D1A6801210132FEF7D8FE96
:109AE00020460121FEF782FF204603B0BDE830404A
:109AF000FFF72CB9498E0508F8B5164604460D4601
:109B0000520093B1CB1C1A440221FFF7CFFE45EA65
:109B1000062301221D212046FFF715F800222046CA
:109B20001146BDE8F840FEF72EBF8B1C1A440221F7
:109B3000FFF7BCFE33462A461C21ECE72DE9F7432C
:109B400004460F4616460121B0F84820DDF828905B
:109B50004FF002081D46FFF743F80123CDF80080BF
:109B6000A06D1A461946FEF7DDFD55EA09052DD10F
:109B70002046FEF7A5FFA06D2A464146FEF705FDEB
:109B800039692046FFF776F8A06D03221A21FEF707
:109B9000B4FEA06D32460121FEF7F7FC32460221E9
:109BA0002046FFF783FE25B16FF001012046FEF746
:109BB000C1FEA06D03222B21FEF79FFE002211465D
:109BC000204603B0BDE8F043FEF7DDBE06F1020912
:109BD0004A4641462046FFF769FE49462046FEF7C1
:109BE000A9FEFEF76DFFCBE72DE9F34104461546CC
:109BF0000F46B0F8482001214FF002081E46FEF73C
:109C0000EFFF0123CDF80080A06D1A461946FEF73C
:109C100089FD354318D12046FEF752FFA06D2A4634
:109C20004146FEF7B2FC39692046FFF723F8A06DE4
:109C300003221A21FEF761FE00221146204602B0DF
:109C4000BDE8F041FEF79FBE204642464146FFF781
:109C50002DFE2046FEF734FFE5E770B5042A86B0F6
:109C600004460E4615462AD102294FF0000518D1A8
:109C700001220DF1170100950DF11603FFF76CF9A4
:109C8000A06D2A463146FFF7BFF826212046FEF791
:109C900042FF00221146204606B0BDE87040FEF7A4
:109CA00072BE0DF1150301930123009302950DF18E
:109CB000160302220DF11701FFF782F9E5E7012AE9
:109CC00001D9032A04D1324601212046FFF7EEFDD7
:109CD000133500233246E9B22046FEF709FFD8E7E4
:109CE00038B5042204460D460021FFF7DFFD20466B
:109CF0000421FEF71FFE1F21FEF70DFFA06D4FF49C
:109D00002051FEF720FBA06D2A460021FEF7C0FD82
:109D1000002220461146BDE83840FEF734BE37B574
:109D200004460D460021FFF7AEFA20464FF0FF3102
:109D3000FEF700FEA36819680231FFF7DFFA20463C
:109D400000225421FEF734FE204600225421FEF763
:109D50002FFE204600225421FEF72AFE204605222F
:109D60000221FFF7A3FD0322204600231C21FEF75A
:109D7000EAFEA36820461968FFF7A1F8A06D2946FE
:109D8000FEF7C2FA20460121FFF77DFA20460221A4
:109D9000FEF72CFEA06D01220021FEF781FCA06DD4
:109DA0004FF42051FEF7CFFAA368A06D1A68022580
:109DB00002320021FEF76CFD002300951A46A06DCB
:109DC0000121FEF7AFFC204601220021FEF7DBFD5A
:109DD000002211462046FEF7D6FD204600225421DF
:109DE000FEF7E6FD294620460522FFF75FFD00232A
:109DF000032220461C21FEF7A6FE20461021FEF776
:109E00008AFEA06D4FF42051FEF79DFAA368A06D65
:109E10001A6800210132FEF73BFDA368204619684D
:109E2000FFF76CFAA06D4FF40051FEF78CFAA06DAD
:109E300000220121FEF720FCA368196820460131A9
:109E4000FFF75CFA0121204603B0BDE83040FEF781
:109E500071BD0000436D73B5DD8A15F0010604463F
:109E600013D001220021FFF721FD0022022120460C
:109E7000FEF710FE0022A06D1146FEF786FBA06DD6
:109E800000221221FEF7F8FB1BE0027D002A47D0DA
:109E90003146FEF7F5FD5428C5F3871525D1204638
:109EA000FEF755FDADB9A06D2A462946FEF7ACFF79
:109EB000636D9A8C002AE2D1DB8A03F01103002B38
:109EC000DDD1226BE168204602B0BDE87040FFF7AB
:109ED00061BAA06D32463146FEF757FB01232A4690
:109EE00004212046FEF704FEE2E70DF107013246A9
:109EF0002046FFF723F89DF80710A9420DD0284609
:109F0000FEF70EFD02460846FEF70AFD07496668A1
:109F10000346074807F012F93060002DC8D0DDE78E
:109F20000DF10701FFF70AF8C2E700BF518E0508DF
:109F3000F4E40508F8B5164604460F46FEF7C0FDE2
:109F400031462046FEF70EFD0025E36C2A46B54259
:109F50000CD1B4F84A20394620461A44FFF78EFC4B
:109F600029462046BDE8F840FEF7E4BC5819616A6E
:109F7000013521F83020EAE773B50D4616460DF19C
:109F8000070100220446FEF7D9FF721C2A4420462E
:109F90000221FFF7CFFF012345EA062228212046B0
:109FA00002B0BDE87040FEF7A3BD37B504460D46CC
:109FB00000220DF10701FEF7C1FF2A4620460221CB
:109FC000FFF7B8FF01232A462721204603B0BDE84A
:109FD0003040FEF78DBD37B50D4600220DF107016B
:109FE0000446FEF7ABFF5DB1204604220121FFF7D6
:109FF000A1FF1E21204603B0BDE83040FEF78BBD17
:10A000002A46A06D0121FEF7C0FA20461E21FEF768
:10A0100082FD2A462946204603B0BDE83040FEF7BF
:10A02000B2BC37B504460D468AB103220121FFF7C1
:10A030003DFC022201212046FFF77CFF00232A4637
:10A040000B21204603B0BDE83040FEF7A0BE0DF165
:10A050000701FEF773FF022211462046FFF76AFF51
:10A0600001232A460A21ECE77FB5012504460DF1BC
:10A070000F030DF10E0100950022FEF76DFF9DF814
:10A080000E109DF80F6020460022FEF77CFC2A4649
:10A090003146204604B0BDE87040FEF774BCF8B508
:10A0A00004460F4601211D461646FEF79FFC20463A
:10A0B000FFF7DAFF0F212046FEF734FE2046FFF7B8
:10A0C000D3FF39462046FEF7FAFE20464FF0FF3117
:10A0D000FEF78CFC31462046FFF710F92046FEF7CC
:10A0E00036FCA06D01220021FEF7DAFA00221146AB
:10A0F0002046FEF748FCA06D4FF42051FEF723F9EF
:10A10000A06D2A460021BDE8F840FEF7C1BB000063
:10A11000138B2DE9F34104460161D81E43424341AC
:10A12000237500230E46E364118CA36962658B429C
:10A13000154605D2E069F6F7B6F82B8CE061A3610D
:10A14000626D538B928B1344EA8A510748BF0133E7
:10A1500092074FF0000248BF01331146934240F08E
:10A16000DB80227D002A40F0EB80A2699A4200F257
:10A17000E980226A002360219A4240F0EC80042E9C
:10A1800014BF01210221A06DFEF796F8626D002335
:10A19000A4F84830938CD28A02F01101194305D0FB
:10A1A000D20740F1DD801523A4F848308B492068A0
:10A1B000FDF756FB2F8C6B8C94F814803B440646BD
:10A1C0006364A06DB8F1000F00F00C81626D918C9A
:10A1D000002940F0CA80D28A12F0010F0CD1394612
:10A1E000032F6F8BA8BF0321032F88BF01F1FF311D
:10A1F00012F0110F00F0BB80B4F84820023292B286
:10A20000A4F84A201A44511A0227FEF7B4F800971E
:10A21000A06D012300220721FEF784FA0722009790
:10A220001146A06D0323FEF77DFA072200973346FF
:10A230001146A06DFEF776FA636D9A8C1AB9DB8A27
:10A2400003F030032BB1B4F84810A06D0022FEF7E4
:10A2500013FAA06D01220021FEF7E3F8A06D02229F
:10A260000121FEF7DEF80322A06D0621FEF7D9F8E2
:10A27000A06D4FF42451FEF766F8A368A06D1A682C
:10A2800001210432FEF704FB6A8BA06D0221FEF768
:10A290007CF9A06D022300224FF48541FEF7BCF843
:10A2A000A368A06D1A6800210532FEF7F1FAA368D1
:10A2B000A06D19680431FEF727F86B8BA06D4FF085
:10A2C00002125A430221FEF760F9A06D03222C21ED
:10A2D000FEF713FBA368A06D19680531FEF714F8AB
:10A2E00000250226636D5A8BAA4248DC032A0DD949
:10A2F0009A8C5AB9DB8ADB0708D4B4F84A20636C1D
:10A30000A06D1A44033A0621FEF7CAF9204602B0AE
:10A31000BDE8F041FFF7A8B9E069815401321DE7BB
:10A32000C86A00EBC20001324178CF0741BF4788BD
:10A33000E0690909C155616D088D9042F0DC14E7B0
:10A340000022F8E7227D002AE2690CBF002160218B
:10A35000D154013309E7606A20F8331001330BE769
:10A360000BB9132320E714231EE7002144E7EF8AEB
:10A37000B4F84820BF067FF543AF01323FE70096AF
:10A380002B460622A06D0021FEF7CCF9E3695A5D49
:10A3900022B1012303212046FEF7AAFB022D12DC85
:10A3A000636D9A8C7AB9DA8AD2070CD4022D02D165
:10A3B0005B8B032B07D10A4BA06D595D0022FEF782
:10A3C00030F801358EE7B4F84A10636C194401394E
:10A3D0000022491B2046FEF75DFBF2E7C0DE0508C0
:10A3E00080DD0508E26B0421FDF79FFFD4E91530FD
:10A3F000DF8A17F0010742D0226C0421FDF795FF98
:10A40000B4F84810A06DFDF7B6FF4FF4A023A36485
:10A41000A06D42460621FEF704F80227A06D012236
:10A420001421FEF729F90097B4F84830A06D0622F0
:10A430004146FEF777F90097A06D01234246414659
:10A44000FEF770F90097A06D032342464146FEF7E0
:10A4500069F90097A06D334642460721FEF762F97D
:10A460002046FFF701F9636D9A8C002A49D000233A
:10A4700019462A8D9A425BD802B0BDE8F081B4F843
:10A480004830616C05339BB24FF00208A4F84A30A3
:10A490001944FDF770FFCDF80080A06D3A46012306
:10A4A0000721FEF73FF9CDF800800722A06D114685
:10A4B0000323FEF737F9CDF8008007223346A06D5D
:10A4C0001146FEF72FF9B4F84810A06D3A46FEF792
:10A4D000D3F8626CA06D3946FEF757F8B4F848100F
:10A4E0003A4620460331FEF7D5FAB4F84820A06D6D
:10A4F0003946FEF7E9F8A06D04222D21FEF7FDF99B
:10A50000AEE7DE8A16F00106B1D1104F2B8CB342B4
:10A51000ADDDB4F84A20636C17F8011BA06D1A4436
:10A52000013A921B0136FEF7BBF8032EEED19EE7EF
:10A53000EA6A02EBC30012F83320052A04BF4288FE
:10A54000E06903F1010308BF815492E780DD05084B
:10A550002DE9F3410E4601EB4201044615461F4624
:10A56000FEF78EFA70288DF8060035D1E26C636A2A
:10A5700003EBC2030021204613F80C6CFEF780FAAF
:10A58000072805460DD888B12046FEF7DFFBE36CAF
:10A59000626A03F10053013B02F8336002B0BDE888
:10A5A000F0815428F0D01F4803F014FE02460DF14C
:10A5B00007012046FEF7C2FC2046FEF7C8F93246E6
:10A5C00003210123FEF794FA2A463146204602B0C1
:10A5D000BDE8F041FEF7D7B946EA05286FB18A1CFD
:10A5E00020460221FFF762F9434600221D21204642
:10A5F000FEF7A9FA00221146E8E7354304D00A46DF
:10A6000020460221FFF752F90DF1060120460022F3
:10A61000FEF794FC012342461B212046FEF768FA10
:10A62000E8E700BF598E05082DE9F041C66CD0F867
:10A6300024C0DDF81880013E0CEBC60715467A7879
:10A64000012A044613D1D7F804E09E450FD0C64531
:10A650000DD01CF836300B7079682960FEF78BFA44
:10A6600020464FF0FF31BDE8F041FEF763B90A46DE
:10A670002B6801212046FEF72FFCF1E77FB5002370
:10A6800003934FF0FF33009303AA0DF10B0104462F
:10A69000FFF7CAFF9DF80B50039E2946324620461D
:10A6A000FEF771F932462946204604B0BDE87040F5
:10A6B000FEF769B9F7B504460E461546002A57D18C
:10A6C000134601210DF10702FEF706FC0222114696
:10A6D0002046FFF72FFC012320460D220A21FEF71A
:10A6E00056FB0DF1070120460222FEF727FC0DF173
:10A6F000070120460122FEF721FC2A460DF1070141
:10A700002046FEF71BFC9DF80770204639460122C3
:10A71000FEF739F9394620460222FEF734F90222C3
:10A7200011462046FFF706FC012320460C220A2191
:10A73000FEF72DFB022211462046FFF7B7F82B4605
:10A740002A4620461C21FEF7FEF92A4629462046C5
:10A75000FEF719F92046FEF791FB2046012231460B
:10A76000FEF763F9204603B0BDE8F040FFF786BF6F
:10A77000FEF784FBAB1E5A425A413146204603B0D5
:10A78000BDE8F040FEF751B970B5044686B00D46FD
:10A79000164623B906B0BDE87040FEF7BBBC0022E8
:10A7A0001146FEF7E8F9204600220121FEF7E3F901
:10A7B000324629462046FEF727FA002304934FF03D
:10A7C000FF33009304AA0DF10F012046FFF72CFF81
:10A7D000049D009501262B4605AA0DF10F01204688
:10A7E0000596FFF721FF022300930599A06D3346DC
:10A7F0002A46FDF7D7FF06B070BD7FB504460D466B
:10A80000164623B904B0BDE87040FEF7FDB900223A
:10A810001146FEF7B0F9324629462046FEF7F4F914
:10A820004FF0FF330025009303AA0DF10B012046E2
:10A830000395FFF7F9FE02230093039AA06D2946C2
:10A840000123FDF76FFF2A462946204604B0BDE8E4
:10A850007040FEF798B800007FB50E460021044610
:10A86000FEF70EF9831E012B05468DF80B0038D834
:10A87000002E34D0012E19D10B460391009103AA6A
:10A880000DF10B012046FFF7CFFE039D44F240215E
:10A890002B462A46A06DFDF7BFFD9DF80B102A46FA
:10A8A000204604B0BDE87040FEF76DB8022E0ED110
:10A8B0000B460391009103AA0DF10B012046FFF70F
:10A8C000B3FE039D44F2C0312B462A46E2E7104B0B
:10A8D00064689A5D0F49104806F030FC206004B0AF
:10A8E00070BD70B901220DF10B012046FEF726FB69
:10A8F000324611212B462046FEF7FAF82A46294611
:10A90000CEE7FEF70DF8054964680246E3E700BFAD
:10A91000FCF60508618E0508F4E405086A8E050852
:10A920002DE9FF410D4601210446FEF7A9F800215B
:10A9300007468DF80A002046FEF7A2F8BB1E012B41
:10A9400006468DF80B0000F2D380831E012B00F227
:10A95000FA80A5F109030C2B9CBF0D35EDB21F2D1C
:10A9600001D0212D24D10023009301220DF10A03EF
:10A970000DF10B012046FEF7EFFA9DF80A30022B8D
:10A9800007D07A4B7A495A5D7A48666806F0D6FB5A
:10A9900030601F2D0CBF2E212F212046FEF7BBF863
:10A9A00000220221204604B0BDE8F041FDF7EBBFD4
:10A9B00001260223039303AA0DF10B012046009602
:10A9C0000023FFF731FE32460DF10A012046FEF763
:10A9D000B5FA1D2D7DD8DFE805F04C4C4C4C4C4CA5
:10A9E0007C7C7C7C7C7C7C7C7C7C7C7C7C7C7C7CA7
:10A9F000252D320F0F374347192DA06D9DF80A60A2
:10AA0000039B4FF0010206D14FF48141FDF704FD95
:10AA100001223146C6E7032E0CBF44F2C0014FF4B9
:10AA20008241F3E7039B01224FF48641A06DFDF7BD
:10AA3000F3FC11E0039B012244F24001F6E7039B83
:10AA400001224FF48041F1E7039941F60903A06D1B
:10AA500043EA8111FDF777FC9DF80A100122A1E776
:10AA6000039941F60923F2E7039B012244F24031A6
:10AA7000DCE79DF80A609DF80B30B34205D03E49F3
:10AA80003C48676806F05AFB38600022032E1146E6
:10AA9000204614BF06260026FEF76DF80122039B10
:10AAA000A06D4FF48541FDF7B7FC2E44334BA06DEC
:10AAB00033F81610FDF747FCA06D42F20101FDF7D7
:10AAC00042FC4FF40051A06DFDF73DFC0022012136
:10AAD00068E720460121FDF72DFF244B28495A5DE8
:10AAE0002448646806F02AFB206004B0BDE8F081C9
:10AAF00057EA000827D1012600960DF10A03022229
:10AB00000DF10B012046FEF727FA322D17D0332D19
:10AB100017D0464600232A4612212046FDF7E8FFBB
:10AB200056B1A06D00220121FDF77BFC002303221A
:10AB300011212046FDF7DCFF0022114632E70625F1
:10AB4000E8E70725E6E720464FF0FF31FDF7F2FE84
:10AB50003846FDF7E5FE02463046FDF7E1FE0949BD
:10AB600064680346034806F0E9FABDE7FCF6050809
:10AB70007A8E0508F4E405088A8E050890DC05083D
:10AB80009D8E0508AB8E05082DE9F0430446C1688B
:10AB900085B0FEF7B3FB626DD18A928C01F0110390
:10ABA00013432ED011F0010117D1B4F848202046EC
:10ABB0000132FEF715F8636D9D8C55B9A06D4FF409
:10ABC0002051FDF7C0FBE268A06D01322946FDF778
:10ABD0005FFE05212046FDF79EFF21212046FDF75F
:10ABE0009AFF636DDA8AD20706D49B8C23B9E16899
:10ABF00020460131FEF782FBA06D12220021FDF7F5
:10AC00004FFDA06DFDF7E9FB237D002B5ED1A36D09
:10AC1000656C5B68A36323685B88E363636D013DD8
:10AC20005E8BDF8AB3F81C90B3F81E80EA0006F052
:10AC3000030302F0780207F00F071A432D09B60844
:10AC400045EA0703334343EA090353EA0803A06DC7
:10AC500065D10121FDF769FBB4F85060B4F852707A
:10AC6000A06D720007F0010302F07E027F08B609B2
:10AC700057EA060542EA030218BF42F080020121AA
:10AC8000FDF753FB002DEBD1636DA76D998A20680A
:10AC90007E68FCF7CFFD47490246384610F086FC37
:10ACA000626D538B918B108D0B44AB4271DCA36DA5
:10ACB0009F88BE1BA4F850600025D4E915301A8D7A
:10ACC000AA4268DC4368DB1BA4F852302369042BDA
:10ACD00021D1A36DD3E9027623685868237D5BB93F
:10ACE000A56BE16B3544002962D001318900F5F78D
:10ACF000DAFAE36B40F823500023656D217DCDE93E
:10AD00000233EB8ACDE90003033128693B46324622
:10AD1000C9B201F02BFE012005B0BDE8F08342F07E
:10AD200080020121FDF701FBBA012B0103F0300382
:10AD300002F040021A4308F001031A434FEAC90324
:10AD400003F008031A43B30003F004031A43AD08E9
:10AD50007F0876084FEA59094FEA580870E7D36A26
:10AD600003EBC1035F78FF070ED55F88AF420BD1BD
:10AD700059682068A76DFCF75DFD0E49024638460C
:10AD800010F014FC01358BE701318142E7DB05212E
:10AD9000EFE70021F9E7DB6A03EBC50213F8353072
:10ADA000052B03D152880121FDF7BFFA013584E755
:10ADB0002846A1E7E98202082DE9F04188B004465F
:10ADC0000D4607AE002940F0BD800121FDF758FE79
:10ADD00007468DF8170078BB01462046FDF750FE68
:10ADE000C0B9012231462046FEF7A8F800220DF135
:10ADF00017012046FEF7A2F804220F210223204665
:10AE0000FDF776FE00221146204608B0BDE8F0416D
:10AE1000FDF7B9BD3A4631462046FEF78FF89DF85A
:10AE20001C20204601230421FDF762FEA06D3A4656
:10AE30000121FDF7F6FAD9E7E36C626A013B02EB08
:10AE4000C30032F8332040F202239A422BD14768E4
:10AE50004FF001082046FDF77AFD434632460DF1DA
:10AE60001701CDF800800795FFF7DEFB20462A4644
:10AE70002946FDF780FE9DF8170006280DD007280B
:10AE80000ED0052854D10095079AA06D3B4629465F
:10AE9000FDF748FC00220221B6E7CDF80080F3E779
:10AEA00002230093F0E72B460791324606A920467D
:10AEB0000095FFF7B9FB2A460DF117012046FEF772
:10AEC0003DF820462A462946FDF755FE9DF8180014
:10AED000831E012B08D9FDF723FDA14965680246B1
:10AEE000A04806F02BF928609DF8170006280BD023
:10AEF000072813D005281BD10799890141F4B841CF
:10AF0000A06DFDF720FAC5E70799A06DC90041F0D3
:10AF10004201FDF718FA4FF4B541F1E70799A06D2A
:10AF2000C90041F08201FDF70EFA4FF4B141E7E7A5
:10AF3000FDF7F6FC8C49656802468A4806F0FEF883
:10AF40002860A7E7012940F0FB80FDF799FD07463F
:10AF50008DF8150050BB01462046FDF791FD0221FA
:10AF600005468DF818002046FDF78AFD05438DF84B
:10AF70001C0008D0394620460322FEF797FC032127
:10AF80002046FDF7D7FC0223CDE90163002300939F
:10AF900006A920460DF115030122FEF711F80F2135
:10AFA000204608B0BDE8F041FDF7B5BDE36C626A2C
:10AFB000013B02EBC30132F8332040F202239A42F4
:10AFC0003ED12046D1F80480FDF7C1FC02230022C7
:10AFD000CDE90623009306AA2B460DF11501FFF7D4
:10AFE00023FB069F00953B46204632460DF1170194
:10AFF000FFF71AFB9DF81700431E022B08D9FDF737
:10B000008FFC5A4965680246564806F097F8286052
:10B010009DF8150006280FD007280FD0052840F00E
:10B020008580002300930799A06D43463A46FDF7BB
:10B03000B9FB08B0BDE8F0810123F3E70223F1E793
:10B0400002230793009306AA00230DF11601204660
:10B050000695FFF7E9FA204600220DF11501FDF7EC
:10B060006DFF9DF81600831E012B08D9FDF758FCD3
:10B070003F49656802463B4806F060F82860069D37
:10B0800000950023204632460DF11701FFF7CCFA58
:10B090009DF81700431E022B08D9FDF741FC3349E8
:10B0A000666802462F4806F049F830609DF81500A2
:10B0B00006280ED0072825D0052837D1079941EA60
:10B0C000851141F4A841A06D08B0BDE8F041FDF73D
:10B0D0003AB90126AE40A06D46F43441FDF733F98C
:10B0E00045EAC50141F04001A06DFDF72CF9079933
:10B0F00041EA851141F4A441A06DFDF724F946F41D
:10B100003C41E0E70126AE40A06D46F43441FDF736
:10B110001AF945EAC50141F08001A06DFDF713F968
:10B12000079941EA851141F4A041E5E7FDF7F8FBF5
:10B130001049646802460B4806F000F8206078E782
:10B140000025334606A900950122FDF705FF0223DD
:10B150002A460F21204608B0BDE8F041FDF7C8BCE3
:10B16000CE8E0508F4E40508C58E0508D88E0508BE
:10B17000E38E0508DD8E05082DE9F04180465C2050
:10B1800016460F461D46F5F78CF8866008260446DD
:10B19000C0E9008706624020F5F76AF8E66260625F
:10B1A0002020F5F765F860632020F5F77AF8294646
:10B1B000A065FDF76EF82046BDE8F08110B50446A5
:10B1C0000021806DFDF76DF8A06DF5F779F8606BE3
:10B1D000F5F776F8E069F5F773F8606AF5F770F857
:10B1E0002046BDE81040F5F76BB8000002F00F03F1
:10B1F000022B10B5044608D00A460C490C4805F04D
:10B200009DFF636A1860002010BD836A1209002048
:10B21000834204D1238C042BF5D10649EEE7E16A81
:10B2200051F820109142EFD00130F1E7EA8E050885
:10B2300060E50508F08E050870B50646B2B19007C6
:10B2400014D110792E2811D194687CB1A2070DD1A8
:10B250006568EAB2922A09D12D0A022D06D1A268A8
:10B260001A60049BE2681A60012070BD0A46044817
:10B27000044905F063FF736A18600020F5E700BF1A
:10B2800060E50508FC8E05087FB504460D461046AE
:10B2900003A91E46F8F776FD48B90C490C482A4622
:10B2A00005F04CFF636A1860002004B070BD03987D
:10B2B00003F050FE30EA06020346F6D00549009638
:10B2C0002A46034805F03AFFECE700BF188F05084F
:10B2D00060E505081E8F0508038C032B70B5C46A52
:10B2E00003D1856A00239D4205D144F82120FDF752
:10B2F0000BF8012070BD54F82360964201D0013351
:10B30000F1E70020F6E7FDF768B8032910B5044619
:10B31000018442620FD1826AC06A002192001EF04D
:10B32000E3FB01212046FCF7C7FF20460021BDE8D2
:10B330001040FDF720B8042914BF01210221F1E7D4
:10B3400000F00F03022B02D10009F5F7B4BE01484B
:10B35000704700BF4BA7050870B5054610460E465E
:10B36000FFF7EEFF0378732B19D14378BBB1034687
:10B370000A22002013F8014F5CB91F2808D90B4995
:10B380000B481F23324605F0D9FE6B6A1860002077
:10B3900070BD303C092C02D802FB0040EAE70549A9
:10B3A0000348324605F0CAFEEFE700BF348F0508B8
:10B3B00060E50508418F0508F8B5054610460E46BC
:10B3C0001F46FFF7BDFF174C01780022A4466378A3
:10B3D0008B421BD190F801E0A3789E4516D190F8DE
:10B3E00002E0E378734511D16BB91CF82200B84232
:10B3F00008D90D490D483B46324605F09FFE6B6A61
:10B4000018600020F8BDC378002BEED00132152A59
:10B4100004F10404DBD106490448324605F08EFEEF
:10B42000EDE700BF38DE0508348F050860E5050844
:10B430004A8F05082DE9F34706460F46002A3CD0FF
:10B4400093073AD113792F2B37D1926802F00F036B
:10B45000022B08D10F23FFF7AFFF012484402046C1
:10B4600002B0BDE8F08742B312F0030A25D1137988
:10B470009F2B22D1D5682B79A12B1ED192680F2347
:10B48000FFF79AFF4FF0010909FA00F401AAA2217F
:10B4900005F10800F8F7C2FE8046C245DFDA019ADE
:10B4A0000F2352F82A2039463046FFF785FF09FA64
:10B4B00000F004430AF1010AEFE7044904483A4660
:10B4C00005F03CFE736A00241860C8E7508F050839
:10B4D00060E5050810B50446024805F099FD2060B6
:10B4E00010BD00BF60E5050804292DE9F84380463A
:10B4F0000C460DD8151F01F1300930264E450DD0F0
:10B5000055F8040F00F00F03022B0AD00D4900E09C
:10B510000D49D8F82400FFF7DDFF00242046BDE8E0
:10B52000F8830009F5F7C7FD07461EF01BFB02284C
:10B53000ECD13B78722BE9D17B78B342E6D101366E
:10B54000DCE700BF808F0508618F05082DE9F04713
:10B550000F4686B0044603A938461E469146F5F7C5
:10B56000B6FD0378762B054640F01881B9F1020F3D
:10B5700040F0C580A7F2F6470D2F00F20681DFE804
:10B5800017F00E0036003900040104010401040123
:10B590008C0004015E003C0031002E00BB004EF622
:10B5A000B4684FF42C69326829462046FFF7D4FE70
:10B5B0007268074629462046FFF7CEFEFA0249EA9E
:10B5C000500902F47042400142EA090200F02000F2
:10B5D000B90101F04001024348EA010129E04EF6B9
:10B5E000B168DEE74EF6B1684FF42469DBE74EF64A
:10B5F000B868D6E74EF6BD68D3E73068FFF7A0FE1F
:10B60000AB491EF0BDFAC0B132680F23294620466F
:10B61000FFF7D2FE07467068FFF792FEA5491EF0BD
:10B62000AFFA002840F0B1803A0342F421624EF6AE
:10B63000F1612046FCF791FEE9E10F27EBE7306866
:10B64000FFF77EFE03783268722B17D10F2329464D
:10B650002046FFF7B1FE2946726807462046FFF7ED
:10B660007BFE4EF6106180464FEAC812D2B242EA23
:10B67000073242F4216241EA5801DAE729462046BE
:10B68000FFF76AFE2946726880460F232046FFF7BF
:10B6900093FE4FF46E410746E6E74EF69058326847
:10B6A00029462046FFF758FE05AB0093074672680F
:10B6B00004AB29462046FFF7BFFD002800F0A78114
:10B6C000049A072329462046FFF776FE059A064688
:10B6D00029464FF47F732046FFF7D6FDFA02B901E1
:10B6E00002F4704201F0400142EA900241EA08018E
:10B6F00042F4206231439CE74EF68058CFE7B9F11F
:10B70000030F42D1DFF8C481002700F1010A0322B0
:10B71000414650461EF04CFA90BB2B7983BB664BDA
:10B72000326813F8278029462046FFF715FE726815
:10B73000074629462046FFF70FFEB2688146294694
:10B740002046FFF709FE4FEA0813DBB243F42063FB
:10B7500043EA5003400100F02000FA0202F4704274
:10B760000343134308F0F0084FEAC912D2B248F479
:10B770006E48B90148EA590801F040011A432BE725
:10B780000137042F08F10408C1D14B464B494C48FE
:10B790002A4605F0D3FC636A186038E1B9F1030F5B
:10B7A000F3D8DFE819F0040015001901CB0240F2CC
:10B7B0003D439F4205D14FF43F412046FCF7C3FD76
:10B7C00025E140F205539F42DFD14BF63071F4E79B
:10B7D00040F24232974210D1014632682046FFF7CC
:10B7E00005FD01462046FCF740FE002840F00F8191
:10B7F0003449606AFFF76EFE09E140F24A3297422F
:10B8000009D1014632682046FFF7F0FC0146204688
:10B81000FCF785FEE9E740F25232974209D1014632
:10B8200032680F232046FFF7C7FDC10041F48E4167
:10B83000C3E7622B4CD1039B032B0CD0052B40F0AC
:10B840008E80C3785F2B40F08A8003796E2B02D004
:10B85000772B40F0848069781B4B00224FF0FF3734
:10B860005878884205D195F802C09878844508BF79
:10B870001F7801320E2A03F10303F1D17B1C84D01F
:10B88000326829462046FFF7B1FC039B052B024690
:10B890000BD12B79A3F1770CDCF1000343EB0C0304
:10B8A00039462046FCF7FFFD9FE70023F8E700BF7D
:10B8B000958F05089F8F050898DD0508B28F05084C
:10B8C00060E50508BF8F0508FCDD050899DD050862
:10B8D000692B44D14378742B41D13068FFF730FD98
:10B8E000B84B017800221F465E788E4222D190F834
:10B8F00001C09E78B4451DD18678DEB9AE1C3146B4
:10B900000B46013118780028FAD1691D8B423FF6A9
:10B910003CAF02EB42020821BF5CFA43D200F800C0
:10B92000013B0A4008409E420AD941EA071141F40E
:10B930003F4142E701320E2A03F10303D4D124E749
:10B9400013F801C9BCF1740F4FEA510101D1014351
:10B95000E9E7BCF1650F7FF418AF1143E3E740F26C
:10B9600071339F4202D14BF2726126E740F272338B
:10B970009F4202D14BF262611FE740F266439F4251
:10B9800013D1326829462046FFF754FD10F43F4F8B
:10B99000024607D146044ABFC1B240F4344141F4E3
:10B9A00035410AE74EF62D1143E6782F7FF4EDAED0
:10B9B000326829462046FFF73DFD10F4FE4F02464F
:10B9C00007D105044ABFC1B240F43C4141F43D41B6
:10B9D000F3E64EF6BD012CE6736803F00F03022B6D
:10B9E00040F09E80B7F5866F14D1014632680F2370
:10B9F0002046FFF7E1FC7268074629460F232046E0
:10BA0000FFF7DAFC394602462046FCF70AFD06B08D
:10BA1000BDE8F08740F261339F421CD14FF6B02958
:10BA20004FF2800732680F2329462046FFF7C4FCF7
:10BA30007268804629460F232046FFF7BDFC47EA7F
:10BA4000000242EA082249EA0001F2E54FF6902995
:10BA50004FF2A007E6E740F271439F42F6D040F272
:10BA600034439F422AD132680C2301462046FFF717
:10BA7000A3FC07467068FFF763FC01460646524880
:10BA80001EF07EF80346A0B1504831461EF078F80B
:10BA900070B12A464E494F4805F050FB636A0022B8
:10BAA000186042EA072242F400424FF2EF31C0E54B
:10BAB0000123494A03EBC303D25CF2E740F235337A
:10BAC0009F4215D14FF4804732682946072320460C
:10BAD000FFF772FC72688046294607232046FFF76D
:10BAE0006BFC4246034639462046FCF795FC8EE740
:10BAF000DFF8EC8000270322414628461EF058F864
:10BB000040B9EB7833B9354B13F827703F0147F450
:10BB10008047D9E701370F2F08F10408EBD134E64D
:10BB200040F233439F422BD8B7F5866F1FD240F2C5
:10BB300063339F423DD040F2FD339F4200F0878047
:10BB400040F22B339F4237D040F2FB339F4200F04C
:10BB5000DD80B7F57F7F00F0DB8040F2FE339F424F
:10BB600000F0D880972F40F09F800323A1E06FF46E
:10BB700086600744022F22D8DFE807F04B344E00DE
:10BB800040F2CA439F4240F08B804FF460573268C6
:10BB9000072329462046FFF70FFC29468046726896
:10BBA000FF232046FFF770FB47EA000141EA082126
:10BBB00003E64FF42057EAE74FF44057E7E74FF426
:10BBC0000057E4E7FCDD050827DE050830DE050840
:10BBD000A58F050860E5050826DE0508C0DD050817
:10BBE000C1DD05084FF2402832680F232946204660
:10BBF000FFF7E2FB726807464FF6FF7329462046BF
:10BC0000FFF742FB3A46034641462046FCF71BFC41
:10BC1000FDE64FF2C028E7E7294632680F232046A9
:10BC2000FFF7CAFB2946074672684FF0FF332046EC
:10BC3000FFF72AFB3A4683B205464FF240212046E1
:10BC4000FCF701FC2B0C3A464FF2C021DDE7014620
:10BC500032680F232046FFF7AFFB05AB0093074682
:10BC6000726804AB29462046FFF7E6FA00283FF445
:10BC7000CEAE049A0F2329462046FFF79DFB059A76
:10BC800006462946FF232046FFF7FEFA820842EACD
:10BC9000073246F4684142F4706241F05001C8E452
:10BCA00040F2C6439F4237D0B7F5996F7FF46DAD30
:10BCB0000523844A294632F8237032680723204638
:10BCC000FFF77AFB05AB00938046726804AB294608
:10BCD0002046FFF7B1FA00283FF457AD049A2946F1
:10BCE00007232046FFF768FBF904059A064615D599
:10BCF0001F2329462046FFF7C7FA47EA08078001B5
:10BD000047EAC60700F4F861394356E50023D0E757
:10BD10000123CEE74B46CCE70423CAE73B0406D514
:10BD20003E2329462046FFF7AFFA4008E5E77C238B
:10BD300029462046FFF7A8FA8008DEE740F20C43C8
:10BD40009F4221D100273268072329462046FFF76A
:10BD500033FB72688146072329462046FFF72CFBF8
:10BD600029468046B2681F232046FFF78DFA47EA2E
:10BD7000090747EA801747EAC8011EE54FF4006744
:10BD8000E1E74FF48057DEE740F20D439F42F5D0E4
:10BD900040F23E339F42F4D040F22B339F422BD1EE
:10BDA0004FF4C0583268072329462046FFF704FBAA
:10BDB00072680723074629462046FFF7FDFAB26856
:10BDC00002F00F03022B81460ED10723294620469D
:10BDD000FFF7F2FA47EAC90141EA080141EA801196
:10BDE000EBE44FF4D058DDE707232946204648F41A
:10BDF0008068FFF749FAEDE740F29F439F4222D166
:10BE00004FF6903832680F2329462046FFF7D4FAC0
:10BE1000726881460F2329462046FFF7CDFAB268A3
:10BE2000074629460F232046FFF7C6FA40EA0920B5
:10BE300040F4704242F0F00248EA0701FFF7F9BB14
:10BE40004FF6B038DEE740F2E9439F42F8D040F2C7
:10BE5000CA439F42C5D040F2C7439F427FF495AC8E
:10BE6000014632680F232046FFF7A6FA72680F23B7
:10BE7000294607462046FFF79FFA05AB0093804608
:10BE8000B26804AB29462046FFF7D6F900283FF4F4
:10BE9000BEAD049A0F2329462046FFF78DFA059A76
:10BEA00006462946FF232046FFF7EEF93F0247EA00
:10BEB000083746F4684147EA900241F04001FFF735
:10BEC000B8BB00BFA8DD050838B505463020F4F73B
:10BED000CFF92022044600211DF006FE2946204607
:10BEE000FCF7D7F9A562A800F4F7C2F9E062204692
:10BEF00038BD10B50446C06AF4F7E2F920460021C7
:10BF0000FCF7CFF92046BDE81040F4F7D9B92DE988
:10BF1000F04F099FDDE90BC4DDE90D5650B18842B1
:10BF200008D3710747BF0137013401350A2158BFD3
:10BF3000B0FBF1F016F0020E39D0002D37D00BDB3C
:10BF40000A998D4233DA2C44A74203DC07F1FF3C07
:10BF5000A4EB0C0C00252AE0291D28DB69424FF0D8
:10BF600000084FF00A0AB0FBFAF90AFB19041CB1E9
:10BF700008EB0504414604E008F1010888454846FD
:10BF8000F1D11D464FF0300905F8029B7F1A091BBD
:10BF90004FF02E084C1E83F801802346A846002B44
:10BFA0005DDC002908BF00242B190025FF2407F1C0
:10BFB000FF3841464FF00A09002954DA611CB942A2
:10BFC00060DBFE2CD4BF002101213B44BCF1000FFB
:10BFD00007D0A4EB0804A4EB0C0C2E2030276445FA
:10BFE00055D1BEF1000F09D041B119460B4611F8E9
:10BFF000010D3028FAD02E2808BF0B4606F00101AB
:10C00000294327D0710725D4002DBABF6D422D21B9
:10C010002B2106F02004632D597044F04504C8BF5D
:10C0200064211C704FF00A00C9BFB5FBF1F19C1CE4
:10C03000DC1C3031C8BF9970B5FBF0F62346B6FB67
:10C04000F0F100FB1161303103F8021B00FB1651C7
:10C050003031617000211970981ABDE8F08F08F82E
:10C06000019B013B9BE78C42B4BF01F1010B8B4666
:10C07000B0FBF9FA09FB1A00303003F80B00013964
:10C08000504699E701332E21195501219DE714B936
:10C0900003F8010B012103F8017B013C9FE700003D
:10C0A0002DE9F04F2DED028B884610EE101A97B057
:10C0B00000291C46B0EE408A9DF888300E902ADA9E
:10C0C000B4EE400AF1EE10FA25D6B1EE408A2D23E7
:10C0D0000E9F07F8013B08F1FF389FED7D7AF0EEE7
:10C0E000C87AF4EE477AF1EE10FA02F0200316DD7A
:10C0F00043F0490443F04E00FA1C43F0460100238C
:10C1000078703C70B97013700E9BD01A17B0BDECEC
:10C11000028BBDE8F08F002BDAD10E9FDDE7B4EE85
:10C12000488AF1EE10FA06D743F04E0143F0410081
:10C13000FA1C0C46E3E742F02002662A4FD143F096
:10C14000040B002CA8F1030650DA0624A64233465D
:10C15000A8BF23460C9318EE103A002B099353D036
:10C16000C3F3C7537F3B07EE903A9FED5A7AF8EE40
:10C17000E77A18EE103A67EE877AB3F17E5FFDEE4C
:10C18000E77A38BF4FF0000917EE905A28BF4FF0FA
:10C19000010909EB0500B7EE000A00F047FA099B18
:10C1A000B3F17E5F2CBF4FF0010A4FF0FF3AB4EEBF
:10C1B000C80AF1EE10FA94BF012300234B451BD0AF
:10C1C0001BF0040F4CD0002D20DD6319023398457D
:10C1D0001CDA8BF0040343F0020B013444E0672ABD
:10C1E0000CBF43F0020B43F0010BAAE7632CADD167
:10C1F00010230C930924AEE7554405EB0900B7EE74
:10C20000000A00F013FAD2E7099DD9E7A8F102026B
:10C21000A242D4BF33462346002D1EDA022B15DD81
:10C22000AA1C17DA6E429E42A8BF1E46023E9C1B05
:10C23000092C0DDD1BF00403A4F1090207934FF054
:10C2400009041CD004230793032319E05C1C002677
:10C250000022F7E75C1C0026EAE76C1C1C44FAE7A6
:10C260001BF0020FB9D034B1092C4FF00006E1DC0D
:10C270003246079603E02646224607940124072308
:10C28000062CA146A8EB0408A8BF4FF00609A8EBAE
:10C290000308A9EB0503013B0D939045D4BF04EBC4
:10C2A0000803A3181193119BA3EB09030F93099B98
:10C2B000002B00F0CB80079B002B00F0C380002DEB
:10C2C00080F2BD8046B909F1FF3008963B4613E085
:10C2D000FFFF7F7F9B209A3E3B46302103F8021BE5
:10C2E0002E227A70184632461DF0FEFBFF220346CE
:10C2F000334409EB060008920A214FF0010C0A9121
:10C30000E14500F3A880B9F1060F40F3AF800128A2
:10C3100040F3AC80B9F1070F00F0A480022800F0D0
:10C32000A18002384FF06408B0EE480A0B9300F089
:10C330007DF9F6EE007A30EE270A0A99BCEEC00AC3
:10C340003A4610EE103A08FB03F8089B03930F9B44
:10C3500002930C9BCDE9045BCDE9009340460B9B17
:10C360001093FFF7D4FD15AA01460B90384600F054
:10C370008DF9DDED157A0B9977EEC87A17EE902AD4
:10C38000002A58D0B9F1060FC4BF09EB4902123A8E
:10C390004FF0010AC8BF0AFA02FA0C22109BCDF82E
:10C3A0002C80F0EE678A109217EE902A002A089AE5
:10C3B00003920F9A02920C9A0A991393B4BFD04435
:10C3C000A8EB0A08CDE90092CDE9045B3A46404665
:10C3D000FFF79DFD15AA01461290384600F056F968
:10C3E000DDED157A129977EEC87A17EE902A12B31E
:10C3F000B0EEE77AF0EEE86A37EE667A139B17EE56
:10C40000102A002A35DB4FF00A0CB8FBFCF00CFBBD
:10C4100010800243002A0B9A08BF42460B9208BFC5
:10C42000F0EE678ABAF1010F28D0109A013A4FEA6C
:10C430005A0A1092B8D10E9B3944C81A66E60D9874
:10C44000089543E7079B0D9808933FE7099A0892E0
:10C450003B46104650E70A990A2251430A910CF1D3
:10C46000010C4DE701384FF00A085DE74FF0010875
:10C470005AE7CDF82C80F0EE678AD3E70D9AA145F4
:10C4800002F101020D9202DA09F101090BE70B9AA0
:10C490009045D0D0089A03920F9A02920C9ADDE947
:10C4A0000A10CDE90092CDE9045B3A46FFF72FFD73
:10C4B0000146C0E7012910B5136823D90178302956
:10C4C00020D1417841F02001782900F1020406D101
:10C4D00033F0100314D110231360201A10BD6F29FC
:10C4E00004D133F008030BD10823F5E7622904D106
:10C4F00033F0020304D10223EEE70BB901231360EA
:10C500000446EAE7002BFBD10A23F8E708B5044606
:10C5100031B1054B4A6B03600968002304F05AFEF1
:10C520002046F3F77DFE00BF60E505082DE9FF41D9
:10C53000044601921F4646182AB1023A222A02D91D
:10C54000374801F079FCB442254626D34FF0000865
:10C55000711B284601AAFFF7ADFF019B0544284641
:10C560000024B04201462AD3B8F1000F00D0644243
:10C57000640044F00104A94204D00D46B5422B46A4
:10C5800042D348D0019A27492748012A08BF0022F0
:10C5900004F0D4FD3946FFF7B9FF14F8010BF5F7A5
:10C5A00073FB80460028CED12B782B2B01D125465A
:10C5B000CEE72D2BCAD125464FF00108C8E710F869
:10C5C00001CBACF13002092A0AD9BCF15F0FC8D007
:10C5D0004CF02002A2F1610CBCF1190FC4D8573AFB
:10C5E0009342C1D983FB0441B1EBE47F03D11444EE
:10C5F00094EA4402B5D5711B424603A8039505F0A1
:10C60000B8FF03990446B6E718780135F5F73CFB07
:10C610000028B3D1B6E7204604B0BDE8F08100BFE2
:10C62000CA8F0508DF8F0508D0E4050808B52DED91
:10C63000028BE8B1B5EE400AF1EE10FA18D010EE18
:10C64000103AC3F3C752024462F3DE5310F10A0FEB
:10C6500008EE103A0FD3434200EE903AB1EE040ACE
:10C66000F8EEE00A1BF0DCFEF0EE407A88EE270AD6
:10C67000BDEC028B08BD07EE900AB1EE040AF8EE9D
:10C68000E70A1BF0CDFE28EE000AF1E700232DE9B2
:10C69000F0470144044690469E461D4618461F46F4
:10C6A0009A461E468C4257D2A4461CF8012BA2F192
:10C6B0003009B9F1090F38D8022E07D1354A904216
:10C6C00002DC0A2202FB00906446EBE7B9F1000F9E
:10C6D00014D0314A974211D80A24B5B975460A24B4
:10C6E000CDB997421ED8012E4FF00A0208BF03F1C0
:10C6F000FF3302FB07974FF0000EE5E70EB9013557
:10C70000E2E70EF1010E0126DEE7974294BF674390
:10C710000133013DE1E797429CBF03F1FF336743DB
:10C72000013DDDE77EBB0133E5E78EB92E2AEAD075
:10C7300042F02009B9F1650F0CD1614504D9627846
:10C740002B2A19D104F1020C8C4520D00226BBE71C
:10C75000022EEDD15F2AB7D0BAF1000F15D107EE46
:10C76000907A1D44B8EE670A2844FFF75FFF88ED12
:10C77000000A2046BDE8F0872D2AE7D104F1020C1B
:10C780004FF0010AE0E7AE46BDE74042E7E700248C
:10C79000EFE700BF64666606979999192DE9F04F97
:10C7A0002DED048B83B09FED658ADDF840909FED01
:10C7B000649A054690461F4646184FF0000AF0EE70
:10C7C000488ACDED018AB5422C466CD34FF0000B60
:10C7D000A31C9E4240F28980237843F02003692BFA
:10C7E00073D1637843F020036E2B7ED1A37843F09E
:10C7F0002003662B79D14FF0FF430193E31D9E4246
:10C8000004F103001AD9E37843F02003692B15D112
:10C81000237943F020036E2B10D1637943F020037A
:10C82000692B0BD1A37943F02003742B06D1E37954
:10C8300043F02003792B01D104F10800B8F1000F77
:10C840000ED0B0420CD2037843F020036A2B07D1FC
:10C85000844204BF4FF07E53019301304AF0020A34
:10C86000BBF1000F05D0DDED017AF1EE677ACDED79
:10C87000017A844240D00446B442254643D348D18D
:10C88000BAF1010F38D09DED010ABAF1000F4AD07C
:10C89000F0EE400AB0EE480A03B0BDEC048BBDE8F0
:10C8A000F04F03F08BBB15F8010BF5F7EDF983465C
:10C8B000002888D123782B2B01D12C4688E72D2BFB
:10C8C00084D12C464FF0010B82E76E2B0DD163789B
:10C8D00043F02003612B08D1A37843F020036E2B93
:10C8E00003D1E01C8DED019AA8E701AA311B204677
:10C8F000FFF7CCFE0028A1D11249134804F088FBB1
:10C900004946FFF703FE28780134F5F7BDF9002802
:10C91000B2D1002FF0D0BAF1000FEDD19DED018A18
:10C920004FF0010A4DE717B1DFED040AB4E703B099
:10C93000BDEC048BBDE8F04F04F040BD00000000EA
:10C940000000C07FEB8F0508D0E4050808B5102073
:10C95000F3F7A7FC0123837008BD10B503F00103B2
:10C960000224C0E901128470C37010BD9DF8043028
:10C97000426003F00103C370009B8360029B03735A
:10C98000C368039A817062F31F23C360704700007D
:10C9900070B504460D4623881046CBB10A460023E5
:10C9A000214605F0BDF82346002213F8011B1D1B8C
:10C9B000090605F1FF3503D4D30725D51C4B19E033
:10C9C00013F8011BC1F3801606FA05F52A43EEE7BA
:10C9D000A3786668042B0FD0052B16D0032B0A46CC
:10C9E000A36831461DD105F09BF8124B0360E37834
:10C9F00053B1114B036007E01049A468102002F006
:10CA0000B3F9C0E90154C66070BD0D49257BE468E7
:10CA1000102002F0A9F9C4F31724C0E90156C4603C
:10CA2000F2E705F07DF8E378002BEDD0C6E700BF14
:10CA300078EA050830E905085CEA050818E9050800
:10CA400000E9050838B5144612F4807218BF1A467A
:10CA50001D46FFF79DFF620902F008022A44E1B279
:10CA6000BDE8384003F044BAD0E90003184770B578
:10CA700005460C468E18B44200D170BDD5E90003BE
:10CA8000984704F8010BF6E738B504460025D4E9C9
:10CA90000003984700F07F0343EAC5150306F6D468
:10CAA000284638BD2DE9F04186B00546FFF7DCFF8A
:10CAB000C4B2042C06D8284B53F82440204606B0B4
:10CAC000BDE8F0812846FFF7DFFF064630B9062CA7
:10CAD00004D12846FFF7C8FF204CEFE70A2C10D1FD
:10CAE0000021304609F022FF0027044600F1040827
:10CAF000B742E3D02846FFF7D5FF013748F8040FC7
:10CB0000F6E7314602A8F4F7BFFB049932462846FF
:10CB1000FFF7ADFF631F012B0CD82846FFF7A4FFDA
:10CB2000052C02A803D108F023F80446C6E708F054
:10CB300025F8FAE7072CDDE903104FF0000303D1D5
:10CB40000A22FFF7F3FCF0E7093C624200936241DE
:10CB5000FFF724FEE9E700BF8CDE05082CF205088C
:10CB60002DE9F8432B4E04460F46904600252068D9
:10CB7000FFF77AFF5FFA80F9B9F1FF0F01D1BDE845
:10CB8000F883C1070CD52068FFF77EFFC20748BFB6
:10CB9000A3684FEA50054FEA850554BFED19ED181B
:10CBA0004FEA5903082B21D8DFE803F005050505F6
:10CBB0000505171B1E00DB070DD52068FFF764FF76
:10CBC0005FEA990923D0B9F1010F0CBFA368E368AC
:10CBD0000246294616E00120F2E763689B680120BF
:10CBE000F6E76368DB68FAE73346F8E703F180436A
:10CBF000084A093B52F82330F1E751F804CB9C4432
:10CC000041F804CC013AF8D205EB8005AFE7434682
:10CC1000DEE700BFC0DE05082DE9F04F8FB080468B
:10CC20000991FFF731FF00F003039A1C0492C20838
:10CC300000F004090792002B3FD11046F3F718FBD0
:10CC40004FF0000A0146079A06464046FFF70FFFDD
:10CC50005746CDF820A05446CDF814A05546B9F15A
:10CC6000000F00F098804046FFF70EFF049B8146BE
:10CC7000032B08BF01308000F3F7FAFA4FF0000BE6
:10CC80000690CB457DD1FFF761FE049B022B8346C6
:10CC900040F08C803246002312F8011B901B0906DD
:10CCA00000F1FF307AD4069A9BB231465846FFF71E
:10CCB00054FE58460FB0BDE8F08F0798F3F7D8FA46
:10CCC000079A014606464046FFF7D1FE049B032B18
:10CCD000404618D1FFF7D8FE04463018335D411C9A
:10CCE00000270A1A1D0602F1FF3204D44FF0000A91
:10CCF000CDF820A0B0E711F8013BC3F3801505FA89
:10CD000002F21743EDE7FFF7BFFE049B052B074632
:10CD10000BD14046FFF7B8FE08904046FFF7B4FE3F
:10CD2000002482460594254699E710F0200B23D075
:10CD30004046FFF7A9FE824617F0400002D0404669
:10CD4000FFF7A2FE1AEB000418D0C51C25F003055E
:10CD50000AEB0500F3F7A5FA05900544BBF1000FB7
:10CD600004D0524629464046FFF781FE4FF0000AA4
:10CD7000CDF820A0544672E7DA46DDE7A2460894D3
:10CD8000D0E709994046FFF747FF069B43F82B0081
:10CD90000BF1010B75E7CDF8189074E712F8011B41
:10CDA000C1F3801404FA00F0034377E7099BCDF840
:10CDB0002880CDE90B35059B0D93FB0610D5154D4D
:10CDC000D5F8CC0020B9014606F078F8C5F8CC00BB
:10CDD000314605F0E8FD324631460AA8FFF7C0FEAD
:10CDE000049B032B06D13444B9F1000F03D0069BFA
:10CDF00043F82940069C089B0293BFB2CDE9004747
:10CE0000079B0499CDF80CA032465846FFF7AEFDBB
:10CE10004FE700BF700400202DE9F04786B083681B
:10CE2000049304460368059302A80F463E49F3F7AE
:10CE3000BDF904220DEB02012046FFF718FE9DF814
:10CE400006509DF80420AB084D2A03F02F030CD1A7
:10CE50009DF80520062A08D11BB105F00302032A1C
:10CE600003D19DF807201F2A02D9304800F0E4FFC3
:10CE700023B1043B032B01D92D48F7E715F04005FA
:10CE8000F3D12046FFF700FE81462046FFF7FCFD68
:10CE90004FEA49060336804600EB96008000D7F83B
:10CEA00000A0F3F7E5F926F00306CAF808003044BD
:10CEB000CAF80C004D450DD10025454539682AD1E9
:10CEC0002046FFF7A9FE78600120F3F777F906B056
:10CED000BDE8F0872046FFF7D7FDC3074FEA5006AD
:10CEE00013D43046F3F7C4F9324601468246204651
:10CEF000FFF7BDFD2046FFF7B7FD31465046F4F77A
:10CF000015F806465046F3F7DBF93B689B6823F8B3
:10CF100015600135CEE72046CE68FFF7C3FD46F821
:10CF200025000135C9E700BF4BD00208F18F050885
:10CF3000FD8F05081FB50C46014601A817F0D6F96C
:10CF4000214601A8FFF768FF04B010BD024B8268BC
:10CF50001A61C268DA60704770040020838803F4A5
:10CF6000C071B1F5C07F02460FD0190604D5C37B4E
:10CF700000EB83021069704713F4807006D0D37BF6
:10CF800002EB83021369586870470148704700BF7D
:10CF90004182030870B5274CF3F76EFF002501238B
:10CFA000E561A4F80C32D4F810320BB1A4F80C529D
:10CFB000A4F8185203F0B4FF1F4B204E20486564BC
:10CFC000C4E90F3503211F4BA364C4F8005284F851
:10CFD000045203F029FD0121304603F025FDAA2269
:10CFE000BA21304603F02AFE00210846C4E9036650
:10CFF000C4E92C55C4E96955E566C4F8CC50C4F8B9
:10D00000B85005F05BFF0A21C4F83C0105F0CBFCE9
:10D0100040F2E261D4F83C0105F0C5FC002106F1C4
:10D02000440005F003FE40F21A7240F2DA63C4E9EC
:10D03000502370BD7004002030E80508CC040020A7
:10D04000BC04002008F605087047D0E902301847F4
:10D0500008B5074BD86E08B9064808BD002241F64E
:10D060009A01043001F05CFC0028F5D04068F4E738
:10D0700070040020F4FC0508034BC0000A4640F091
:10D080000201D86803F0DABD70040020034BC10030
:10D0900041F00201D86803F0DFBD00BF700400203A
:10D0A000034BC0000A4640F00201186903F0C6BDF8
:10D0B00070040020034BC10041F00201186903F025
:10D0C000CBBD00BF70040020F8B51C46930707468F
:10D0D0000E46154608D113689A88910615D5520652
:10D0E00010D5B3889B0501D52560F8BD50B9114B0B
:10D0F0009E4207D010490C2001F036FEC0E90165C0
:10D100002060F2E7C4E90057EFE70C4A934202D1EE
:10D110006B682360E9E70A4A9342E5D130B101F038
:10D120002FFE084B834214BF06463E466B68C4E997
:10D130000036DAE7ACED0508A0DE050890F6050834
:10D1400078F60508D8F6050800232DE9F041C2E974
:10D1500000330E460746144601F012FE0A2E05461D
:10D1600002D12060BDE8F081192E07D1838803F435
:10D17000C0731BB1144BC4E90037F3E76B7B5BB1A1
:10D1800005EB830322461B6931463846984763689E
:10D19000042BE7D100236360EB7C002BE2D005EB8E
:10D1A0008303F1001869002241F00201043001F00C
:10D1B000B7FB0028D6D04268234629463846BDE84A
:10D1C000F041FFF781BF00BF68FC0508F0B593B0E0
:10D1D000054668460E4617461C46F3F709F840B95F
:10D1E0003A4631462846FFF7AFFFF2F7D7FF13B0B4
:10D1F000F0BD002CFBD1019B044918680AF07AFBB2
:10D200000028F4D10198F3F70BF800BFECE605080D
:10D2100008B519B903F0F7FEF3F702F803F0F8FECA
:10D22000FAE70EB403B503AA52F8041B019203F007
:10D230001DFFF2F7F5FF000070B5124EC400054661
:10D24000306944F0020400222146043001F068FBFA
:10D250000246A0B9F06E30B12146043001F060FB07
:10D2600008B1406870BD00220748214601F058FB14
:10D27000024620B9054906482A46FFF7D2FF506802
:10D28000F0E700BF70040020A4F805080990050825
:10D29000F0E505080A4B10B50446D3E903039842AC
:10D2A00007D0E100002241F00201043001F038FB18
:10D2B00020B92046BDE81040FFF7BEBF406810BD52
:10D2C00070040020032837B505460C4607D10846F0
:10D2D00001F078FF00B30E24204603B030BDCA072A
:10D2E0002FD54B1008282AD801A252F820F000BFF1
:10D2F000D9D2020821D302083FD302083FD3020843
:10D3000015D302083FD30208D9D202081DD3020860
:10D31000D9D20208002BDED01E24DDE7002BDBDA99
:10D32000B3F1404F06D14FF0804003B0BDE830402C
:10D3300005F0FAB85B425B0043F00104CCE7DB4345
:10D34000F9E7062825D101F00703022B10D08B073F
:10D350001FD10B681A7BE2B103EB82031A69204BE1
:10D360009A4216D1486840B98B68C86801930CE0AE
:10D37000CC082046F3F788FE18B1400040F00104C5
:10D38000AAE701A92046F3F7A2FE0199F3F764FD8D
:10D39000F3E7204601F0F4FCC37ABBB100EB830055
:10D3A0002146036928469847B0B9042DB4D0A5F1A9
:10D3B0000803022B12D90B4B20465D5D01F0ECFCFB
:10D3C000094903462A460948FFF72BFF062DECD1F1
:10D3D000640044F001047FE704467DE700247BE716
:10D3E0007D5303082EF705081590050818E5050874
:10D3F0002DE9F04105460E461746984601F0C0FC5F
:10D40000847A54B100EB8404434624693A46314699
:10D410002846A446BDE8F0416047284601F0BCFC20
:10D42000024902460248FFF7FCFE00BF1E900508B5
:10D4300018E5050800231A461946FFF7D9BF000072
:10D44000F0B51546124A87B00C461169049106469C
:10D45000D168059102A80F49C2E90335F2F7A6FE8B
:10D460002246376831466846F6F7ECFEB4FA84F295
:10D47000520939466846F9F795FF044615B1FFF79A
:10D48000D9FF04460120F2F799FE204607B0F0BD0F
:10D49000700400204DCF020807B50022019101ABB6
:10D4A0000121FFF7A5FF03B05DF804FB30B4556818
:10D4B000003D144618BF0125C5F1020302EB8303AA
:10D4C0000A462918206830BCFFF792BF10B5044601
:10D4D00003F042FE30B1002320461A461946FFF7FA
:10D4E00087FF0446204603F051FE28B9BDE81040EE
:10D4F0000249034803F08CBD204610BD2490050866
:10D5000018E505087FB5114B0592C00040F00200F8
:10D510000190186902900620CDE90301D86E78B118
:10D52000002241F6CA01043001F0FAF940B1406826
:10D5300001AB00220521FFF75BFF07B05DF804FB9C
:10D5400001A905200BF0B2FAF7E700BF7004002034
:10D5500070B5164604460D46FFF7F6FD336893B9DD
:10D56000A30709D12268084B9A4205D1E2880749EE
:10D570002B460748FFF755FE204601F00DFC0549F4
:10D5800002462B46F5E770BDD8F60508459005081C
:10D59000ECE605084E90050807B56A46FFF7D8FF88
:10D5A000DDE9000109B102F043FC03B05DF804FBC2
:10D5B0002DE9FF41174606460C461D4601F0E0FBEB
:10D5C000374A904208D12B463A462146304604B0AD
:10D5D000BDE8F04104F066BB818811F4C07812D038
:10D5E000062C2DD12F4F00233B62FFF7B7FC0346DB
:10D5F000304698472860D8B93B6A002B18BF1C46B4
:10D600002C60002015E0062C1AD101AA1921304601
:10D61000FFF79AFD019B7BB901AA8A213046FFF7EB
:10D6200097FF039401AA00210120FFF73FFF286024
:10D63000012004B0BDE8F08101AA41464046F4E76C
:10D64000002CE9D1384601F09BFB17490AF052F94A
:10D6500001AA60B147213046FFF776FD019B73B107
:10D6600001AA21462046FFF721FF2860C9E79B2138
:10D670003046FFF769FD019B0BB10397D2E70B49D9
:10D68000384603F097FD30B109490A4803F0C0FC61
:10D6900028600220CDE73846FFF718FFF8E700BF03
:10D6A000E8E90508700400200CE80508A0E7050873
:10D6B00056900508A8E505087FB54FF4447102AA05
:10D6C0000546FFF741FD029CDCB1204601AA6946F0
:10D6D00001F0DCFC0024009BA34201D804B070BD23
:10D6E000019B53F8240007F0A1FD02AA014606465B
:10D6F0002846FFF72DFF02993046FFF7BDFC0134A5
:10D70000E9E7284602AA40F21631FFF721FF029D01
:10D71000AB68A342E2D9EB6853F83400E60080B16D
:10D7200004280ED007F09AFD03785F2B09D0EB6830
:10D7300053F8340007F07AFDEB6833445968FFF77B
:10D740009BFC0134E4E7000073B505460C46164621
:10D7500001F016FB437B5BB10422CDE9002600EB10
:10D7600083022146136928466A469847009B43B1C5
:10D77000284601F011FB0449024623460348FFF7FF
:10D7800050FD02B070BD00BF4E900508ECE60508E4
:10D7900073B50C46064601F0F3FA83881906054670
:10D7A00032D4C37BB3B14CB900EB83031A69174B76
:10D7B0009A4203D01020F2F75BFD0446EB7BAA8867
:10D7C00005EB8303D2051B69214648BF1B68304621
:10D7D000984778B96A460F213046FFF7B5FC009BA1
:10D7E00053B11CB91020F2F743FD044621466846A8
:10D7F00004F048FB02B070BD304601F0CDFA044998
:10D8000002460448FFF70DFD3046F3E7816D03083B
:10D810006D90050818E5050837B5044601F0B0FA23
:10D82000818811F4C0750AD0104B00221A62FFF7EC
:10D8300095FB0346204603B0BDE8304018476A46D2
:10D8400019212046FFF780FC009B3BB9204601F0E0
:10D85000A3FA074902460748FFF7E3FC6A46294650
:10D860002846FFF723FE03B030BD00BF7004002040
:10D870007A90050818E5050830B5054695B000F022
:10D8800051FF284601F07CFA848814F4C0740AD051
:10D890001B4B00221A62FFF761FB0346284615B0B6
:10D8A000BDE8304018476A4619212846FFF74CFC6E
:10D8B000009BE3B102A8F2F79BFC014640B96A461F
:10D8C000FFF7F4FD0446F2F769FC204615B030BDC1
:10D8D000039B0C4918680AF00DF80346039823B11E
:10D8E00003F062FB064B1862EFE7F2F799FC28465B
:10D8F00001F052FA044902460448FFF792FC00BFC7
:10D9000070040020A0E705087A90050818E50508CE
:10D910002DE9F04F8DB0136802930446002857D1CB
:10D9200002F10408C1F307294FEA4903CFB253FAC1
:10D9300081F14FEA810B58F8216076105ED13546AF
:10D94000BB00039308EB8703009308EB0B030193E1
:10D9500008EB870A4FF0000B019B9A4552D1D9443E
:10D960004FEA490B07F1010A002E5FD10BEB0A05C4
:10D97000A800F2F77DFC814614B1046057460126E9
:10D98000039A414609EB86001CF06AF83C46A34422
:10D99000AB4506D948464FEA8B01F2F784FC5D4659
:10D9A0008146DFF804A22646DDE90032934240F0CA
:10D9B0008A80321B21464B4652080298FFF718FD19
:10D9C00004464846F2F77CFC20460DB0BDE8F08FD7
:10D9D000546802F10808A5E726FA0AF3D80708D523
:10D9E00058F82A0001F0D0FB18B101F0A7FA01386D
:10D9F00005440AF1010A5745EED1A1E74FF0000AAC
:10DA00005546F8E7DAF800206AB9DAF8040050B1B0
:10DA1000810708D1026864498A4204D103F00BF9F6
:10DA20000BF1FF3B83440AF1080A95E755445D4436
:10DA3000A800F2F71DFC81460CB1046001244FF0F0
:10DA4000000A5745A3D026FA0AF3DA0758F82A0045
:10DA500035D5830716D10368544A934202D0544AFD
:10DA600093420FD108AA07A901F010FB079A089961
:10DA700009EB840092001BF0F3FF079B1C440AF1A2
:10DA8000010ADEE708A9FFF783FEA7EB0A0303906C
:10DA900004930398FFF7F0FE03460028EFD0049AA2
:10DAA0002244954207D8E90048460593F2F7FBFB6C
:10DAB000059B81466D0049F824300134E9E749F8B7
:10DAC00024000134DBE7009BD3E9002B002A62D15C
:10DAD0001BF0030726D1DBF80030534522D1DBF8D9
:10DAE00008309F4203D3009B083300935CE7DBF8C8
:10DAF0000C3053F837004FEAC70888B104280FD01C
:10DB000000F00703022B01D008F0A2FB49F8260021
:10DB1000DBF80C30B20043444A445B685360023681
:10DB20000137DCE708AA6A215846FFF711FD0021FA
:10DB300008AA0846FFF7BAFC0021FFF729FE039068
:10DB40000398FFF799FE07460028CCD0731CAB4220
:10DB500007D3E9004846F2F7A6FB4FEA450881469D
:10DB6000454607F00703022B03D0384608F070FB48
:10DB7000074608AA0F215846FFF7EAFC08AA002129
:10DB800001200A97FFF792FCB3004B4449F8267036
:10DB900002365860D4E7B3004B4449F826200236D9
:10DBA000C3F804B09FE700BF0CE4050844F605087D
:10DBB00024EC050870B5830786B00C4615461BD1CA
:10DBC00003681D4A934202D01C4A934214D102AA10
:10DBD00001A901F05BFA019BA34227D319D8029B4C
:10DBE000043D03EB84049C4201D106B070BD54F89F
:10DBF000042D45F8042FF6E702A9FFF7C9FD00231D
:10DC000006469C420193304606D8FFF735FE0028B1
:10DC1000EBD00B4922460BE0FFF72EFE019B28B10B
:10DC2000E21A013A013345F82200EAE7019A054970
:10DC30000548FFF7F6FA00BF44F6050824EC05088E
:10DC40009D90050888900508D0E405082DE9FF415E
:10DC500083071546CFB2C1F3072436D10368384A8B
:10DC6000934202D0374A93422FD10290029803AADE
:10DC700001A901F00BFA01983B1983425AD8039984
:10DC8000002601EB8003A64214D1C01B01EB8701E3
:10DC9000801B05F013F9039945F82600BC0005EB3D
:10DCA00086080B1942468B420AD10023029304B026
:10DCB000BDE8F08153F8042D45F826200136E2E74F
:10DCC00053F8040D42F8040FEDE70021FFF760FD63
:10DCD000002380469F42019317D80021084605F093
:10DCE000EDF806464046FFF7C7FD0146C0B9B368E8
:10DCF000A3421FD345F8246005EB840205EB8301A2
:10DD0000AA4211D11B1BB360D1E74046FFF7B4FD17
:10DD1000019B78B1FA1A2244013345F82200D9E771
:10DD2000304604F040FEDDE7F768881A385842F8BC
:10DD3000040DE5E7019A04490448FFF772FA00BFB1
:10DD400044F6050824EC050888900508D0E4050889
:10DD50002DE9F04F85B000AF07F1080205460C46EB
:10DD6000FFF7F2F9D7E9020129B102F061F814379F
:10DD7000BD46BDE8F08F0028F9D107F1080240F256
:10DD80001A312846FFF7E0F9BB6823B91E491F483E
:10DD90002246FFF746FA07F1080228461721FFF747
:10DDA000D3F9391DB86807F0C7FA82462046F3F761
:10DDB00077F9D7F8049009F101068519EB1D23F0D6
:10DDC0000703ADEB030D6B464A4651464FEAD30BB2
:10DDD00068461BF045FE2E2309F83B302046F3F73A
:10DDE0006AF981462046F3F75BF96E4402464946DC
:10DDF00030461BF035FE29466846F3F797F80122B6
:10DE00001E21FFF77FFBB2E7BA900508A4E60508DC
:10DE100008B50446F2F72EFB18B104490448FFF791
:10DE2000F7F9044902482246FFF7FBF9C0900508BC
:10DE300014E60508E7900508014608B50148FFF714
:10DE4000E7F900BFD0E405082DE9F043831E87B051
:10DE5000054688461746062B3BD8DFE803F0093A0B
:10DE60003A093A040F00B94212D04FF00E09ECE023
:10DE70003A4607B0BDE8F04301F0CCB9384603F0AC
:10DE80006BF940B13946404603F094F90028ECD0D4
:10DE90004FF01E09D9E017F0030440F000813A6802
:10DEA000A14B9A4240F0FB8007F104097B68A34232
:10DEB000DBD959F8046F304603F04EF9002800F022
:10DEC0005D813146404603F075F90028E0D1013408
:10DED000ECE711F0010F00F0FF804E10F90740F160
:10DEE000CE807C10232800F2DA80DFE800F0B2B6A2
:10DEF000D8BABED8D8D8D8121D20233D46484AD813
:10DF000050586A72121D20233D46484AD850586A1C
:10DF1000729446EA040090EA40034FEA400900F197
:10DF2000A88049F0010990E086EA0400F3E706EAD8
:10DF30000400F0E7002C02DA7C48FFF77DFF1F2C7D
:10DF400009DC6FF040432341B34204DB4FF0404310
:10DF50002341B34205DD3046F11704F0D5FA80467F
:10DF6000C0E006FA04F0D6E7002CE5DB1F2C2046C3
:10DF7000A8BF1F2046FA00F0CDE73019CBE7301BD1
:10DF8000C9E786FB0404B4EBE07FC4D0E3E7002CD0
:10DF900000F0F680214630460DF050FFBBE7002C24
:10DFA00000F0EE8007EE906AB8EEE70A07EE904ABE
:10DFB000F8EEE77A80EE270A07B0BDE8F04303F0F9
:10DFC000FDB9002C00F0DC80214630460DF028FF22
:10DFD000A1E7002C1CDA07EE906AB8EEE70A394692
:10DFE00007B0BDE8F04303F055BA33460120E2071D
:10DFF00006D580FB0302B2EBE07FACD1012C8AD0C6
:10E0000083FB0332B2EBE37F4FEA6404EFD0A2E775
:10E01000EBD101207FE7002C00F0B280002102202C
:10E0200008F084FC2146814630460DF007FF400091
:10E0300040F00100C9F80800214630460DF0F0FE1E
:10E04000400040F00100C9F80C00484607B0BDE8A8
:10E05000F083A642FFF61CAF07E7A6423FF718AFD2
:10E0600003E7A6427FF714AFFFE6A642BFF610AF64
:10E07000FBE6C11707B0BDE8F04304F045BABB07A3
:10E080002AD13B682A4A934219D107EE906A394651
:10E09000B8EEE70A03F0FEF981460028D5D1254BFA
:10E0A00040465D5D00F078FE0446384600F074FEA0
:10E0B00021490090234621482A46FFF7B2F8204A1A
:10E0C000934209D107EE906ADFED1E0AB8EEE70A27
:10E0D000394602F049F8DFE7062D03D143462425EF
:10E0E000B8461F46404600F04BFE037B33B9A5F10E
:10E0F00009030C2B0DD80D35EDB2F3E700EB8300CF
:10E100003A46036941462846984781460028EED0A2
:10E110009BE7A5F116030C2B16D843460F35B846DE
:10E12000EDB21F46DEE700BF44F60508159105086D
:10E13000B4E80508FCF605082A91050818E5050865
:10E1400020E2050800000000242D04D943460F3DBD
:10E15000B846EDB21F46242DA1D102A94046FFF7D3
:10E1600017FB04462046FFF787FB00283FF47DAEEF
:10E17000394601F0C7F80028F4D089E637468EE723
:10E1800001490248FFF744F83D91050834E70508C6
:10E19000014608B50148FFF73BF800BF18E5050840
:10E1A0002DE9F041044617461E460D4641B1186858
:10E1B00000F0E6FD6368834202D00548FFF7E8FF00
:10E1C000A06833463A462946BDE8F041FFF710B94A
:10E1D00049910508014608B50148FFF719F800BF45
:10E1E00084E5050807B50022019101AB012102F089
:10E1F0002BFEF2F715F80000014608B5024809B9F0
:10E20000FFF706F8FFF7EEFFA0E7050808B500F0F6
:10E21000C3FD024902460248FFF703F84F91050883
:10E2200018E50508410008B5024841F00101FFF773
:10E23000D9FF00BFCCE5050808B5024842F2A201AB
:10E24000FFF7D0FFA8E5050830B593B0044668464F
:10E250000D46F1F7CDFF48B920462946FFF71CF9D6
:10E260000446F1F79BFF204613B030BD01990248E8
:10E2700000F0C0FD0024F6E714D40508054BD86172
:10E28000B3F80C2212B2012A04BF0022A3F80C2218
:10E29000704700BF70040020EFF3108172B6084A87
:10E2A000B2F80C321B0443BFB2F80C3203F1FF3357
:10E2B0001BB24FF6FF73A2F80C3281F3108870473F
:10E2C00070040020EFF3108172B60C4BB3F80C22EF
:10E2D000013212B2A3F80C2252B9DA692AB9D3F882
:10E2E000102212B993F818222AB10022A3F80C22A6
:10E2F00081F3108870470122F8E700BF7004002006
:10E3000070B5EFF3108572B60F4B93F81822082AF8
:10E3100018D0B3F80C4224B2012C04BF0024A3F897
:10E320000C4293F81942561C224402F0070228328C
:10E3300083F8186203EBC203C3E90201012085F3ED
:10E34000108870BD0020FAE7700400200228F8B59C
:10E350002C4C034610D0E26972B1EFF3108272B612
:10E36000E06938B10021012BE16103D182F310880B
:10E37000F1F756FF82F31088B4F80C321BB243B9A0
:10E38000EFF3108272B6B4F80C6236B216B182F3B3
:10E390001088F8BDD4F814724FF6FF73A4F80C324D
:10E3A00097B1D4F810526B68C4F810320BB9C4F8A6
:10E3B00014322B682E6082F3108828469847EFF3BA
:10E3C000108272B6AF42ECD194F81852BDB194F8F5
:10E3D000193203F12801013304EBC10103F00703F3
:10E3E000013DD1E9020184F8193284F8185282F310
:10E3F0001088FFF729FFBDE8F840FFF763BF82F3FD
:10E400001088F8E7700400200120FFF79FBF08B5CF
:10E41000FFF7FAFF30BF08BD08B5FFF7F5FF30BFC3
:10E4200008BD000038B1044A1369984202D0106157
:10E4300018467047002070477004002001F00F015B
:10E4400008290DD8DFE801F011050A0C0C0C0C0CA2
:10E450000E0000280CBF0E201E20704704F064B888
:10E4600004F07DB8C00040F00200704708B500F02D
:10E47000BBFD10EE100A27F07BFD41EC100B08BD30
:10E4800000F0B2BD08B551EC100B27F0C9FDBDE896
:10E49000084000EE100A02F091BF02F08FBF0000AA
:10E4A000F0B593B00546684616680F461446F1F776
:10E4B0009FFE78B9002E0CBF394600212346324614
:10E4C0002846FFF775F80546F1F768FE012D0CD1D7
:10E4D000284612E0019B23601049206802F06AFE82
:10E4E000034620685BB9F1F79BFE2368002DF3D14A
:10E4F0000BB90623236036B9002013B0F0BD02F03B
:10E5000053FD2060F7E70649304602F053FE00282D
:10E51000F2D03046FEF7DAFFE5E700BFA0E70508D6
:10E520000CE80508036803B94068FFF7A5B913466E
:10E53000C1F30722C9B2FEF75BBF1FB501F00F039D
:10E54000012B04460CD011F00E0F0BD0023B012B17
:10E550000AD9012201A900F01DFF50B1019801E084
:10E5600000F030FE04B010BD04B0BDE8104000F073
:10E57000F1BC204600F0EEFCF4E708B528B106280F
:10E5800003D0FEF7A3FFF1F74BFE08BD10B50C4614
:10E5900019B9BDE81040FFF7FBB8FFF7F9F884425E
:10E5A0001CBF0023C4E90030002010BD40F26243CC
:10E5B000984217D840F25E43984209D85E281DD091
:10E5C00075281DD03E2814BF4FF0FF300120704742
:10E5D000A0F58C60022815D8DFE800F00C0E0200D0
:10E5E0000520704740F2EA43984214BF4FF0FF30D5
:10E5F00003207047062070470720704702207047AD
:10E60000002070470420704738B5034614460D4675
:10E6100061B152B111462846984760B16B683BB969
:10E620006C6045F00103AC60E3602C46204638BDC9
:10E63000AB68DC60F5E76368EB606560002BF5D1E3
:10E6400044F00103A560EB60F0E7F8B5064631B190
:10E65000002511F0010304D00023EB602946084691
:10E66000F8BDCC68CB6014F0010307D1E768E36024
:10E6700022463046FFF7C8FF3C4601460A46304670
:10E680002946FFF7C1FF21460546E2E78A422DE908
:10E69000F04184460F4606D1002351685360BDE81F
:10E6A000F041FFF7D2BFD66896B11446E468E3079D
:10E6B000FCD524F0010451686368934206F0010818
:10E6C00016D1002339B9984518BF1E466660D1603F
:10E6D0003846BDE8F0815360D3606046FFF7B5FF70
:10E6E00005466060EE60B8F1000FF1D0A560EFE77D
:10E6F0001D46DB689342FBD100225A60DA60604617
:10E70000FFF7A3FF0028EDD0E8600546EAE7000028
:10E71000034B82B0186801ABC01A02B0704700BF4B
:10E720007004002007B5064A1368526801A95B1AF5
:10E730009A4201D8FFF780FD03B05DF804FB00BFEB
:10E740007004002010B503461446500CC2F34F026B
:10E7500021B1E10702D40C48FFF71AFD904206D11F
:10E7600098420FD0094902460948FEF75AFD9842DF
:10E7700004D9C21A07490648FEF753FD9A4201D24E
:10E780000549F1E710BD00BF5691050860910508E5
:10E7900018E50508729105087A9105082DE9F74FEB
:10E7A000DDE90CA7002406468B4615460193A046DA
:10E7B000A146019B9C4204D1B1453CD22248FFF7BF
:10E7C000E7FCB44210D2BAF802209205F6D45BF806
:10E7D000240009F101099AF80220012A24D100F04D
:10E7E000F1FC07F8240017E0BAF80010C900002275
:10E7F00041F00201284600F093F888B9BAF80220E7
:10E80000D30505D5BAF8002010491148FEF709FDD7
:10E81000DAF8042047F8242001340AF1080AC8E78E
:10E82000406808F10108D6E7022A01D100F086FB12
:10E8300047F82400F0E72B68B8EBD30F01D2054866
:10E84000BDE703B0BDE8F08F8C91050887910508FE
:10E8500018E505089691050870B586B0044615467A
:10E8600002EB800203A81E4600F031F80B9B0193D7
:10E870000A9B009303AA334629462046FFF78EFFE2
:10E8800006B070BD08B50148FFF7A4FCA0910508CB
:10E8900007490346002231F8020B984206D20132A2
:10E8A000222AF8D103EB530343F00100704700BF65
:10E8B0001CE0050810B50446416019B90123A160A8
:10E8C000236010BDC800F1F7ECFC0146F6E741609B
:10E8D000C90041F0070101608260704703789B071F
:10E8E00010B5044602D48068F1F7EAFC23680022E0
:10E8F00062F3DF036260236010BD03789B0710B5ED
:10E90000044602D48068F1F7DBFC236803F00403BB
:10E9100043F0010323600023C4E9013310BD00006C
:10E920002DE9F04F022A85B004460E46904612D0DB
:10E93000426882B1904BC1F386010B4493F81A32BE
:10E94000B3FBF2F102FB1133826802EBC30552F80C
:10E950003330B34213D0237813F00102019213D065
:10E9600006F00702022A0FD016F0030203D1306826
:10E970008249884207D0B8F1010F05D0002528460A
:10E9800005B0BDE8F08F01925B076AD52768A568DE
:10E9900027F007072F44BD4232D3B8F1010FEDD164
:10E9A000D4E90032B2EBD30FC3F3DC0111D104314F
:10E9B0006160A068C900F1F776FCD4E90032A2EBEF
:10E9C000D30223F00703A060D200002118441BF0FB
:10E9D0008BF82368A168C3F3DC02501C01EBC2056D
:10E9E00060F3DF03236041F83260002206F007067F
:10E9F0006A60022EC3D0237862F300032370BEE75F
:10EA00002868B04224D1B8F1020F17D12368D5F895
:10EA10000480083B7A1B05F108012360083A284668
:10EA20001BF04EF82568A368C5F3DC0225F0070546
:10EA30001D44002143F83210C5F804804E4BC6F344
:10EA400086061E44A368EB1ADB1086F81A3296E796
:10EA5000019B23B9314600F055FC0028D3D108357D
:10EA600099E763682BB9B8F1010F87D1204600F010
:10EA700087F806F0070BBBF1020F2BD1F008F2F775
:10EA800003FB81466368B9FBF3F203FB129A574616
:10EA90000025A26852F83700FB00029302EBC7037F
:10EAA000F8B9B8F1010F7FF469AF2268C2F3DC0155
:10EAB0000131002D18BF2B4661F3DF02BBF1020FBD
:10EAC0002260C3E9006003D0227860F30002227064
:10EAD0001D4654E731460620FEF7F4FB4FEA600975
:10EAE000D0E7042819D1002D08BF1D4663680137FF
:10EAF000B7FBF3F203FB1277BA45CAD1B8F1010FA5
:10EB00007FF43CAF002D32D023680022083323600D
:10EB1000BBF1020F2E606A606CE7B04218D1B8F109
:10EB2000020F0ED12168606808392160791CB1FBA1
:10EB3000F0F500FB1511A06850F83110A9B9F800E4
:10EB400011500D4AC6F38606164486F81A72BFE7BE
:10EB500001990029CAD13146CDE9023200F0D2FB39
:10EB6000DDE902320028C1D0D9E70421E7E72046D9
:10EB700000F006F886E700BF70040020FCF40508EA
:10EB80002DE9F04146680446701CFFF781FE0546FA
:10EB9000C000A768F1F785FB2368656003F00603F2
:10EBA00043F001032360A0603D1D4FF00008B04515
:10EBB00004D13846BDE8F041F1F782BB55F8041C9A
:10EBC00039B1042905D001222046FFF7A9FE2B68A0
:10EBD000436008F101080835E9E710B50023044651
:10EBE000016043608800F1F75CFBA06010BD036822
:10EBF0002DE9F74F04460F46934623B912F0010F53
:10EC000065D000F067F839460620FEF75BFB4FEA57
:10EC1000600A2368BAFBF3F603FB16A635464FF0ED
:10EC20000008A16851F82590AA0001EB8503B9F10D
:10EC3000000F0CD11BF0010F49D06268B8F1000F32
:10EC400018BF4346013262601F60B94633E0B9F134
:10EC5000040F17D1B8F1000F08BF9846236801359B
:10EC6000B5FBF3F203FB1255AE42DAD11BF0010FF4
:10EC70002DD0B8F1000F26D0636801336360C8F867
:10EC80000070E2E739464846019200F03BFB019AEA
:10EC90000028E3D01BF0020F0DD063682068A16844
:10ECA000013B63606B1CB3FBF0F400FB143351F8C1
:10ECB000233023B98B50484603B0BDE8F08F0423BE
:10ECC00041F82530F7E7204600F004F8A1E74FF0BF
:10ECD0000009F0E7F8B5076886680446781CFFF776
:10ECE000D7FD0025206065608000F1F7DAFAA060AA
:10ECF000BD4204D13046BDE8F840F1F7E1BA56F81C
:10ED0000251029B1042903D001222046FFF76FFF07
:10ED10000135EDE770B5016802460023994201D143
:10ED2000002015E0946854F823009E000133002869
:10ED3000F4D00428F2D05568013D5560B3FBF1F2E0
:10ED400001FB123354F82330002B18BF0423A351C6
:10ED500070BD10B504468068F1F7B2FA0023C4E92B
:10ED60000033A36010BD704710B50C46F1F780FA70
:10ED7000046010BD10B50C46F1F788FA046010BDB0
:10ED800083070FBF0068034B00F00F0053F820000B
:10ED9000704700BF60E0050808B5FFF7F1FFBDE868
:10EDA0000840C088F2F787B970B50D46044616468C
:10EDB000FFF7B8FC2846FFF7E3FF437A43B100EBC7
:10EDC00083033246294620461B69BDE87040184738
:10EDD000C28803492046BDE87040F2F707BF00BF74
:10EDE000C59105080A4601460148FFF7DDBF00BF8F
:10EDF00064040608F7B5044608460E4602F0C6F954
:10EE000070B101AA6946304602F022FA009B3BB17C
:10EE100016492046F2F731FB009D033D002D0BDA29
:10EE2000314620460222FFF7BFFF1149204603B0BA
:10EE3000BDE8F040F2F721BB019A0E4902EB8503D1
:10EE400020465B6852F82520F2F7D0FE019BAF0008
:10EE50003B449A6822B906492046F2F70EFBDCE7EC
:10EE600005492046F2F7C2FED7E700BFCA91050860
:10EE700094A70508EE9105080392050808B5024617
:10EE8000FFF77EFF837A53B100EB830306491B69CA
:10EE90008B4204D1BDE80840104608F0FFBC181EA4
:10EEA00018BF012008BD00BFC1760308830713B552
:10EEB000044603D102680D4B9A4208D0214608202F
:10EEC000FEF700FA10B92046FFF7A0F9044614F047
:10EED000010103D06010E11702B010BD6B4608229B
:10EEE000204603F049FADDE90001F5E70CEB0508DF
:10EEF0000E2838B503460C4604D1002323600125B3
:10EF0000284638BD1E2801D10123F7E710F001057E
:10EF100001D04310F2E7820707D10168064A914207
:10EF200003D103F045FB2060E9E719460820FEF70E
:10EF3000C9F90028F5D1E3E70CEB050813B501A9E1
:10EF40000446FFF7D5FF10B92046FFF75FF9019897
:10EF500002B010BDC20705D4830705D10268034B78
:10EF60009A4201D103F01DBBFFF7E8BF0CEB050887
:10EF70000E2838B503460C4629D01E282AD010F09A
:10EF8000010508D0431000EE103AB8EEC00A84ED37
:10EF9000000A012519E081070CD102680F498A4255
:10EFA00002D103F04FFCF2E70D498A4202D102F090
:10EFB0006DFAECE719460920FEF784F928B18207BB
:10EFC00003D10268064B9A42F1D0284638BD9FED26
:10EFD000050ADCE7B7EE000AD9E700BF0CEB05082D
:10EFE000B4E805080000000013B501A90446FFF7C6
:10EFF000BFFF38B92046FFF7CFFE04490246044858
:10F00000FEF70FF99DED010A02B010BD0C92050844
:10F0100018E50508F8B504460F461646FFF7A8FFA1
:10F02000054620B10023336001252846F8BDA1071D
:10F0300009D122680B4B9A4205D132463946204607
:10F0400001F08CF8F0E721460A20FEF73BF9002892
:10F05000EBD08207E9D10268024B9A42E5D13246F1
:10F060003946EDE720E2050810B50446FFF7D2FF68
:10F0700038B92046FFF790FE024902460248FEF7E3
:10F08000D0F810BD1792050818E50508830710B5DC
:10F090000FD103680A4CA34204D143680B600830C7
:10F0A000106010BD074CA34203D183680B60C06899
:10F0B000F6E7FFF771FE044902460448FEF7B1F88F
:10F0C00044F6050824EC05081E92050818E5050815
:10F0D00013B50C4601A9FFF7D9FF019BA34204D049
:10F0E000034904482246FEF79CF802B010BD00BF59
:10F0F00027920508D0E40508F7B51F46D307064652
:10F100000D4614460DD5541001940198002823DAB9
:10F110002844B7B100281DDBA84228BF284603B009
:10F12000F0BD01A91046FFF7E3FE0028EDD120460F
:10F13000F588FFF731FE0A4903462A460948FEF7DB
:10F1400070F8002801DBA842E9D3F2880649074895
:10F15000FEF767F80020E2E7002FDDD1F3E700BFFC
:10F160003992050818E50508509205085CE605087F
:10F17000820701D003F0D8B9002801DA03F0EFB913
:10F18000400040F001007047830710B5014608D1E8
:10F1900002680B4B9A4204D18068400040F00100A5
:10F1A00010BD0846FFF7ECFDC37A33B100EB8300D6
:10F1B000BDE810400369052018471846F0E700BF76
:10F1C000CCF405080E2810B5044620D01E281CD00B
:10F1D00006281CD0C20703D5013818BF01200EE055
:10F1E000FFF7CEFDC37A5BB100EB830021460369D4
:10F1F0000420984720B1A0F11E035842584110BD89
:10F200002046FFF7C1FF0138E7E70120F7E70020BC
:10F21000F5E7000005282DE9F04707BF4FF00E087D
:10F220004FF01E094FF01E084FF00E09914207469D
:10F230000C46154607D1C8075FD40846FFF7A0FD66
:10F240008388590759D504F00703022B05D0A2077C
:10F2500017D122682A4B9A4213D105F00703022BDB
:10F2600005D0AB0712D12A68254B9A420ED1294608
:10F27000204605F094FF00283FD14B461846BDE8D4
:10F28000F08714F0010623D0EE07F6D401262846B5
:10F29000FFF776FD027B82465AB38188080704D4C3
:10F2A0002046FFF76DFD824523D1052F14D09AF833
:10F2B0000C300AEB830322461B692946022098473B
:10F2C0000346B0B1022FD9D0FFF77CFFD3E7012668
:10F2D0002B4625461C46DAE7CB06E8D50AEB820228
:10F2E0002946136938462246984703460028DED04F
:10F2F000C4E7002EEBD0AC42BFD14346BEE700BF0F
:10F30000FCF4050808B50A4601460220FFF782FF13
:10F31000BDE80840FFF756BF10B50446FFF734FFBD
:10F3200038B92046FFF738FD024902460248FDF78A
:10F3300078FF10BD5792050818E5050838B5044652
:10F34000FFF71EFD837B15462BB100EB830003699D
:10F3500020469847A0B9204635B9FFF71DFD094959
:10F3600002460948FDF75DFF042D04D1FFF714FDA7
:10F3700006490246F5E7FFF70FFD05490246F0E7AB
:10F3800038BD00BF6492050818E505087E9205089F
:10F390009092050838B50546FFF7F2FC037C144649
:10F3A0001BB914F004000BD138BD00EB830302F04D
:10F3B00003021B69284698470028F2D10120F3E791
:10F3C0000148FEF7E5FE00BFA2920508042803D01D
:10F3D000052807D0002070478B68002B0CBF0E203B
:10F3E0001E2070478868400040F001007047000010
:10F3F000084A0346C1E900230022C1E90222084667
:10F40000054A1968914202BF5B68C3F31723836002
:10F41000704700BFA8E00508F4E00508F8B50D4600
:10F420000179044601F07F0116464020002208F0D1
:10F4300017FFA268E36827682B6042436A6022795D
:10F4400002F07F01A96009498F4201D00020F8BD78
:10F45000110601D4B20706D46268C2F3172200FB7A
:10F4600002332B60F2E70120F1E700BFF4E005086A
:10F47000F8B5002205460E460146402008F0F0FE91
:10F4800007461020F0F7F4FE094A0A4B0571012DDA
:10F4900008BF13460360436803F0FF030446C0E956
:10F4A000013606FB07F0F0F7E3FEE0602046F8BD0A
:10F4B00034E10508C0E005084268C36891688B42E2
:10F4C00030B40AD21479D16882685D1CC5601A44D0
:10F4D00004F07F0030BC08F037BF002030BC70471C
:10F4E0004368FF2B70B504460E461AD801790022F6
:10F4F000402008F0B5FEA168083105464143E068A8
:10F50000F0F7D1FE6368E060082262F31F236360B6
:10F51000A36803FB0553C5EBC502002118441AF08C
:10F52000E3FA20793346D4E9022109F049F9A368C6
:10F530000133A3606368A3F580736360062070BD28
:10F5400070B50E79012E05460C460ED11949F1F71A
:10F5500094FFD4E902213346284605F0BBF828463B
:10F560001549BDE87040F1F788BF14493246F2F7FB
:10F570003DFBA368002BF2D011492846F1F77DFF2F
:10F580000026A368B34204D80E492846F1F775FF58
:10F59000E5E71EB10C492846F1F76FFF3246E168F6
:10F5A000207908F0D1FE012201462846FFF7FCFB36
:10F5B0000136E6E7B092050878AE0508BC9205086A
:10F5C000C7920508A0A60508CB9205082DE9F04FC3
:10F5D000044689B00D4616460AB90025DDE011F053
:10F5E00003078068DFF844A240F0EC800B68874A8C
:10F5F000934240F0E78002AA08F0C6FA10B98448A6
:10F60000FEF7E8FD2179042E01F07F013A464FF024
:10F61000400000F0A38008F023FE16F00302054628
:10F6200062D131688B7B002B4FD001EB83031869CB
:10F63000784B984249D13179402001F07F0108F0A0
:10F640000FFEA84202D07448FEF7F6FB336853451C
:10F65000D6E9029B45D17368C3F3172805FB08F868
:10F66000DDE902032268E7681B1A5245A9EB03068D
:10F670003CD194F90420002AAFDA002EE3D162686D
:10F68000C2F3172205FB027705FB09F20BEB080119
:10F6900005FB007001931AF013FA0399A26802980F
:10F6A000521A48446A4305FB017105FB00701AF0C9
:10F6B00007FA019BA068A3EB090230446A430021CA
:10F6C00005FB00701AF010FA3BE0544B99420BD145
:10F6D000012DB8D1052205A93046FFF75BFEDDE913
:10F6E00005B94FF00008BBE74D4889E7002ECBDD98
:10F6F0006368B6EB132F2FD9A168314469433846AC
:10F70000F0F7D1FD6368E06066F31F238246636013
:10F71000BB4508BF83460298A26803994844324417
:10F72000121A6A4301FB05A105FB00A01AF0C8F9F3
:10F73000029805FB09F20BEB080100FB05A01AF08B
:10F74000BFF96368C6EB132262F31F236360A368EB
:10F750003344A360062520E0BA46DCE708F080FDCC
:10F760002268029B524506461BD1B3F1807F03DB22
:10F770002C492D48FDF74CFD1020F0F779FD05468A
:10F7800094E80F0085E80F00029A02EB112363F35F
:10F790001F216960039B9B1AAB60284609B0BDE836
:10F7A000F08F03992079C91AFFF762FEDDE9023272
:10F7B000E168D21A0546724306FB0311C0681AF0CD
:10F7C0004FF9EAE700232A4601462068FFF794FC38
:10F7D00023685345024620790ED16368042E02EB5C
:10F7E00013220BD003067FF5F8AEE168334600F034
:10F7F0007F0008F0E5FFADE7042EF6D1E16800F0E8
:10F800007F0009B0BDE8F04F08F09EBDF4F1050897
:10F81000CE920508CDF50208F2920508CCF4050851
:10F820000D9305082893050858E70508F4E0050836
:10F830002DE9F043012885B007460E4608D08B0716
:10F8400024D10B68254A934202D0254A93421DD108
:10F85000012201A93046FFF79DFDB8B100223946CB
:10F86000402008F0FDFC029EB6FBF0F6054631464E
:10F870003846FFF7FDFD0199044606FB05F2C06816
:10F880001AF0EEF8204605B0BDE8F0833046FFF7E9
:10F890007BFC054600B1451029463846FFF7E8FDD8
:10F8A000002104463046FDF773FF4FF0000806467E
:10F8B0003046FDF7E1FF03460028E3D025B919469D
:10F8C0002046FFF70DFEF3E74246E16808F1010923
:10F8D000384608F075FFC846EAE700BFCCF40508D3
:10F8E00034E1050838B50C462046114606221D466F
:10F8F000FEF728FF2CB92146BDE838400120FFF76C
:10F90000B7BD2968CA0705D48B0708D10B680C4A14
:10F9100093420DD10846FFF711FB0146ECE701F0D9
:10F920000703022B07D1012C05D10648FEF730FC56
:10F93000054A9342F6E7BDE838400120FFF778BF5B
:10F940000CEB05083D930508FCF4050838B50D4699
:10F950001C4611462846094AFEF7F4FE206805F0C9
:10F960007DFC012D007804D1BDE838400021FFF76F
:10F970007FBD6168BDE83840FFF75ABF0400020050
:10F98000F0B50F4685B001A9044601223846FFF7BD
:10F9900001FD014678B93846FDF7FAFE05462846CE
:10F9A000FDF76AFF014610B9062005B0F0BD2046FC
:10F9B000FFF796FDF3E700222179402008F050FC84
:10F9C0006368029DB5FBF0F5B5EB132F0646C3F354
:10F9D00017221ED9A16829444143E068F0F763FC6F
:10F9E0006368E06003F0FF03BC42636004D105225A
:10F9F00001A92046FFF7CEFCD4E90203019900FBE0
:10FA0000063005FB06F21AF02BF8A3682B44A3601E
:10FA1000CAE7521B62F31F236360EDE7F0B51B28B2
:10FA20008DB006460C46154626D005D804286BD95D
:10FA30000E2850D000244BE02428FBD1012203A93A
:10FA40002846FFF7A7FC00284ED0A1075AD122680C
:10FA5000474B9A4256D1012209A92046FFF7DEFC06
:10FA600001230093DDE90901DDE9032304F0F8FE39
:10FA7000002847D01E242BE00A683E4B9A42D9D07A
:10FA8000012206A92046FFF7C9FC052209A928463C
:10FA9000FFF780FC9DF8207000223946402008F0D6
:10FAA000DFFBA1680A9EB6FBF0F6054631443846F6
:10FAB000FFF7DEFC079F069904463A46C06819F036
:10FAC000CFFFE068099906FB05F2384419F0C8FF3A
:10FAD00020460DB0F0BD0A68264B9A42AAD02946AE
:10FAE0002046FFF74DFFF3E7EA0702D50020FEF7B7
:10FAF00071FBAB0706D12B681F4A9342F6D01F4A11
:10FB00009342F3D00E24E3E7012206A92046FFF733
:10FB100085FC012209A92846FFF73CFC0028F1D00A
:10FB2000089A012A1DD05A2A1DDC203201460B9B5F
:10FB3000012B1AD05A2B01DC203301469342D5D138
:10FB400023F00203642BD1D0022E01D00029CDD0A6
:10FB50000A9B0093DDE90612099B304608F053F832
:10FB600086E74222E1E70021E1E74223E4E700BF24
:10FB700034E10508F4E005080CEB0508B4E80508D5
:10FB800070B50646102014460D46F0F771FB054A85
:10FB9000067102604268C46002F0FF02C0E90125FC
:10FBA00070BD00BFF4E005087FB51D46084611464C
:10FBB0004FF00212FEF7C6FD052201A92868FFF7E3
:10FBC000E9FB9DF80C40029E21460022402008F0EF
:10FBD00047FB019AB6FBF0F12046FFF7D1FF044640
:10FBE0002868FFF7CDF80D4B834209D12A68616878
:10FBF0005368C3F3172363F31F216160D368E36085
:10FC00002868032201A9FFF7C5FB18B1237963F027
:10FC10007F032371204604B070BD00BFF4E00508E7
:10FC200070B505460E4601460120FFF721FC2A4625
:10FC300004463146C06819F013FF204670BD00002D
:10FC400038B505460C4610200349FFF78DF8012210
:10FC5000C0E90125C46038BD34E10508136870B5FA
:10FC60006BB94468A51C50F825509C4207D055F844
:10FC70002360B14204D1023350F82330136070BDC9
:10FC80000133F2E72DE9F0410F46124916460446CA
:10FC9000F1F7F3FB06F1040800257368AB4205D8C1
:10FCA00020460D49BDE8F041F1F7E7BB1DB10B4916
:10FCB0002046F1F7E2FB57F8252009492046F1F7E5
:10FCC00095FF58F8041F01222046FFF76DF8013513
:10FCD000E3E700BF5095050878AE0508CB9205080C
:10FCE000519305084B6802330A4651F82310FFF779
:10FCF000C9BF0E3918BF0121490041F00101FEF7CB
:10FD0000A3B8052807D00E3918BF0121490041F0DA
:10FD10000101FDF7D7BA002070470000032A05D182
:10FD20000E2914BF04490549F1F7A7BB0E2914BFDA
:10FD300003490449F8E700BFB88A0508BD8A0508E9
:10FD4000288B0508228B050838B50C46204611463D
:10FD500002221D46FEF7F6FC1CB12868FFF732FAB6
:10FD600008B90E2038BD1E20FCE7062801BFD1E9E6
:10FD700001305840400040F0010018BF002070479B
:10FD800002280AD188689368984208D14868536865
:10FD900098420CBF1E200E207047002070470E2096
:10FDA0007047136813B94068FDF7CEB970472DE965
:10FDB000F84F984602EB43035D1C042B00AF8246CC
:10FDC0008B4616464FEA85051FD8EB1D23F0070327
:10FDD000ADEB030D6C464FF000092046B96A40F8C0
:10FDE00004BB2A1F19F03CFE23464246711C5046B4
:10FDF000FDF7FEFA0446B9F1000F02D04846F0F7CD
:10FE00005FFA2046BD46BDE8F88F2846F0F73BFA7A
:10FE100004460028D9D08146DFE707B50093134692
:10FE20000A46D0E90101FFF7C2FF03B05DF804FB09
:10FE300038B505460C460C200249FEF795FFC0E98F
:10FE4000015438BDB8E1050810B50349044608203F
:10FE5000FEF78AFF446010BDDCE105082DE9F04F94
:10FE6000866806EB010A04460AEB420001EB4209F0
:10FE7000052887B00F46154698464FEA890904F1D0
:10FE80000C0B16D801AFB60032465946384619F069
:10FE9000E7FD4A464146B81919F0E2FD60683B4665
:10FEA0002A465146FDF7A4FA0446204607B0BDE8AD
:10FEB000F08F8000F0F7DCF9A26859469200064600
:10FEC00019F0CEFDA0684A46414606EB800019F0C5
:10FED000C7FDA168606833462A463944FDF788FAB1
:10FEE00004463046F0F7ECF9DFE74068FDF72CB93F
:10FEF0002DE9F041CD1CAD0080460E46284608494C
:10FF00001746FEF731FFA5F10C02C0E90186044651
:10FF100039460C3019F0A4FD2046BDE8F08100BF41
:10FF2000F0E10508D1ED017AF5EE407AF1EE10FA34
:10FF300073B504460D4624D01349144EF1F79DFACB
:10FF40004FF0FF336320CDE9003000231A4695EDD2
:10FF5000010A67212046F1F727FC02224FF0FF3308
:10FF60006321CDE90031204695ED020A0023672187
:10FF7000F1F71AFC3146204602B0BDE87040F1F7B7
:10FF80007CBA034E0022E9E7509505085593050811
:10FF900058930508136810B5144643B940F28643D8
:10FFA000994205D190ED010A01F008FA206010BDD8
:10FFB000B1F5777FFBD190ED020AF5E708B5084966
:10FFC0002DED028B0C20F0EE408AB0EE608AFEF739
:10FFD000CBFEC0ED018A80ED028ABDEC028B08BD2C
:10FFE00020E2050808B5072841D8DFE800F013260D
:10FFF000404004401532D1ED017AF5EE407AF1EE41
:020000040803EF
:1000000010FA36D1D1ED027AF5EE407AF1EE10FA1F
:100010002FD10E21084608BDD1ED027AFDEEE77A18
:1000200017EE903AD1ED017AFDEEE77A17EE902ABD
:1000300053405B0043F00101ECE7D1ED020A91ED82
:10004000010ABDE80840F1EE600AB1EE400AFFF790
:10005000B5BF91ED020AD1ED017A20EE000AA7EEBC
:10006000A70A19F0F9FCBDE8084001F0A7B9002182
:10007000D0E71E21CEE7000030B52DED028B0C46F7
:1000800085B01146204604221D46FEF75BFBF4B105
:10009000012C286826D082074DD102682C4B9A4249
:1000A00049D190ED018AD0ED028A6868830749D171
:1000B0000268274B9A4245D1D0ED027A38EE678A22
:1000C000D0ED017A78EEA70AB0EE480A03E0DFED42
:1000D000210AB0EE600A05B0BDEC028BBDE83040ED
:1000E000FFF76CBF00F00702022A034605D0810724
:1000F00016D1026818498A420FD103A905F01CF9EC
:1001000000230093012303991A46FCF747FB03469B
:10011000184605B0BDEC028B30BD0D498A42F7D0C0
:1001200003AA02A9FEF7A0FFDDED030A9DED020A76
:10013000FFF744FFEBE7FEF757FFDFED068AB0EE6F
:10014000408AB2E7FEF750FF70EE280ABCE700BF16
:1001500020E2050800000000FCF4050843680B607D
:10016000836813607047000010B52DED048B82B0DA
:10017000044601AA08466946B0EE409AB0EE608A8D
:10018000FEF748FF002800F0CC80A01E202800F2D7
:10019000CC80DFE800F0B6CACACACACACACACACA8C
:1001A000CACA11205BCA292CCA68CACACACACA11DB
:1001B000205BCA292CCA6800DDED008ADDED017ADA
:1001C00079EE288A38EE278AF0EE480AB0EE680AFF
:1001D000FFF7F4FEA5E0DDED008ADDED017A79EEB2
:1001E000688A38EE678AEFE75248FDF7D1FFDDED08
:1001F000017A9DED007AF5EE407AF1EE10FAB5EE57
:10020000407A0BD1F1EE10FA03D14B494B48FCF781
:10021000FFFFC9EE078A88EE078AD5E7F1EE10FAEC
:1002200006D1B1EE499AC8EE278A89EE278ACBE734
:1002300067EEA76AF1EE677AE7EE076A87EE266A4D
:1002400087EEA67A8DED006A8DED017A9DED007A3C
:10025000DDED017A68EE678A27EE088AE7EE098A03
:10026000A7EE898AB0E728EE080AA9EE090A19F074
:10027000F3FBB5EE400AF1EE10FADDED019A19D16B
:10028000F5EE409AF1EE10FA12D1DDED007AF5EEBE
:10029000C07AF1EE10FA0BDBF5EE407ADFED287A4A
:1002A000F1EE10FAF7EE008A18BFF0EE678A8BE7DE
:1002B0002449ABE718F036FDF0EE490AF0EE408A2B
:1002C000B0EE480A16F0D6FDDDED007AB0EE408AB9
:1002D00027EE888A29EEC00AA8EEA98AA7EEA80A06
:1002E00018F050FBB0EE409AB0EE480A18F0D8FE75
:1002F00060EE098AB0EE480A19F020FB20EE098A68
:1003000062E7DDED007AF4EE497AF1EE10FA0ED1F3
:10031000DDED017AF4EE487AF1EE10FA0CBF1E2002
:100320000E2002B0BDEC048B10BD0020F9E70E20BA
:10033000F7E700BF5A9305086F93050834E70508EF
:10034000000000007C9305080B46D3ED020A93EDF4
:10035000010A1146FFF708BFD0E902120346C86838
:1003600082420AD00869496850F8220001328A4264
:10037000DA6003D10022DA60704700207047000085
:100380000346084603499A6801600349C260C0E910
:10039000011370475CEE05085903030870B5C56882
:1003A0004268466984686B1C9A4208BF0023F607BE
:1003B00005D5A34203D108490848FCF729FF06697F
:1003C000A34246F82510C36004D101339A4208BF06
:1003D00000238360062070BD279A05085CE60508A7
:1003E000836810B55BB14469C268E40703F1FF3369
:1003F00007D5934205D109490948FCF709FF43682D
:10040000F1E704698360934244F8231003D103B9F0
:100410004368013BC360062010BD00BF279A050852
:100420005CE6050830B585B0054608466946FDF727
:10043000AFF904462046FDF71FFA014610B9062021
:1004400005B030BD2846FFF7A9FFF3E770B50446B5
:100450000E461546CAB1D4E90223991A48BF63680B
:10046000006848BFC91832460023FEF745FEA3685E
:1004700018446368834298BFC01A2369042D0EBFD5
:1004800053F8205043F820500625284670BD000040
:10049000F8B51E460F46044611463846124AFEF786
:1004A00051F97068FEF74AFD051E02DA0020FDF7DB
:1004B000C3FC21461820FEF757FC04460023681CA5
:1004C0006060C4E902338000EFF7EBFE022F206189
:1004D00003D9B068FEF732FD606131682046FFF74E
:1004E000A1FF2046F8BD00BF0600040008B5D0E912
:1004F00002239A4203D107490748FCF789FE03B952
:1005000043680269013B0021C36052F8230042F8AE
:10051000231008BD899305085CE60508042803D06C
:10052000052808D000207047D1E9020398420CBF8B
:100530000E201E207047D1E90230C01A44BF4B681C
:10054000C018400040F0010070470000D0E90231BF
:100550008B4210B5024603D108490948FCF758FE02
:100560000169002451F8230041F823405168013308
:100570008B4208BF2346936010BD00BF89930508D6
:100580005CE60508042803D0052807D00020704742
:100590004B68082B34BF0E201E2070474868C0F3FC
:1005A000DC00400040F00100704700000346054AAF
:1005B0000A601A7A0A715B688B6000230846CB6078
:1005C000704700BF74E30508062802D10B7A022B9E
:1005D00002D04968FFF7D6BF490041F001007047DB
:1005E000044B0B6001230B7100238860CB6008462D
:1005F000704700BF74E3050810B5044904460C2099
:10060000FEF7B2FB02220272446010BD8CE30508C3
:1006100008B503799B0702D50020FDF7B9FD08BD99
:10062000F8B50F6806460D46144612B13846FFF776
:10063000EFFF69682246381DFEF772F9034608B1DC
:10064000406870B9022E05D1022C08D169680748AC
:10065000FDF7C8FDA868012C00D15860F8BD062040
:10066000F9E7022C04BF00225A60F7E738E60508D4
:100670000122FFF7D5BF0222FFF7D2BF0022FFF70A
:10068000CFBF10B50446FFF7C3FF201DFEF735F9B5
:10069000062010BD30B50B6885680246AB4201D319
:1006A00000200AE0D46804EBC30054F8334001335F
:1006B000002CF3D0042CF1D00B6030BD13B50446F0
:1006C00000F10C018068FFF7E5FF60B12379012B91
:1006D0000BD0022B43680AD0026869460220CDE99C
:1006E000002306F023F902B010BD0068FBE71846AE
:1006F000F9E700007FB5174B0A7A0D46044653F818
:100700002210F0F7BAFE14492046F0F7B6FE134B5C
:1007100000932B7A8DF804306B68029300230393C7
:1007200001266846FFF7CAFF054630B90C49204646
:1007300004B0BDE87040F0F7A0BE1EB909492046DC
:10074000F0F79BFE012229462046FEF72DFB0026EE
:10075000E7E700BF68E305088C93050874E3050824
:100760008F930508CB9205081FB50446FFF750FF8D
:100770006368072B03D812491248FCF749FD002291
:1007800001922279510744BFC3F3DC0303F1FF3325
:1007900001A9204648BF0193FFF77CFF6368083B2F
:1007A0006360036802934368039304220023C0E953
:1007B000002302A9022006F0B9F804B010BD00BF62
:1007C0009293050838E605082DE9F74F0B68DFF826
:1007D000F090032A0EBFD0E902ABDFF8E8B0DFF8F3
:1007E000E8A0154618BF01254B450446884605D0AC
:1007F000032D03D0DA882C49F1F7F8F92B4920466C
:10080000F0F73BFE00230193012701A94046FFF7C3
:1008100041FF064680B926492046F0F72EFED8F85B
:1008200000304B453CD0032D3AD02249204603B03E
:10083000BDE8F04FF0F721BE1FB951462046F0F752
:100840001CFE032D2AD1336803F00702022A25D0AB
:1008500013F0030708D11B681A7B2AB103EB82034C
:100860001A69154B9A4204D014492046F0F705FE48
:10087000012731682A462046FEF796FA1FB10F4934
:100880002046F0F7FAFD59462046F0F7F6FD71686C
:100890002A462046FEF788FA0027B6E70027E8E751
:1008A00003B0BDE8F08F00BFAB930508AF93050818
:1008B0005F8F050878AE05087D530308B1930508DE
:1008C0000CE405083CA60508CB92050810B50449C0
:1008D00004460C20FEF748FA00220272446010BD64
:1008E0008CE3050810B5044904460C20FEF73CFAD9
:1008F00001220272446010BD8CE3050810F003036E
:100900000CD10268117A31B102EB81021369044AF9
:100910009A1A5342534103F0010070470023FAE74B
:10092000510A03082DE9F3470C681646074620468E
:100930000D46FFF76DFE3168314AC9083846FDF7AC
:1009400001FF022F12D16F683846FFF7D7FF01462B
:10095000E8B12B689F4209D00023019304F10408F9
:10096000686801A9FFF796FE074640B900250434E0
:100970007368AB4233D8062002B0BDE8F08739680F
:1009800001224046FDF7CCFF7B684360E8E738462C
:10099000FCF7FEFE04F1040A81464846FCF76CFFB2
:1009A0000028E3D00021FCF7F3FE8046FCF764FF4B
:1009B00007464046FCF760FF05464046FCF75CFFF3
:1009C00017B91048FDF738FA002DFAD00028F8D1F1
:1009D000012239465046FDF7A3FF4560DDE7B368C5
:1009E00053F8351003EBC50739B1042905D00122AE
:1009F0002046FDF795FF7B6843600135B8E700BFEF
:100A000005000200B393050810B5002204300C461F
:100A1000FDF786FF18B903482146FDF7E3FB406860
:100A200010BD00BF38E60508024B40F8043BFDF757
:100A300041BF00BF0CE4050838B505461020EFF7AC
:100A400017FC29460446FFF7EFFF204638BD00009B
:100A50002DE9F041804686B000200D4616461F461F
:100A6000FFF7EAFF0F4BC0F80080984502BF0379FB
:100A700043F00403037155EA060304460DD03B68B6
:100A8000019007EB8502314603A80293FDF71FFF93
:100A900003AA01A9681CFFF745FF204606B0BDE880
:100AA000F08100BF3CE40508F8B50C46064600217D
:100AB0006068FCF76DFE022E054660688CBFA66874
:100AC0000626FEF761FB50B9FFF7B6FF0446071D87
:100AD0002846FCF7D1FE014618B92046F8BD401063
:100AE000F2E701223846FDF71BFF4660F0E738B514
:100AF00004468068FFF7A0FF2368626803602379DB
:100B000022F0070203F0050313434360A268E16883
:100B10000546D200C06818F0A3FF284638BD000083
:100B2000F0B5162885B00C46154663D005D80228C6
:100B300010D0092862D0002409E02428FBD100222B
:100B40002946201DFDF7ECFE00282ED10E2420465C
:100B500005B0F0BD02F003038A0728D10A682B49CB
:100B60008A4224D1002BF1D12968914221D1CDE9CB
:100B7000013301A92046FFF78DFD02A9074628464B
:100B8000FFF788FD064677B10028DFD03168386866
:100B9000FEF7B8FB0028D9D071687868FEF7B2FB81
:100BA0000028E6D1D2E70028D0D11E24CFE7002BC1
:100BB000CCD12A68164B9A42C8D163686A68534000
:100BC000072BC3D800230293043502A92046FFF760
:100BD00061FD06460028E8D0316800222846FDF76E
:100BE0009FFE0028B2D041687068FEF78BFB00289A
:100BF000EBD1ABE70846FFF77AFF0446054A02A9A6
:100C00000220CDE90245FFF78DFEA0E73CE4050890
:100C10000CE4050874E4050810B40C7A012C06D124
:100C2000242804D149685DF8044BFFF779BF002000
:100C30005DF8044B70474068C008704770B50446C3
:100C40000E461546FFF7E4FC01223146201DFDF754
:100C500067FE4560204670BD13B50222CDE9000154
:100C6000044669461046FFF7DBFC204602B010BD83
:100C700038B50C461AB9FFF7EFFF06200BE0042A3F
:100C80000AD100220430FDF74BFE18B90448214672
:100C9000FDF7A8FA406838BDFFF7D0FFEDE700BFC9
:100CA00038E6050813B504464068FCF7E5FD58B181
:100CB000A3685A1C5B0043F00103CDE90030A26039
:100CC0006946022005F032FE02B010BD1FB5044691
:100CD000084611461A4602AB01930A4B00930223C1
:100CE000FDF7BAFD21460C20FEF73EF80021044630
:100CF0000298FCF74DFD039B60602046A36004B0A2
:100D000010BD00BF80E40508C3685A68012A70B5A9
:100D100006462AD19D68AB0727D12A68154B9A420F
:100D200023D1EC682378FF2B20D14A20EFF7ABFAD0
:100D3000044638B9104AD2F80832343B492B12D94C
:100D4000946B3434E9682046F0F72AFAEC602046C8
:100D500018F008FF0023A8606B60A9682046F0F730
:100D60007BF8686001E0054BF36070BD6B68002B99
:100D7000FBD1F2E7FCF405087004002008F6050832
:100D8000F8B5164602F07F07320605460C460AD42F
:100D90007B1E012B0DD80B68D888F0F78CF9014623
:100DA0002846F0F76AFB022F03D123492846F0F7C3
:100DB00064FB2046FFF7A8FF16F07D0734D1E368F7
:100DC0000BB15A682AB928461C49BDE8F840F0F72B
:100DD00054BB20681A4988421FD1022A1DD898683E
:100DE000C3071AD509F056FB0346B0B1E2681549AE
:100DF000926828465210F0F7F9FEE3685B68012B11
:100E000019D90D492846F0F738FBE368D9683A4606
:100E10002846BDE8F840FDF7C7BFE3685A68012AD5
:100E200002D199680022F3E7E16832462846BDE81E
:100E3000F84005F001BDF8BD3CA605084BA7050824
:100E4000CCE50508E59305082DE9F8430D46044671
:100E500011462846194A1A4F9846FDF773FC102090
:100E6000EFF711FA002814BF8146B9460023C9F8EC
:100E70000040C9F808302DB9124CC9F80C4048465A
:100E8000BDE8F883AE1CB6003046EFF7FCF9044627
:100E900048B9D7F8E02106F118039A42A7F12807CC
:100EA000EADBBC6B1834084BA6F10802C4E9003534
:100EB000414604F1080018F0D3FDDEE7FEFF010013
:100EC0009804002008F6050844F60508F8B515460C
:100ED000D0E901320F465119994204460FD30178E7
:100EE000D9B105F110061E44C06801223146EFF762
:100EF000E5F978B96568A3682070013DED1AD4E979
:100F000002302A461844394618F0AAFDA3682B443B
:100F1000A360F8BD6660E060F1E7013B9D1AEEE773
:100F2000024B0022C3F808229A6370477004002025
:100F300010B5FEF703F8041E11DDEFF799F903462B
:100F4000084A906BEFF3108172B6C2F808429363BF
:100F500081F3108808B1EFF7B3F9062010BD002324
:100F6000EEE700BF7004002038B50546FDF708FF26
:100F7000007A70B12846FDF703FF04462846FDF7C6
:100F8000FFFE037A04EB8304024B2069C31A584224
:100F9000584138BD490E030810B50446FFF7E4FF79
:100FA00000B92469204610BD10B5FFF7F5FFC368EE
:100FB0005B68044623B1FFF7A7FEE368986810BD9D
:100FC0000620FCE738B513680546144653B140F2D5
:100FD0001F33994205D15368062B02D10023C380E9
:100FE000236038BD3D2903D1FFF78EFEEB68F7E79C
:100FF000A22903D040F2A2339942F2D12846FFF74A
:10100000D3FF2060EDE700231A461946FFF71CBF07
:1010100073B5054610200E46EFF735F9044630B992
:10102000104BD3F80822332A12DD9C6B24340E4B6C
:101030002360304618F096FD0022C4E90206626083
:1010400001AB012128460194FFF7FEFE02B070BDFE
:10105000034602460146284602B0BDE87040FFF74D
:10106000F3BE00BF70040020FCF405082DE9F04336
:1010700006469BB010200D461746EFF704F90446CC
:10108000284618F06FFD00F1010980464846EFF749
:10109000FAF80CB1002848D12549D1F80822432A92
:1010A00029DD886BA2F1340900F1240401213430D8
:1010B00003AB01931F4B02932B78CDF8109081F076
:1010C00001010022FF2BCDE905208DF80C1004D181
:1010D000294607A8F0F764F807AD3A46294601A863
:1010E000F0F7D4FBDDE905320021D154059BA36064
:1010F000069BE3600CE044B9234622462146304675
:101100001BB0BDE8F043FFF79FBE70B9C4E902858C
:101110000022094B2360626007AB0121304607942F
:10112000FFF792FE1BB0BDE8F0830021C0E700BFCF
:1011300070040020CD0E0308FCF405080EB403B5BE
:1011400003AA52F8041B0192FFF790FF02B05DF86A
:1011500004EB03B07047000083070BD10268084B13
:101160009A4207D1037A2BB100EB83031A69054B2E
:101170009A4202D0044906F0BDBB0120704700BF6F
:10118000D8F60508490E030878E8050810B50446A6
:10119000FFF7EAFE50B92046FDF7F2FDFFF7DCFF4E
:1011A00020B12069024BC01A18BF012010BD00BF3A
:1011B0003CF7050838B504460D46FFF7E7FF18B1C0
:1011C0002046FDF7DDFD044629462046BDE83840AF
:1011D00006F090BB2DE9F041884617461E46FFF702
:1011E000DBFE04468068E0B90C20EFF74CF8A06005
:1011F000A8B9164BD3F80822172A0EDD986BA06009
:101200000623A3800023E380E38800EB8302D91C3C
:10121000E18040F82380C2E90176BDE8F081032334
:10122000EFE7E388A5880233AB42EDDB074B9B6B0E
:101230009842F2D003350122A900EFF73FF80028C9
:10124000EBD0A388A0600333A380DDE77004002007
:1012500038B50D461446FFF79FFE83681BB1C28860
:101260002A60236038BD1A46FAE737B50446A068FD
:10127000FCF702FB019068B16568062D05D001AB53
:10128000002201212846FCF7B3F8FDF79BFF002858
:10129000EDD0019803B030BD38B50446084611467C
:1012A0004FF004121D46FDF74DFA21460C20FDF7C4
:1012B0005BFD2B684360044600216868FCF768FA10
:1012C000A060204638BD13B54FF0FF336322CDE94F
:1012D00000320C4694ED010A00234FF4807267211E
:1012E000F0F762FA02B010BD38B52DED048BD0EDE9
:1012F000009A91ED009AB0EE690AF0EE490A0546AF
:101300000C4616F063FB79EEC07AB5EE400AF1EEBA
:1013100010FAC7EE898AB0EE408A21D119EE103A50
:101320009FED248ADFED247A002BB8BFB0EE678AE8
:10133000F5EE408AF1EE10FA29D1C9EE897A9FEDD7
:101340001D0A17EE903ADFED1C7A002BB8BFB0EE05
:10135000670A85ED000A84ED008ABDEC048B38BD78
:10136000B5EEC00AF1EE10FAB5EEC09A4CBF0122FC
:101370000022F1EE10FA4CBF012300239A421EBF57
:10138000F7EE007A30EE098A78EEE78AD0E7B0EE21
:10139000680A17F009FE78EEC08AF6EE007AF4EEDD
:1013A000E78AF1EE10FAC4BFF7EE007A30EE270AB2
:1013B000CFE700BF000000000000008008B5082053
:1013C0002DED028BB0EE408AEEF752FF80ED018AE0
:1013D000BDEC028B014A026008BD00BFB4E80508FD
:1013E00030B50D4687B01146284602221C46FDF74F
:1013F000A9F935B99FED100A07B0BDE83040FFF7F5
:10140000DDBF2068012203A9FDF7C4FF40B100231E
:10141000DDE9030100931A46FBF7C0F907B030BDC0
:101420002068830703D10268044B9A42F6D0FDF787
:10143000DBFDFFF7C3FFF1E700000000B4E805089B
:1014400091ED010A07281DD8DFE800F00A181C1CDE
:10145000041C0C14B5EE400AF1EE10FA14D01E2153
:1014600008467047BDEEC00A10EE103A590041F030
:101470000101F5E710EE103A002BF1DAB1EE400A67
:10148000FFF79CBF0021EBE70E21E9E790ED010A91
:101490007047000030B52DED028B0C4687B0054635
:1014A00003A920468DED010AFDF762FD002800F03A
:1014B000C680232D00F22781DFE815F0E900F50052
:1014C00001010D0119012501250125012501250134
:1014D000250125012501250124002D0034002501C9
:1014E0003B004F005D008F002501250125012501EE
:1014F000250124002D00340025013B004F005D0034
:101500008F00CE00DDED017A9DED037A77EE877ACC
:10151000CDED017A1CE0DDED017A9DED037A77EEE9
:10152000C77AF5E7DDED017A9DED037A67EE877AFC
:10153000EEE7DDED037AF5EE407AF1EE10FA03D135
:1015400072497348FBF764FE03A901A8FFF7CCFEBC
:101550009DED010AFFF732FF71E0DDED037AF5EE54
:10156000407AF1EE10FAEBD0DDED016A86EEA77A53
:101570008DED017AECE79DED038AB5EE408AF1EE40
:1015800010FADDD09DED010AF0EE480A16F01EFAC1
:10159000B5EE400AF1EE10FA0AD118EE103ADFED7E
:1015A0005D7A9FED5D7A002BB8BFF0EE477AAFE72A
:1015B000B5EEC00AF1EE10FAB5EEC08A4CBF0122BA
:1015C0000022F1EE10FA4CBF012300239A4240D0D2
:1015D00038EE008A8DED018ABAE7DDED018A9DEDD6
:1015E000038AF5EE408AF1EE10FA0DD1B5EEC08A0D
:1015F000F1EE10FA08D59FED497AF0EEC87AF4EED4
:10160000477AF1EE10FA9BDDF5EEC08AF1EE10FAA2
:1016100019D5B0EE480A17F0C7FCB4EE480AF1EE4F
:1016200010FA10D0B4EE488AF1EE10FA0BD6DFEDC6
:10163000390A2146B0EE680A2220FEF795FD07B070
:10164000BDEC028B30BDF0EE480AB0EE680A16F031
:10165000E7FE8DED010A7BE7DDED037AF5EE407ADA
:10166000F1EE10FA3FF46CAF03A901A8FFF73CFEBE
:101670009DED010AFFF7A2FE9DED030A0490FFF71E
:101680009DFE04A90590022005F050F9D7E79DEDD5
:10169000017ADDED037AB4EEE77AF1EE10FA4CBF91
:1016A0001E200E20CBE79DED017ADDED037AB4EE2E
:1016B000E77AF1EE10FACCBF1E200E20BFE79DEDB9
:1016C000017ADDED037AB4EE677AF1EE10FA0CBF21
:1016D0001E200E20B3E79DED017ADDED037AB4EE16
:1016E000E77AF1EE10FA94BF1E200E20A7E79DEDD9
:1016F000017ADDED037AB4EEE77AF1EE10FAACBFD1
:101700001E200E209BE7002099E700BF3D910508B1
:1017100034E705080000000000000080FFFF7F7F25
:1017200010B40C4611468A0794ED010A034609D10C
:101730000C68074A944205D1DFED060A5DF8044BB8
:10174000FEF712BD5DF8044B1846FFF7A3BE00BFBD
:1017500020E205080000000010B5044608461146C6
:101760000022FCF7EFFF6368BDE81040184770B532
:101770001C460546084611464FF00212FCF7E2FFF0
:101780006B682068BDE87040184770B505461C4678
:10179000084611464FF00412FCF7D4FFD4E90001CB
:1017A0006B68BDE87040184770B51C460546084692
:1017B00011464FF00612FCF7C5FFD4E901126B6821
